:04000000ADEF00F070
:100008005682D9CF08F0DACF09F00F0112A91BD018
:100018008EBC02D0839483928EA802D083A20ED085
:10002800899425EE04F0010EDBBE07D0000EDE5CDD
:10003800020EDE5802E3899201D089828EB883B21B
:1000480001D08984129912A17CD08EB883B289928A
:10005800901C0A6E8E1C0B6E04C50CF005C50DF0C5
:100068000DBE03D0020E0D5C2FE28EA802D083A233
:100078002BD00C4A0D2A0CC004F50DC005F502C59D
:100088000CF003C50DF0060E0C24D96E050E0D20DC
:10009800DA6E0AC0DFFF060E0C24D96E070E0D209B
:1000A800DA6E0BC0DFFF0C4A0D2A0468010E056EDC
:1000B8000CC006F00DC007F00450061605500716D0
:1000C80006C002F507C003F58EB883B28984898417
:1000D8008EA0FED78EA802D083A202D0899401D028
:1000E800898425EE04F0010EDBBE07D0FE0EDE5C2F
:1000F800010EDE5802E3899201D089820BA81FD035
:100108000BD0838202D0838405D0839418D083A235
:1001180016D08394839213D00A507F0B046E056A1D
:1001280005500DE10450040AF2E0100AF0E0340A28
:10013800E8E01F0AEFE07F0AE6E01F0AE6E00F01A9
:1001480012910E01CA9909C0DAFF08C0D9FF569268
:1001580011000AEF50F07DC0D9FF7EC0DAFFDE6AD9
:10016800DD6A7CC00EF0DCEC48F00EC098F00FC0E1
:1001780099F0000199BF0B0CD8909835D96E993534
:10018800DA6E4E0ED926010EDA22DECFAFF0DDCFC1
:10019800B0F0AF51B01101E10C0C7DC0D9FF7EC0A9
:1001A800DAFFAFC0DEFFB0C0DDFF7F91AFC0D9FF7F
:1001B800B0C0DAFFDF5012E020EE01F0AF51D926CF
:1001C800B051DA22DF509BEC63F00001A46FA4B1B8
:1001D80005D07F51D8A4A4A5000C0A0CAFC0D9FF44
:1001E800B0C0DAFFDF6A20EE01F0AF51D926B05176
:1001F800DA2298C0DFFF20EE01F0AF51D926B051C6
:10020800DA22DF507DEC45F00001A46FA4B1030CA5
:100218007F5102E0A4B50A0CAFC060F0B0C061F035
:10022800636B626B77EC49F060C0ADF061C0AEF013
:10023800040EAD19AE1101E1010CAE5103E1020E3D
:10024800AD5D01E30D0C20EE2BF0AF51D926B05176
:10025800DA22DECFA0F0DECFA1F0DECFA2F0DECF33
:10026800A3F03A0EAF250E6E000EB0210F6E91EC82
:1002780061F0020E0F180E1001E00D0C450E000182
:10028800AF250E6E000EB0210F6E91EC61F00EC01E
:10029800A9F00FC0AAF00001AB6BAC6BA951AA1171
:1002A800AB11AC1110E1530EAF250E6E000EB0214C
:1002B8000F6EDCEC55F00EC0A9F00FC0AAF010C00C
:1002C800ABF011C0ACF0000120EE17F0AF51D92609
:1002D800B051DA22A9C0DEFFAAC0DEFFABC0DEFF44
:1002E800ACC0DEFF20EE3FF0AF51D926B051DA2284
:1002F80010EE02F0AF51E126B051E222DFCFE7FF66
:1003080020EE02F0AF51D926B051DA22DE040AE01D
:1003180020EE02F0AF51D926B051DA22020EDE18D3
:1003280001E00D0CA9C00EF0AAC00FF0ABC010F090
:10033800ACC011F020EE02F0AF51D926B051DA224C
:10034800DF50126E136A146A156AEAEC59F00EC08F
:10035800A9F00FC0AAF010C0ABF011C0ACF020EEAD
:100368003CF0AF51D926B051DA22DF50806F816B53
:1003780020EE09F0AF51D926B051DA2280C0DEFF55
:1003880081C0DDFF20EE09F0AF51D926B051DA2245
:10039800DE50DE10D8B40D0C20EE09F0AF51D9268E
:1003A800B051DA22DECF80F0DDCF81F08269836937
:1003B80020EE09F0AF51D926B051DA22DECF84F011
:1003C800DDCF85F08251842783518523805184179E
:1003D800815185178451851101E00D0C400EAF2520
:1003E8000E6E000EB0210F6E91EC61F0000120EE50
:1003F80007F0AF51D926B051DA220EC0DEFF0FC088
:10040800DDFF20EE07F0AF51D926B051DA22DF50D8
:10041800806F0F0E801701E00D0C420EAF250E6E97
:10042800000EB0210F6E91EC61F00EC09CF00FC071
:100438009DF000019E6B9F6B9C519D119E119F1119
:1004480010E14F0EAF250E6E000EB0210F6EDCECE2
:1004580055F00EC09CF00FC09DF010C09EF011C06A
:100468009FF03D0E0001AF250E6E000EB0210F6EFD
:1004780091EC61F00EC09AF00FC09BF000019A5108
:100488009B1101E10D0C20EE07F0AF51D926B051B8
:10049800DA22DECF80F0DDCF81F0040E826FD890B3
:1004A80081338033822FFBD79A518025836F9B51EC
:1004B8008121846F856BD8B0852B866BA9518325E4
:1004C800946FAA518421956FAB518521966FAC51D9
:1004D8008621976F94519C5D95519D5996519E59CF
:1004E80097519F5901E20D0C94519C5D0E6E9551E8
:1004F8009D590F6E96519E59106E97519F59116EC6
:1005080020EE09F0AF51D926B051DA22DECF80F0C3
:10051800DDCF81F080C012F081C013F0146A156A33
:10052800E2EC5AF00EC0A5F00FC0A6F010C0A7F07C
:1005380011C0A8F00001A551A611A711A81101E149
:100548000D0CAD6BAE6BF60EA55DFF0EA659FF0E3A
:10055800A7590F0EA85903E2AE6B030EAD6FA85151
:10056800A71108E1F60EA55DFF0EA65903E2AE6BD2
:10057800020EAD6FA851A71108E1F60EA55D0F0E8A
:10058800A65903E2AE6B010EAD6FAD51AE1101E19C
:100598000D0C020EA525806F000EA621816F000E9E
:1005A800A721826F000EA821836F20EE13F0AF51B0
:1005B800D926B051DA2280C0DEFF81C0DEFF82C0BA
:1005C800DEFF83C0DEFF20EE1BF0AF51D926B0510D
:1005D800DA22A0C0DEFFA1C0DEFFA2C0DEFFA3C0FA
:1005E800DEFF9A51A025806F9B51A121816F000EDB
:1005F800A221826F000EA321836F20EE1FF0AF515E
:10060800D926B051DA2280C0DEFF81C0DEFF82C069
:10061800DEFF83C0DEFF9451A025806F9551A12194
:10062800816F9651A221826F9751A321836F20EE8B
:1006380027F0AF51D926B051DA2280C0DEFF81C041
:10064800DEFF82C0DEFF83C0DEFF030EAD19AE11F0
:100658004DE1590EAF250E6E000EB0210F6E91ECD4
:1006680061F00E500F1001E00D0C000120EE07F0B4
:10067800AF51D926B051DA22DE50DE1001E00D0C60
:100688005B0EAF250E6E000EB0210F6EDCEC55F040
:10069800000120EE23F0AF51D926B051DA220EC066
:1006A800DEFF0FC0DEFF10C0DEFF11C0DEFF20EE50
:1006B80013F0AF51D926B051DA22DECF80F0DECF69
:1006C80081F0DECF82F0DECF83F0020ED890803743
:1006D800813782378337E82EF9D780C090F081C000
:1006E80091F082C092F083C093F0B8D020EE07F06A
:1006F800AF51D926B051DA22DE50DE1001E10D0CDF
:1007080020EE1FF0AF51D926B051DA22DECF80F0AB
:10071800DECF81F0DECF82F0DECF83F0A9518025D5
:10072800846FAA518121856FAB518221866FAC51AC
:100738008321876F20EE23F0AF51D926B051DA22FA
:1007480084C0DEFF85C0DEFF86C0DEFF87C0DEFF17
:10075800020EAD19AE116BE020EE13F0AF51D926A1
:10076800B051DA22DECF80F0DECF81F0DECF82F02A
:10077800DECF83F0010E8015846F856B866B876BE7
:1007880020EE13F0AF51D926B051DA22DECF88F02F
:10079800DECF89F0DECF8AF0DECF8BF0030E880340
:1007A800F3CF8CF0F4CF8DF08E6B8F6B8903F35001
:1007B8008D27F4508E23000E8F238803F3508D2746
:1007C800F4508E23000E8F23030E8A03F3508E27D6
:1007D800F4508F23000E8903F3508E27F4508F2393
:1007E800000E8803F3508E27F4508F23030E8B03DB
:1007F800F3508F27000E8A03F3508F27000E8903CA
:10080800F3508F27000E8803F3508F27D8908F332B
:100818008E338D338C3384518C25906F85518D2187
:10082800916F86518E21926F87518F2116D020EEBD
:1008380013F0AF51D926B051DA22DECF80F0DECFE7
:1008480081F0DECF82F0DECF83F0D8908035906FD4
:100858008135916F8235926F8335936FFF0E9025A6
:10086800806F010E9121816F000E9221826F000E20
:100878009321836F0A0E05D0D89083338233813356
:100888008033E82EF9D720EE17F0AF51D926B051B2
:10089800DA228051DE5C8151DE588251DE58835164
:1008A800DE5801E20D0C20EE0FF0AF51D926B05101
:1008B800DA22DE68DE68DE68DD68DD52DD5210EEC1
:1008C8000BF0AF51E126B051E222DECFE6FFDECFDA
:1008D800E6FFDECFE6FFDECFE6FF20EE04F0AF5105
:1008E800D926B051DA22800EDF6E030EAD19AE1193
:1008F80001E090D05F0EAF250E6E000EB0210F6E96
:1009080091EC61F00E040F1001E084D0AFC03AF012
:10091800B0C03BF0010E0001A0253C6E000EA121E5
:100928003D6E000EA2213E6E000EA3213F6ED1EC5B
:1009380056F000096FE1000120EE04F0AF51D9260E
:10094800B051DA22DF6A2D0EAF250E6E020EB021ED
:100958000F6E91EC61F0550E0E185CE1AA0E0F189F
:1009680059E12F0E0001AF250E6E000EB0210F6E5B
:10097800DCEC55F0520E0E184DE1520E0F184AE1FC
:10098800610E101847E1410E111844E1130E0001E1
:10099800AF250E6E020EB0210F6EDCEC55F0720E14
:1009A8000E1838E1720E0F1835E1410E101832E1B9
:1009B800610E11182FE1170E0001AF250E6E020E01
:1009C800B0210F6EDCEC55F0000120EE0FF0AF51B6
:1009D800D926B051DA220EC0DEFF0FC0DEFF10C0EC
:1009E800DEFF11C0DEFF1B0EAF250E6E020EB0211A
:1009F8000F6EDCEC55F0000120EE0BF0AF51D9265C
:100A0800B051DA220EC0DEFF0FC0DEFF10C0DEFFDD
:100A180011C0DEFFAFC0D9FFB0C0DAFFADC0DFFF45
:100A280001014C4B4D2B000120EE05F0AF51D926AA
:100A3800B051DA224CC1DEFF4DC1DDFF000C77C09A
:100A48007AF078C07BF00101426B436B96D376C095
:100A580060F07A0E0001616F79C062F06151D96E61
:100A6800DA6ADECFF6FFDDCFF7FFF86A000EF86E20
:100A78000800F550250AD8A45ED36151D96EDA6A08
:100A8800DE2A000EDD220101446B456B4C6A4D6A7B
:100A98004669476900016151D96EDA6ADECFF6FF0F
:100AA800DDCFF7FFF86A000EF86E0800F550640A0B
:100AB800D8B40FD06151D96EDA6ADECFF6FFDDCF38
:100AC800F7FFF86A000EF86E0800F550690AD8A416
:100AD8007DD16151D96EDA6ADE2A000EDD226251BB
:100AE800D96EDA6ADF50DF2ADF2AD96EDA6ADECFFA
:100AF80065F0DDCF66F0000E66BFFF0E676F686FAA
:100B0800696F6A6F6B6F6C6F60C028F065C029F001
:100B180066C02AF067C02BF068C02CF069C02DF0C1
:100B28006AC02EF06BC02FF06CC030F029C041F0C5
:100B38002AC042F02BC043F02CC044F02DC045F031
:100B48002EC046F02FC047F030C048F048AE02D063
:100B5800010E01D0000E3F6E406A3F504010D8B4DD
:100B680010D0481E471E461E451E441E431E421EE8
:100B7800416C000E4222432244224522462247224B
:100B88004822010147BF01D04C9247BF05D04751C9
:100B980007E14605D8B004D03C6A010E3B6E04D08C
:100BA80046C13BF047C13CF044C13DF045C13EF071
:100BB8003F504010D8A402D04CA403D03D06D8A082
:100BC8003E064A6A1F0E496E02018F6B6ED04906B7
:100BD800D8A04A06700E4924D96E020E4A20DA6E51
:100BE80041C00EF042C00FF043C010F044C011F0F5
:100BF80045C012F046C013F047C014F048C015F0C5
:100C08000A0E166E176A186A196A1A6A1B6A1C6A2B
:100C18001D6AE7EC4CF00EC031F00FC032F010C086
:100C280033F011C034F012C035F013C036F014C0E0
:100C380037F015C038F031C020F033C021F0DCECBB
:100C480061F02050300FDF6E3B06D8A03C063D0611
:100C5800D8A03E0641C00EF042C00FF043C010F0CD
:100C680044C011F045C012F046C013F047C014F05C
:100C780048C015F00A0E166E176A186A196A1A6AB9
:100C88001B6A1C6A1D6A3AEC48F00EC041F00FC09E
:100C980042F010C043F011C044F012C045F013C038
:100CA80046F014C047F015C048F04ABE1FD04A505D
:100CB80003E14904D8A01AD041504210431044100F
:100CC8004510461047104810D8A481D73CBE05D01F
:100CD8003C5002E13B04D8B07AD73EBE07D03E5024
:100CE80003E13D04D8A002D04CB271D73F50401068
:100CF800D8A402D04CA415D04906D8A04A063F5023
:100D08004010D8A403D03A6A2B0E02D03A6A2D0EAE
:100D1800396E700E4924D96E020E4A20DA6E39C037
:100D2800DFFF28C01DF0700E49241E6E020E4A20F7
:100D38001F6E3DC020F03EC021F04CA008D01EC060
:100D480017F01FC018F01DC019F0F4EC61F021BEB7
:100D580005D020C025F021C026F002D0256A266AD9
:100D6800236A246A0AD0000E106E200E0F6E1DC072
:100D780011F063EC59F0234A242A2550235C2450AF
:100D8800800A226E2650800A2258D8A0ECD74CB090
:100D980008D01EC017F01FC018F01DC019F0F4ECE1
:100DA80061F01EC00EF01FC00FF09CEC5FF02550E4
:100DB8000E241D6E26500F201E6E1DC028F01EC06A
:100DC80029F028C060F029C061F0CFD16151D96EF7
:100DD800DA6ADECFF6FFDDCFF7FFF86A000EF86EAD
:100DE8000800F550780AD8B40FD06151D96EDA6A84
:100DF800DECFF6FFDDCFF7FFF86A000EF86E0800C9
:100E0800F550580AD8A46CD16151D96EDA6ADECF90
:100E1800F6FFDDCFF7FFF86A000EF86E0800F5CF91
:100E280075F06151D96EDA6ADE2A000EDD22625150
:100E3800D96EDA6ADF50DF2ADF2AD96EDA6ADECFA6
:100E480063F0DDCF64F063C06DF064C06EF06F6B6B
:100E5800706B716B726B736B746B60C027F06DC0D5
:100E680028F06EC029F06FC02AF070C02BF071C056
:100E78002CF072C02DF073C02EF074C02FF075C026
:100E880030F0010147BF01D04C9247BF05D0475110
:100E980007E14605D8B004D03A6A010E396E04D08D
:100EA80046C139F047C13AF044C143F045C144F066
:100EB8004CA804D0FE0E4326FF0E442228C03BF067
:100EC80029C03CF02AC03DF02BC03EF02CC03FF0BA
:100ED8002DC040F02EC041F02FC042F0486A1F0ECE
:100EE800476E02018F6B6DD04706D8A048060F0EDB
:100EF8003B14456E466A46BE08D0465004E10A0EC9
:100F0800455CD8A002D0570E01D0300E4526000E01
:100F18004622BF0E316E32683050336E346A31501B
:100F2800332632503422345005E11A0E335C02E283
:100F3800010E01D0000E356E366A35503610D8B421
:100F480025D09F0E316E3268200E4510336E000E8C
:100F58004610346E3150332632503422345005E175
:100F68001A0E335C02E2010E01D0000E376E386AA9
:100F780037503810D8B40AD045C014F046C015F020
:100F880059EC5FF014C045F015C046F0700E4724C8
:100F9800D96E020E4820DA6E45C0DFFF3906D8A0A8
:100FA8003A064306D8A04406040E316ED890423261
:100FB800413240323F323E323D323C323B32312EBA
:100FC800F5D748BE20D0485004E1020E475CD8A0AF
:100FD8001AD03B503C103D103E103F1040104110BD
:100FE8004210D8A481D73ABE05D03A5002E139045C
:100FF800D8B07AD744BE07D0445003E14304D8A000
:1010080002D04CB271D74CA816D04706D8A04806D3
:10101800700E4724D96E020E4820DA6E30C0DFFF0A
:101028004706D8A04806700E4724D96E020E4820FD
:10103800DA6E300EDF6E27C01DF0700E47241E6E6C
:10104800020E48201F6E43C020F044C021F04CA07F
:1010580008D01EC017F01FC018F01DC019F0F4EC1E
:1010680061F021BE05D020C025F021C026F002D0B5
:10107800256A266A236A246A0AD0000E106E200E9A
:101088000F6E1DC011F063EC59F0234A242A255035
:10109800235C2450800A226E2650800A2258D8A049
:1010A800ECD74CB008D01EC017F01FC018F01DC0F8
:1010B80019F0F4EC61F01EC00EF01FC00FF09CECAC
:1010C8005FF025500E241D6E26500F201E6E1DC089
:1010D80027F01EC028F027C060F028C061F045D076
:1010E8006151D96EDA6ADECFF6FFDDCFF7FFF86A15
:1010F800000EF86E0800F550250AD8A413D06151E7
:10110800D96EDA6ADE2A000EDD22000E106E250E78
:101118000F6E60C011F063EC59F00001616B010EB5
:10112800606F23D06151D96EDA6ADE2A000EDD22A3
:10113800606B616B1AD06151D96EDA6ADECFF6FF47
:10114800DDCFF7FFF86A000EF86E0800F5500F6E55
:10115800106A60C011F063EC59F000016151D96E5A
:10116800DA6ADE2A000EDD22D8D7000160510101BB
:10117800422700016151010143237AC0F6FF7BC079
:10118800F7FF0800F55001E062D442C176F043C190
:1011980077F012000F6E0E6ACED20F5009E151504F
:1011A80007E00E6A01014B6B0A0EB1D083903CD365
:1011B800020E0F1807E1515005E00E6A01014B6B52
:1011C800140EA5D01F0E0F6438D0300E0F6035D026
:1011D800515033E00F50E00F526E0E6A0F0E521846
:1011E80005E15BC150F001015B6BA1D25250220DA9
:1011F8000A0EF324D96E030EF420DA6EDE50DE10E8
:10120800DE10DE1003E0030E526491D2526A010E22
:10121800506E52501C0D1B0EF324D96E020EF42092
:10122800DA6E52501C0D1B0EF324E16E020EF420F0
:10123800E26EE7501009DF6E7AD23F0E0F6428D0B5
:10124800480E0F6025D0515023E052501C0D000E5F
:10125800F324D96E020EF420DA6E0F50C00FDF6E41
:1012680052501C0D000EF324D96E020EF420DA6ED3
:10127800DF500CE052501C0D1B0EF324D96E020EE9
:10128800F420DA6E100EDF6E010E506E0E6A4FD229
:10129800480E0F1808E1515006E00E6A120E0101BF
:1012A8004B6FC00E34D0310E0F1807E1515005E0D6
:1012B8000C0E01014B6F1D0E23D2340E0F1807E1DF
:1012C800515005E001014A6B4B6B0E6A6FD7350E22
:1012D8000F1808E1515006E00E6A0D0E01014B6F20
:1012E800AC0E15D0370E0F1808E1515006E0838078
:1012F8000E0E01014B6F750E03D20D0E0F1809E18A
:10130800515007E00E6A020E01014B6FBC0E4A6F86
:101318004DD7100E0F1807E1515005E0030E0101DB
:101328004B6FE90EEDD1180E0F1807E1515005E08B
:10133800070E01014B6F090EE3D13B0E0F1807E1B1
:10134800515005E00E0E01014B6F7E0ED9D13E0EB5
:101358000F1801E069D2515001E166D20F0E010168
:101368004B6F3D0ECDD152501C0D010EF324D96E9A
:10137800020EF420DA6E0FC0DFFF030E01014B6F7F
:10138800EA0EBED152501C0D020EF324D96E020E85
:10139800F420DA6E0FC0DFFF030E01014B6FEB0E76
:1013A800AFD152501C0D030EF324D96E020EF42057
:1013B800DA6E0FC0DFFF030E01014B6FEC0EA0D1F8
:1013C80052501C0D040EF324D96E020EF420DA6E6E
:1013D8000FC0DFFF030E01014B6FED0E91D152508C
:1013E8001C0D050EF324D96E020EF420DA6E0FC020
:1013F800DFFF030E01014B6FEE0E82D152501C0D20
:10140800060EF324D96E020EF420DA6E0FC0DFFF49
:1014180052501C0D060EF324D96E020EF420DA6E1B
:10142800DF50606F60C061F0626B636B646B63C0B8
:1014380064F062C063F061C062F0616B61C065F026
:1014480062C066F063C067F064C068F0696B68BF2B
:10145800696969C06AF069C06BF069C06CF0525084
:101468001C0D050EF324D96E020EF420DA6EDF503F
:101478006D6F6DC06EF06F6B706B716B6FC071F0DC
:101488006EC070F06F6B6E6B6EC072F06FC073F0F1
:1014980070C074F071C075F0766B75BF766976C0F0
:1014A80077F076C078F076C079F052501C0D040EB3
:1014B800F324D96E020EF420DA6EDF507A6F7AC008
:1014C8007BF07C6B7D6B7E6B7BC07EF07D6B7C6B79
:1014D8007B6B7BC07FF07CC080F07DC081F07EC0DC
:1014E80082F0836B82BF836983C084F083C085F0F8
:1014F80083C086F052501C0D030EF324D96E020EE1
:10150800F420DA6EDF50876F87C088F0896B8A6BAA
:101518008B6B8C6B8D6B8E6B8F6B200ED890883796
:1015280089378A378B378C378D378E378F37E82E48
:10153800F5D77F518825906F80518921916F81510E
:101548008A21926F82518B21936F83518C21946FE2
:1015580084518D21956F85518E21966F86518F21EB
:10156800976F72519025986F73519121996F7451AB
:1015780092219A6F755193219B6F765194219C6F9C
:10158800775195219D6F785196219E6F79519721BA
:101598009F6F65519825A06F66519921A16F67517A
:1015A8009A21A26F68519B21A36F69519C21A46F56
:1015B8006A519D21A56F6B519E21A66F6C519F2189
:1015C800A76F52501C0D070EF324D96E020EF4209B
:1015D800DA6EA0C0DEFFA1C0DEFFA2C0DEFFA3C09E
:1015E800DEFFA4C0DEFFA5C0DEFFA6C0DEFFA7C0E9
:1015F800DEFF839001014A6B4B6B16D152501C0DD4
:101608001A0EF324D96E020EF420DA6E0FC0DFFF33
:10161800070E01014B6F0A0E73D052501C0D190EA4
:10162800F324D96E020EF420DA6E0FC0DFFF070E26
:1016380001014B6F0B0E64D052501C0D180EF32491
:10164800D96E020EF420DA6E0FC0DFFF070E01011B
:101658004B6F0C0E55D052501C0D170EF324D96E3B
:10166800020EF420DA6E0FC0DFFF61D001014A6B71
:101678004B6B506A9BD50FC030F10F0E01014B6FB9
:101688003E0E3ED00FC031F10F0E01014B6F3F0EE1
:1016980037D00FC032F10F0E01014B6F400E30D022
:1016A8000FC033F10F0E01014B6F410E29D00FC04F
:1016B80034F10F0E01014B6F420E22D00FC035F1ED
:1016C8000F0E01014B6F430E1BD00FC036F10F0EEA
:1016D80001014B6F440E14D00FC037F128D00C0E07
:1016E80001014B6F1E0E0CD00C0E01014B6F1C0E2E
:1016F8004A6F0A0E0E6E5AD50E0E01014B6F760E0A
:101708004A6F92D001014A6B4B6B090E0E6E8380B3
:101718008BD00F500CE052501C0D1B0EF324D96EC9
:10172800020EF420DA6E080EDF6E010E506E010113
:101738004A6B4B6B3BD54AC160F04BC161F000016D
:10174800615113E0030A15E0040A27E00B0A33E0AD
:10175800010A37E0030A3BE0010A42E01D0A5AE0A9
:101768000E0A5DE03B0A5EE05FD0605101E115D5ED
:101778005BD06051E90A01E1F6D5030A01E102D61E
:10178800010A01E10ED6070A01E11AD6010A01E1B0
:1017980026D6030A01E132D647D06051090A01E191
:1017A8002DD7030A01E139D7010A01E145D7070A14
:1017B80001E151D739D060511D0A91E0030A94E044
:1017C80033D06051480A01E115D7E40A2DD06051A1
:1017D800750A92E0030A96E0080A01E147D724D087
:1017E80060513D0A01E147D7030A01E14BD7010ADD
:1017F80001E14FD77F0A01E153D7010A01E157D729
:10180800030A01E15BD7010A01E15FD7070A01E199
:1018180063D70AD06051C00A01E17BD705D0605177
:101828002A0A02D060510F0A0E501200A0C0B6F06A
:10183800A1C0B7F0A451D96EDA6ADE6ADD6A9EC02B
:101848000FF09FC010F0C60E116E86EC55F0000127
:10185800B56FB5510AE120EE0FF09E51D9269F5180
:10186800DA22DF50B56FB55102E0B551120020EE13
:101878000EF09E51D9269F51DA22DFA2070C20EEE6
:1018880010F09E51D9269F51DA2210EE10F09E5189
:10189800E1269F51E222E6CFA9F0E6CFAAF0E6CFF3
:1018A800ABF0E6CFACF0A251A925AD6FA351AA21A8
:1018B800AE6F000EAB21AF6F000EAC21B06FDE50E3
:1018C800AD5DDE50AE59DE50AF59DE50B05901E380
:1018D800DFD220EE10F09E51D9269F51DA22DECFBA
:1018E800A5F0DDCFA6F0A51DA26FA61DA36FD0D2CF
:1018F80020EE10F09E51D9269F51DA22FF0EDE14F9
:10190800A56F010EDE14A66F000EDE14A76F000E81
:10191800DE14A86FA551A611A711A81101E0FDD1E9
:1019280020EE10F09E51D9269F51DA22DECFA5F085
:10193800DECFA6F0DECFA7F0DECFA8F00A0E05D0E6
:10194800D890A833A733A633A533E82EF9D7A969C9
:10195800AA6920EE09F0C651D926C751DA22DECF8E
:10196800ABF0DDCFACF0A951AB27AA51AC23A55100
:10197800AB15B86FA651AC15B96FB81101E091D08D
:1019880020EE10F09E51D9269F51DA22DE50DE104B
:10199800DE10DE101EE120EE06F09E51D9269F5182
:1019A800DA22DECFC0F0DECFC1F0DECFC2F0DECF6C
:1019B800C3F0C051C111C211C31127E19EC081F00B
:1019C8009FC082F0836B846B856B866BACEC25F0D3
:1019D80014D09EC081F09FC082F020EE14F09E517A
:1019E800D9269F51DA22DECF83F0DECF84F0DECF16
:1019F80085F0DECF86F0ACEC25F081C0C0F082C067
:101A0800C1F083C0C2F084C0C3F0C051C111C2117B
:101A1800C31101E141D2C005C111C211C31109E1CD
:101A280020EE0FF09E51D9269F51DA22020EDF6E6A
:101A3800020CC0290FE1C1290DE1C2290BE1C3291C
:101A480009E120EE0FF09E51D9269F51DA22010EAE
:101A5800DF6E010C20EE14F09E51D9269F51DA2238
:101A6800C0C0DEFFC1C0DEFFC2C0DEFFC3C0DEFFF4
:101A780020EE06F09E51D9269F51DA22DE50DE1064
:101A8800DE10DE100EE120EE06F09E51D9269F51A1
:101A9800DA22C0C0DEFFC1C0DEFFC2C0DEFFC3C0A5
:101AA800DEFF20EE18F09E51D9269F51DA2210EE63
:101AB8002BF0C651E126C751E222DE50E61812E1AA
:101AC800DE50E6180FE1DE50E6180CE1DE50E618AD
:101AD80009E1C6C027F0C7C028F03BEC46F0000972
:101AE80001E053D1C6C00EF0C7C00FF0000120EED0
:101AF80014F09E51D9269F51DA22DECF10F0DECFA6
:101B080011F0DECF12F0DECF13F075EC4DF00EC001
:101B1800BCF00FC0BDF010C0BEF011C0BFF0000196
:101B2800BC51BD11BE11BF1101E17AD7B851BC2714
:101B3800B951BD23000EBE23BF23A2C0A5F0A3C088
:101B4800A6F0090EA76FD890A633A533A72FFBD709
:101B5800A5C0BAF0A6C0BBF0BA51BB1101E1A2D032
:101B6800BA51B825A56FBB51B921A66F20EE09F06F
:101B7800C651D926C751DA22A551DE5CA651DE58D6
:101B880010E220EE09F0C651D926C751DA22DECF7D
:101B9800A5F0DDCFA6F0B851A55DBA6FB951A65929
:101BA800BB6FB6C01DF0B7C01EF0BCC01FF0BDC0F3
:101BB80020F0BEC021F0BFC022F0BAC023F0BBC0E5
:101BC80024F020EE01F0C651D926C751DA22DF50A1
:101BD80068EC52F0000901E0D8D00001BA51A56FB5
:101BE800BB51A66FA76BA86B20EE2BF0C651D92668
:101BF800C751DA22DECFA9F0DECFAAF0DECFABF0F4
:101C0800DECFACF0BC51A95DAD6FBD51AA59AE6F26
:101C1800BE51AB59AF6FBF51AC59B06FA551AD5D57
:101C2800A651AE59A751AF59A851B0592CE22F0E61
:101C3800C6250E6E000EC7210F6E20EE2BF0C65182
:101C4800D926C751DA22DECFA5F0DDCFA6F0BC51E8
:101C5800A55FBD51A65B090ED890A537A637E82E1B
:101C6800FBD7A551B625106EA651B721116E020EED
:101C7800136E126ABDEC5FF020EE03F0C651D92650
:101C8800C751DA22DF6ABAC0A5F0BBC0A6F0090EB8
:101C9800D890A537A637E82EFBD7A5C0C4F0A6C0B4
:101CA800C5F0A7D020EE0AF09E51D9269F51DA221E
:101CB80010EE10F09E51E1269F51E222DE50E65CC4
:101CC800DE50E658DE50E658DE50E65818E3C6C047
:101CD80027F0C7C028F03BEC46F0000901E055D0DA
:101CE800000120EE2BF0C651D926C751DA22BCC01C
:101CF800DEFFBDC0DEFFBEC0DEFFBFC0DEFF20EEE0
:101D080018F09E51D9269F51DA22BCC0DEFFBDC013
:101D1800DEFFBEC0DEFFBFC0DEFFA569010EA66FF5
:101D280020EE10F09E51D9269F51DA22DECFA7F07F
:101D3800DDCFA8F0A551A717A651A817A7510008ED
:101D4800C46FA851D8A0E82A0208C56FC451A25D83
:101D5800C551A35904E2A2C0C4F0A3C0C5F0C6C0CF
:101D68003AF0C7C03BF020EE18F09E51D9269F519B
:101D7800DA22DECF3CF0DECF3DF0DECF3EF0DECF24
:101D88003FF0D1EC56F0000902E000015AD60001FC
:101D9800A569010EA66F20EE10F09E51D9269F511D
:101DA800DA22DECFA7F0DDCFA8F0A551A717A651FC
:101DB800A817C6C0A9F0C7C0AAF0A751A927A8515B
:101DC800AA232F0EA9250E6E000EAA210F6EB6C0EB
:101DD80010F0B7C011F0C4C012F0C5C013F0BDECCC
:101DE8005FF020EE03F0C651D926C751DA22010E62
:101DF800DF6EC451A25FC551A35BA451D96EDA6AE4
:101E0800C451DE26C551DD22C451B627C551B723BA
:101E180020EE10F09E51D9269F51DA22C451DE26B9
:101E2800C551DE22000EDE22DE2220EE10F09E5189
:101E3800D9269F51DA2210EE0AF09E51E1269F51D1
:101E4800E222DE50E65CDE50E658DE50E658DE5010
:101E5800E65820EE0AF0D8A020EE10F09E51D926C0
:101E68009F51DA22DECFB1F0DECFB2F0DECFB3F091
:101E7800DECFB4F020EE0AF09E51D9269F51DA2227
:101E8800B1C0DEFFB2C0DEFFB3C0DEFFB4C0DEFF0C
:101E9800A251A31101E02CD520EE0EF09E51D926B7
:101EA8009F51DA22000EDB8C000C0F6A0E6A4EEC92
:101EB80063F00101F36F5F6B0F010D6B156B1D6B09
:101EC800226B070E8C6E010E0101F46F656B0F0E0D
:101ED8000F01596F116B196B216B266B2E6B0E6BF3
:101EE800166B1E6B236B2B6B886889688A688A8ED1
:101EF800889088928382020E026E7AEC62F088944F
:101F08008384889C839C889E838E8B688968CE0E88
:101F180000019C6FF90E9D6FAC0E9E6FFF0E9F6FB8
:101F2800D00EA06FFE0EA16F2F0EA26FFF0EA36F33
:101F380070EC63F08A988588ABEC61F0A20E000122
:101F48009C6FFB0E9D6FF3C19EF09F6B70EC63F06E
:101F58000101F32901E1F36B0F0EF31784EC4EF046
:101F68000101F36FBA0E00019C6FFB0E9D6FF3C168
:101F78009EF09F6B70EC63F00400520E0101BA6F83
:101F88002B0EB96F000EE82EFED7B92FFCD7BA2F4B
:101F9800FAD700F0D250F00B0109D26ED09E0E0194
:101FA800C691CF0ECF16CF82CF80C2890F01138181
:101FB80013891489F28E0E01BA893AEC5CF0839287
:101FC8008394F5EC51F0F5EC51F0000E0E6E340EE2
:101FD800C2EC5EF04A0E126EFF0E136E6AEC5AF0F7
:101FE800AC0E126EFF0E136E6AEC5AF0000E0E6EF7
:101FF800390EC2EC5EF08FA22FD0290E0101BA6F04
:10200800960EB96F7F0EE82EFED7B92FFCD7BA2FE0
:10201800FAD7000E0E6E800EC2EC5EF0430E126E02
:10202800FE0E136E6AEC5AF017D0850E00019C6FF5
:10203800FE0E9D6F8FCF9EF09F6B70EC63F0290EA4
:102048000101BA6F960EB96F7F0EE82EFED7B92F31
:10205800FCD7BA2FFAD704008FB2E7D783800400E1
:1020680059EC4CF00101BF6FDDEC33F00101BF6F9B
:10207800F4050EE163510CE1700E00019C6FFD0E3A
:102088009D6F70EC63F0020E0101636F220E626FA8
:10209800F4510EE163510CE1600E00019C6FFD0EDE
:1020A8009D6F70EC63F0010E0101636F040E626FA7
:1020B8005E5102E00DEC43F0C8C193FF18EC2FF01D
:1020C800CFEC54F0000E0E6E800EC2EC5EF08FEC7A
:1020D80062F0000E0E6E800EC2EC5EF00101F3514C
:1020E8000F0D350EF324126E0D0EF420136E6AECEC
:1020F8005AF0010165BF96EC47F00101BE6BC36B56
:10210800000EC16F010EC06FC1BF05D0C15166E19D
:10211800040EC05D63E20F0EC003F3CFB9F1F4CF34
:10212800BAF1C103F350BA27250EB9250E6E0E0E6B
:10213800BA210F6E9CEC5FF00F5003E1030E0E5CAA
:1021480049E3CD0E00019C6FFD0E9D6F0F0E01013E
:10215800C003F3CFB9F1F4CFBAF1C103F350BA27F2
:10216800250EB92500019E6F0E0E0101BA2100014E
:102178009F6F70EC63F0220E0101C003F3CFB9F139
:10218800F4CFBAF1C103F350BA27000EB925000104
:10219800CE6F030E0101BA210001CF6F0F0E0101AE
:1021A800C003F3CFBBF1F4CFBCF1C103F350BC279C
:1021B800250EBB250001D06F0E0E0101BC210001C8
:1021C800D16F030ED26F43EC15F00101BF6FBF5101
:1021D80071EC5EF00101C04BC12B96D7600502E19E
:1021E800070E8C6E020E601901E02FD10F01108BC3
:1021F800070E2D6F2AD18EA8899435EC5FF02150F7
:10220800221001E1F6D0C3C1BDF1C20E0E6E010E5F
:102218000F6E1FEC59F00101C36FC2B9C39F65511E
:102228001BE0350EC31907E1FC0E00019C6FF90E87
:102238009D6F70EC63F0380E00019C6FFF0E9D6F70
:10224800C3C19EF09F6B0101010EC2A9000E0001DF
:10225800A06FA16B70EC63F00101C2A931D0600ED0
:10226800C3192EE15F0EBD192BE1520E00019C6FC0
:10227800FF0E9D6F70EC63F002500209026EFE0EB5
:102288009C6FFE0E9D6F63C19EF09F6B62C1A0F0B4
:10229800A16B70EC63F02BEE35F063C1DFFF2BEE22
:1022A80036F062C1DFFF8384020E1DEC5BF083947D
:1022B80002920101686B27EC63F00101C36BC5D082
:1022C800F45147E0C251100B0001C26F000EC36FFA
:1022D8000101C35187EC3DF0C2C0C4F1C3C0C5F1D0
:1022E800080E0101C419C51101E100F0070E010132
:1022F800C419C51102E141EC5DF0C405C51102E144
:102308001FEC57F0020E0101C419C51102E198EC47
:102318003BF0030E0101C419C51104E199EC2BF03F
:102328000101BE6F050EC419C51104E177EC3EF03A
:102338000101BE6F090EC419C51102E12BEC55F05D
:102348000A0E0101C419C51101E07FD0A1EC63F0A8
:102358007CD0C2C121F0226AC3510BEC18F021C015
:10236800C4F122C0C5F1070E0101C419C51102E16B
:10237800DDEC5CF0020EC419C51102E1A7EC5AF0BD
:10238800C405C51102E12BEC1DF0030EC419C511DB
:1023980002E14AEC53F0040EC419C51102E1D2EC73
:1023A80060F0050EC419C51102E1FFEC4DF0060EF0
:1023B8000101C419C51102E1A9EC63F0080EC419A2
:1023C800C51102E191EC3CF0090EC419C51102E1F6
:1023D80080EC51F00A0E0101C419C51102E13EEC6E
:1023E80060F00C0E0101C419C5112FE15CEC32F04C
:1023F8002CD084EC4EF001015F6F605126E0F35160
:102408005F1923E0838E000E0E6EC00EC2EC5EF0E4
:102418008FEC62F0000E0E6EC00EC2EC5EF0F30E92
:10242800126EFE0E136E6AEC5AF05FC1F3F1000EE5
:1024380000016D6F030E6E6F7BEC60F0DDEC33F026
:1024480001015E5102E00DEC43F08FB22ED0050E73
:102458000101BE192AE0CFD6850E00019C6FFE0E41
:102468009D6F8FCF9EF09F6B70EC63F0290E01017A
:10247800BA6F960EB96F7F0EE82EFED7B92FFCD72C
:10248800BA2FFAD70400000E0E6EC00EC2EC5EF032
:102498008FEC62F0000E0E6EC00EC2EC5EF06A0E9B
:1024A800126EFF0E136E6AEC5AF08FB2D5D7090E72
:1024B8000101BA6F1E0EB96FE40EE82EFED7B92FD0
:1024C800FCD7BA2FFAD700F0839483920001B16B3E
:1024D800B26BFE0EB36FF90EB46FB56B49EC58F0E2
:1024E800BED59EC00FF09FC010F0BC0E116E86ECDA
:1024F80055F00001BE6FBE5108E120EE0FF09E516D
:10250800D9269F51DA22DF50BE6FBE5102E0BE517C
:10251800120020EE0AF09E51D9269F51DA22A051CE
:10252800DE5CA151DE58A251DE58A351DE5816E2F6
:1025380020EE0EF09E51D9269F51DA22DFB20ED03E
:1025480020EE0AF09E51D9269F51DA22DECFA0F064
:10255800DECFA1F0DECFA2F0DECFA3F020EE10F0A8
:102568009E51D9269F51DA22DECFB4F0DECFB5F0E6
:10257800DECFB6F0DECFB7F0B86BB96BBA6BBB6B1A
:1025880020EE10F09E51D9269F51DA22B8C0DEFF06
:10259800B9C0DEFFBAC0DEFFBBC0DEFFA051A1118B
:1025A800A211A31101E100D220EE09F0BC51D926F5
:1025B800BD51DA22DECFA4F0DDCFA5F0A451A66F7D
:1025C800A551A76FA86BA96B090ED890A637A73796
:1025D800A837A937E82EF9D7A6C0BFF0A7C0C0F022
:1025E800A8C0C1F0A9C0C2F0B451B511B611B71155
:1025F80001E196D0FF0EA0250E6EFF0EA1210F6EF1
:10260800FF0EA221106EFF0EA321116EBFC012F0A3
:10261800C0C013F0C1C014F0C2C015F0E2EC5AF00B
:102628000EC0A4F00FC0A5F010C0A6F011C0A7F00E
:10263800FF0E0001B4250E6EFF0EB5210F6EFF0EC2
:10264800B621106EFF0EB721116EBFC012F0C0C0C8
:1026580013F0C1C014F0C2C015F0E2EC5AF00E50ED
:102668000001A45D0F50A5591050A6591150A75943
:1026780057E3FF0EBF25A46FFF0EC021A56FFF0E05
:10268800C121A66FFF0EC221A76FA41DA86FA51DAB
:10269800A96FA61DAA6FA71DAB6FFF0EB425AC6F5F
:1026A800FF0EB521AD6FFF0EB621AE6FFF0EB7213D
:1026B800AF6FA851AC15B06FA951AD15B16FAA5144
:1026C800AE15B26FAB51AF15B36F20EE10F09E513F
:1026D800D9269F51DA22B0C0DEFFB1C0DEFFB2C0FA
:1026E800DEFFB3C0DEFF20EE10F09E51D9269F51C9
:1026F800DA22DE50A05FDE50A15BDE50A25BDD5027
:10270800A35B20EE14F09E51D9269F51DA22DECF2A
:10271800C3F0DECFC4F0DECFC5F0DECFC6F060D0A8
:1027280020EE06F09E51D9269F51DA22DECFC3F063
:10273800DECFC4F0DECFC5F0DECFC6F0C351C41182
:10274800C511C6113FE19EC081F09FC082F0836B26
:10275800846B856B866BACEC25F081C0C3F082C0BE
:10276800C4F083C0C5F084C0C6F0C305C411C51148
:10277800C61109E120EE0FF09E51D9269F51DA22A9
:10278800020EDF6E020CC3290FE1C4290DE1C52931
:102798000BE1C62909E120EE0FF09E51D9269F5181
:1027A800DA22010EDF6E010C20EE06F09E51D926CA
:1027B8009F51DA22C3C0DEFFC4C0DEFFC5C0DEFF02
:1027C800C6C0DEFF20EE14F09E51D9269F51DA22B2
:1027D800C3C0DEFFC4C0DEFFC5C0DEFFC6C0DEFF6B
:1027E800C351C411C511C61101E085D0DDD0BF5158
:1027F800A05FC051A15BC151A25BC251A35B20EE97
:1028080010F09E51D9269F51DA22BF51DE26C051C1
:10281800DE22C151DE22C251DE2220EE0EF09E5190
:10282800D9269F51DA22DFA220D09EC081F09FC016
:1028380082F0C3C083F0C4C084F0C5C085F0C6C0B0
:1028480086F0ACEC25F081C0C3F082C0C4F083C030
:10285800C5F084C0C6F0C351C411C511C6111BE12F
:10286800A06BA16BA26BA36B50D09EC045F09FC01C
:1028780046F0C3C047F0C4C048F0C5C049F0C6C060
:102888004AF059EC2DF045C0C3F046C0C4F047C02B
:10289800C5F048C0C6F00001C32907E1C42905E115
:1028A800C52903E1C62901E176D7C651C511C4116E
:1028B80004E1020EC35D01E25DD720EE13F0BC51C6
:1028C800D926BD51DA22DE50C35DDE50C459DE5030
:1028D800C559DE50C65901E34DD720EE14F09E517C
:1028E800D9269F51DA22C3C0DEFFC4C0DEFFC5C0AF
:1028F800DEFFC6C0DEFFA051BF5DA151C059A25185
:10290800C159A351C25901E272D720EE10F09E516D
:10291800D9269F51DA22A051DE26A151DE22A251EA
:10292800DE22A351DE22A051A46F010EA115A56FCE
:10293800A66BA76BA411A611A71136E0BCC00EF0B8
:10294800BDC00FF0C3C010F0C4C011F0C5C012F074
:10295800C6C013F075EC4DF00EC0B8F00FC0B9F05A
:1029680010C0BAF011C0BBF00001B851B911BA11CA
:10297800BB1101E1FFD6A0C0A4F0A1C0A5F0A2C080
:10298800A6F0A3C0A7F00A0E05D0D890A733A633A7
:10299800A533A433E82EF9D7A451B827A551B923F4
:1029A800A651BA23A751BB2320EE10F09E51D92679
:1029B8009F51DA2210EE0AF09E51E1269F51E22241
:1029C800DE50E65CDE50E658DE50E658DE50E6584B
:1029D8001CE220EE10F09E51D9269F51DA2210EE0B
:1029E8000AF09E51E1269F51E222DECFE6FFDECFBC
:1029F800E6FFDECFE6FFDECFE6FF20EE0EF09E51CB
:102A0800D9269F51DA22000EDB8C20EE10F09E5161
:102A1800D9269F51DA22FF0EDE14A46F010EDE14B0
:102A2800A56F000EDE14A66F000EDE14A76FA4516A
:102A3800A511A611A71101E16AD520EE18F09E5143
:102A4800D9269F51DA22B851DE180AE1B951DE18A9
:102A580007E1BA51DE1804E1BB51DE1801E157D590
:102A680020EE18F09E51D9269F51DA22B8C0DEFF19
:102A7800B9C0DEFFBAC0DEFFBBC0DEFF48D5CE510D
:102A8800CF1101E1090C3F0ED217D00E7C6F7D0EDD
:102A98007D6F010E7E6FD2C07FF0AFEC00F00101B8
:102AA8007F6F7F5101E0A8D27DC180F17EC181F1A5
:102AB800800E0001C06F010EC16FD0C0C2F0D1C03E
:102AC800C3F0E7EC43F001017F6F7F5104E1A7AF4A
:102AD80002D0060E7F6FD2C0D3F01C0E0001D317B0
:102AE80001E1D1D001017F510FE0040E7F1909E106
:102AF800800E0001C46F010EC56F14EC54F0010183
:102B08007F6F0001D2870DD084C1D3F0110E000170
:102B1800D31702E0070E03D0D2A503D0080E010197
:102B28007F6F01017F5101E0BDD00001D2A7BAD06B
:102B38007DC115F07EC116F09AC117F09BC118F03F
:102B480057EC5BF015C06DF116C06EF117C06FF150
:102B580018C070F10E0E01019A250E6E000E9B2111
:102B68000F6E106A116A210E126E500E136EA7ECCA
:102B78005CF0010120EE0BF09A51D9269B51DA2224
:102B8800200EDF6E7DC112F07EC113F09AC114F0E1
:102B98009BC115F0166A176A186A196A1EEC60F06C
:102BA8001C0E01019A250E6E000E9B210F6E106AF5
:102BB800116A126A136AA7EC5CF0010120EE03F0B7
:102BC8007D51D9267E51DA22010EDF6E6D516E11CC
:102BD8006F11701167E020EE2BF07D51D9267E51E0
:102BE800DA22DECF71F1DECF72F1DECF73F1DECF04
:102BF80074F1800E0001816F010E826F6DC183F048
:102C08006EC184F06FC185F070C186F0876B886BE8
:102C1800896B8A6BB4EC44F001017F6F7F5142E10C
:102C28007DC13AF07EC13BF071C13CF072C13DF00C
:102C380073C13EF074C13FF0D1EC56F001017F6FD3
:102C4800FF0E6D250001D36FFF0E01016E210001FB
:102C5800D46FFF0E01016F210001D56FFF0E010136
:102C680070210001D66F010120EE0BF07D51D926AD
:102C78007E51DA22D3C0DEFFD4C0DEFFD5C0DEFF2E
:102C8800D6C0DEFF0FD001017F510CE184A902D02C
:102C9800040E07D00001D2A305D0010184A102D0FF
:102CA800070E7F6F01017F5123E10001D2B7D28D5A
:102CB800010120EE2BF07D51D9267E51DA22000148
:102CC80010EE1CF0CE51E126CF51E222DECFE6FF16
:102CD800DECFE6FFDECFE6FFDECFE6FF20EE20F018
:102CE800CE51D926CF51DA229AC1DEFF9BC1DDFF32
:102CF80001017F5101E080D17DC115F07EC116F040
:102D08009AC117F09BC118F057EC5BF0000120EE58
:102D180006F0CE51D926CF51DA2215C0DEFF16C0F3
:102D2800DEFF17C0DEFF18C0DEFF1C0E01019A256A
:102D38000E6E000E9B210F6EDCEC55F0000120EEAC
:102D48000AF0CE51D926CF51DA220EC0DEFF0FC0CD
:102D5800DEFF10C0DEFF11C0DEFFCEC0D9FFCFC03E
:102D6800DAFF7DC1DEFF7EC1DDFF010120EE05F047
:102D78007D51D9267E51DA22000110EE02F0CE51A3
:102D8800E126CF51E222DECFE6FFDDCFE5FF20EEE0
:102D98000EF0CE51D926CF51DA22D2C0DFFF20EE75
:102DA8000FF0CE51D926CF51DA22DF6A20EE18F083
:102DB800CE51D926CF51DA22DE6ADE6ADE6ADD6AB2
:102DC80020EE10F0CE51D926CF51DA22DE6ADE6A23
:102DD800DE6ADD6AD2AB10D120EE0AF0CE51D926D8
:102DE800CF51DA22DE50DE10DE10DE1001E104D110
:102DF80020EE0AF0CE51D926CF51DA2210EE10F08B
:102E0800CE51E126CF51E222DECFE6FFDECFE6FF4C
:102E1800DECFE6FFDECFE6FF010120EE09F07D51AF
:102E2800D9267E51DA22DECFD3F0DDCFD4F00001EF
:102E3800D351D56FD451D66FD76BD86B090ED890B4
:102E4800D537D637D737D837E82EF9D7D5C069F16F
:102E5800D6C06AF1D7C06BF1D8C06CF120EE06F08D
:102E6800CE51D926CF51DA22DECF79F1DECF7AF1F1
:102E7800DECF7BF1DECF7CF120EE0AF0CE51D926F1
:102E8800CF51DA22DECF75F1DECF76F1DECF77F1E2
:102E9800DECF78F132D0CEC045F0CFC046F079C150
:102EA80047F07AC148F07BC149F07CC14AF059EC3F
:102EB8002DF045C079F146C07AF147C07BF148C092
:102EC8007CF101017C517B117A1105E1020E795DDB
:102ED80002E2020E7F6F792908E17A2906E17B294F
:102EE80004E17C2902E1010E7F6F6951755F6A5127
:102EF800765B6B51775B6C51785B01017F5109E11F
:102F08007551695D76516A5977516B5978516C5989
:102F1800C2E3000120EE14F0CE51D926CF51DA22B7
:102F280079C1DEFF7AC1DEFF7BC1DEFF7CC1DEFF37
:102F380001017F5161E175510001D36F010E01015B
:102F480076150001D46FD56BD66BD311D511D61178
:102F580053E07DC10EF07EC10FF079C110F07AC147
:102F680011F07BC112F07CC113F075EC4DF00EC06E
:102F780071F10FC072F110C073F111C074F1010149
:102F8800715172117311741103E1020E7F6F34D005
:102F980075C1D3F076C1D4F077C1D5F078C1D6F039
:102FA8000A0E06D00001D890D633D533D433D333A4
:102FB800E82EF8D7010171510001D325D76F01011F
:102FC80072510001D421D86F010173510001D5213C
:102FD800D96F010174510001D621DA6F20EE18F083
:102FE800CE51D926CF51DA22D7C0DEFFD8C0DEFFB6
:102FF800D9C0DEFFDAC0DEFF01017F5106E0CEC096
:10300800D9FFCFC0DAFFDE6ADD6A7F511200276E72
:103018002150100B256E225002E0CFEC54F0266AA6
:10302800255001E120D2279E040E271802E14E50B8
:1030380003E1140E271807E10101486B496B226A66
:10304800070E216E070C3F0E271807E14E6A010193
:10305800486B496B216A226A12005F0E271807E144
:1030680001015A6B486B496B216A226A12003F0EB4
:1030780027640BD05F0E276008D0400E271805E0A4
:1030880001015A6B216A226A1200400E27180AE1D0
:10309800010E01015A6F4E6A0101486B496B216AA2
:1030A800226A1200200E271801E0DDD1010E4E6EB3
:1030B800F3D7600E27180CE101015A5109E0585165
:1030C800080ED8B4030E266E0101486B496B33D243
:1030D800600E271809E14E5007E00101585102E03F
:1030E800090EF1D7050EEFD7680E271809E14E50E3
:1030F80007E01A0E0101496F900E5FD183801BD241
:10310800680E271805E101015A5102E0020EDBD7CB
:103118006A0E271807E14E5005E01A0E0101496FA3
:10312800F40E4BD16C0E271807E14E5005E01A0E2D
:103138000101496F2C0E41D1700E271808E10101D9
:103148005A5105E0040E266E486B496BD7D7700EAE
:10315800271801E0F0D14E5001E1EDD11B0E01011D
:10316800496F620E2AD1838027500CE121AA05D02D
:10317800266A0101486B496B83901A0E0101496F59
:10318800AF0E486F020E271805E11A0E0101496FAC
:10319800920E486F050E271805E11A0E0101496FB6
:1031A800AE0E486F070E271805E11A0E0101496F88
:1031B800B80E486F080E271805E11A0E0101496F6D
:1031C800CC0E486F030E271802E027280CE18380F5
:1031D800680E236EE40EE82EFED7232EFCD700D00F
:1031E800266A839071D7140E271805E11A0E01017B
:1031F800496F9E0E486F160E271801E09CD11A0ED3
:103208000101496FA40ECAD0050E271805E11A0E50
:103218000101496FF50E486F080E271801E08BD1A0
:103228001A0E0101496FCC0E486F010E586F83D1F9
:1032380027C052F01A0E0101496F950EAFD02750E2
:10324800246E236A52500C0D000EF324D96E010E21
:10325800F420DA6E23C0DEFF24C0DDFF1A0E010160
:10326800496F960E9BD02750236E246A52500C0D3E
:10327800000EF324D96E010EF420DA6E23C0DEFFAF
:1032880024C0DDFF1A0E0101496F970E87D05250F6
:103298000C0D020EF324D96E010EF420DA6E27C04D
:1032A800DFFF1A0E0101496F980E78D052500C0DAD
:1032B800030EF324D96E010EF420DA6E27C0DFFF67
:1032C8000101486B496B010E37D01A0E0101496F95
:1032D800B90E73D01A0E0101496FBA0E5FD01A0EDB
:1032E8000101496FBB0E486F510E00019C6FFE0E25
:1032F8009D6F70EC63F00101596B486B496B55D0B9
:103308000101486B496B510E00019C6FFE0E9D6FC9
:1033180070EC63F04AD0090E00019C6FFF0E9D6FA0
:1033280070EC63F00101486B496B010E566F3DD09C
:103338000101486B496B060E266EFDD027C052F07E
:103348000101486B496B266A30D00101586B1A0E8F
:10335800496FF70E486F29D01A0E0101496FF70E11
:103368001DD08390270E0101496F0F0E17D0180E3C
:10337800271801E0E0D01A0E0101496F2D0E0ED07A
:103388001A0E0101496F2E0E09D01A0E0101496F5C
:103398002F0E04D01A0E0101496F300E486FCBD0A2
:1033A8000101486B496B0A0E266E8390C4D0040E47
:1033B800266E270E0101496F0F0E486F9FD6838036
:1033C800010104D08390010E0101586F486B496BCD
:1033D800266AB1D08390010E0101586F486B496B82
:1033E800266A52500C0D000EF324D96E010EF420FB
:1033F800DA6EDE6ADD6A52500C0D020EF324D96EC5
:10340800010EF420DA6E2744E846030BDF6E5250B3
:103418000C0D030EF324D96E010EF420DA6E27503A
:103428003F0BDF6ECA0E00019C6FFC0E9D6F27C01C
:103438009EF09F6B52500C0D020EF324D96E010EB4
:10344800F420DA6EDF50A06FA16B52500C0D030E02
:10345800F324D96E010EF420DA6EDF50A26FA36B4D
:1034680070EC63F068D048C123F049C124F02450BF
:1034780007E01A0A09E0010A54E03C0A5AE05BD066
:10348800235001E116D657D023502C0A01E16FD7FB
:10349800010A01E175D7030A01E177D7010A01E1C1
:1034A80079D71F0A01E17CD7A00A01E15CD6020A9C
:1034B80001E1BED6070A01E1C2D6030A01E1D3D66B
:1034C800010A01E1E4D60F0A01E1F0D6060A01E19A
:1034D80022D73A0A01E12CD70A0A01E173D7010A77
:1034E80001E178D7170A01E1F0D6010A01E1F2D625
:1034F800030A01E1F4D6010A01E102D7790A01E1E0
:1035080005D60E0A01E11AD7380A01E17DD6010A6B
:1035180001E11BD7030A01E11FD7010A01E121D705
:103528000AD02350580A01E142D73A0A01E147D7A5
:1035380002D023500F0A26C021F0226A120076C05A
:1035480091F077C092F07AC0D9FF7BC0DAFFDE6ACB
:10355800DD6A74C00FF075C010F09D0E116E86EC18
:1035680055F000018C6F8C510AE120EE0FF0745178
:10357800D9267551DA22DF508C6F8C5102E08C51BC
:10358800120020EE0EF07451D9267551DA22DFA010
:10359800070C20EE10F07451D9267551DA22DECFCF
:1035A8007CF0DECF7DF0DECF7EF0DECF7FF020EE48
:1035B8000AF07451D9267551DA22DECF80F0DECFB9
:1035C80081F0DECF82F0DECF83F07C51805D886FA2
:1035D8007D518159896F7E5182598A6F7F518359F4
:1035E8008B6F78517C6F79517D6F7E6B7F6B7C51CF
:1035F800885D7D5189597E518A597F518B5901E3E4
:1036080021D288C078F089C079F01CD220EE10F061
:103618007451D9267551DA22FF0EDE147C6F010E23
:10362800DE147D6F000EDE147E6F000EDE147F6FD9
:103638007C517D117E117F1101E083D120EE10F0C5
:103648007451D9267551DA22DECF7CF0DECF7DF0B9
:10365800DECF7EF0DECF7FF00A0E05D0D8907F3324
:103668007E337D337C33E82EF9D78069816920EE7B
:1036780009F09D51D9269E51DA22DECF82F0DDCFA6
:1036880083F080518227815183237C518215936F67
:103698007D518315946F931166E120EE10F07451FB
:1036A800D9267551DA22DE50DE10DE10DE100FE169
:1036B80020EE06F07451D9267551DA22DECF8DF04E
:1036C800DECF8EF0DECF8FF0DECF90F01CD074C04E
:1036D80045F075C046F020EE14F07451D9267551A6
:1036E800DA22DECF47F0DECF48F0DECF49F0DECF7A
:1036F8004AF059EC2DF045C08DF046C08EF047C019
:103708008FF048C090F0000190518F118E110CE19C
:10371800020E8D5D09E220EE0FF07451D926755125
:10372800DA22020EDF6E020C8D290FE18E290DE1DF
:103738008F290BE1902909E120EE0FF07451D92669
:103748007551DA22010EDF6E010C20EE14F074516F
:10375800D9267551DA228DC0DEFF8EC0DEFF8FC0FC
:10376800DEFF90C0DEFF9DC00EF09EC00FF020EE81
:1037780014F07451D9267551DA22DECF10F0DECF5D
:1037880011F0DECF12F0DECF13F075EC4DF00EC065
:1037980095F00FC096F010C097F011C098F0000196
:1037A800955196119711981101E1B5D79351952725
:1037B80094519623000E9723982378C07CF079C003
:1037C8007DF0090E7E6FD8907D337C337E2FFBD73A
:1037D8007CC099F07DC09AF099519A1101E1A3D06B
:1037E800995193257C6F9A5194217D6F20EE09F0B1
:1037F8009D51D9269E51DA227C51DE5C7D51DE58DE
:1038080010E220EE09F09D51D9269E51DA22DECF32
:103818007CF0DDCF7DF093517C5D996F94517D599B
:103828009A6F91C01DF092C01EF095C01FF096C00F
:1038380020F097C021F098C022F099C023F09AC0D8
:1038480024F020EE01F09D51D9269E51DA22DF5056
:1038580030EC56F0000901E0ACD0000120EE03F096
:103868009D51D9269E51DA22DF504EE099517C6F46
:103878009A517D6F7E6B7F6B20EE2BF09D51D92680
:103888009E51DA22DECF80F0DECF81F0DECF82F0EB
:10389800DECF83F09551805D846F96518159856F95
:1038A80097518259866F98518359876F7C51845DEF
:1038B8007D5185597E5186597F51875925E220EEE1
:1038C8002BF09D51D9269E51DA22DECF7CF0DDCF38
:1038D8007DF095517C5F96517D5B090ED8907C37C1
:1038E8007D37E82EFBD77C5191250E6E7D519221B4
:1038F8000F6E2F0E9D25106E000E9E21116E020E6A
:10390800136E126ABDEC5FF099C07CF09AC07DF02E
:10391800090ED8907C377D37E82EFBD77CC09BF00A
:103928007DC09CF072D020EE18F07451D9267551E4
:10393800DA2295C0DEFF96C0DEFF97C0DEFF98C092
:10394800DEFF7C69010E7D6F20EE10F07451D926E0
:103958007551DA22DECF7EF0DDCF7FF07C517E1705
:103968007D517F177E5100089B6F7F51D8A0E82AB0
:1039780002089C6F9B51785D9C51795904E278C08C
:103988009BF079C09CF09DC03AF09EC03BF020EEC1
:1039980018F07451D9267551DA22DECF3CF0DECF0B
:1039A8003DF0DECF3EF0DECF3FF0D1EC56F000091F
:1039B80002E00001C1D691C00EF092C00FF00001E4
:1039C8007C69010E7D6F20EE10F07451D926755177
:1039D800DA22DECF7EF0DDCF7FF07C517E177D517D
:1039E8007F179DC080F09EC081F07E5180277F5157
:1039F80081232F0E8025106E000E8121116E9BC031
:103A080012F09CC013F0BDEC5FF09B51785F9C51A5
:103A1800795B7AC0D9FF7BC0DAFF9B51DE269C51C7
:103A2800DD229B5191279C51922320EE10F0745176
:103A3800D9267551DA229B51DE269C51DE22000ED2
:103A4800DE22DE227851791101E0E0D5000C5250D7
:103A58000C0D000EF324D96E010EF420DA6E00016D
:103A6800C969CA6952500C0D080EF324E16E010EA3
:103A7800F420E26EE6CFCBF0E5CFCCF0C951CB27EE
:103A8800CA51CC23DE50CB5DCC51800ACD6FDE50BD
:103A9800800ACD594AE352500C0D020EF324D96E18
:103AA800010EF420DA6EDF50C76FC86BC969CA69A6
:103AB80052500C0D0A0EF324D96E010EF420DA6E62
:103AC800DF50CB6FCC6BC951CB27CA51CC23C75120
:103AD800CB5DCC51800ACD6FC851800ACD5925E302
:103AE80052500C0D030EF324D96E010EF420DA6E39
:103AF800DF50C76FC86BC969CA6952500C0D0B0EED
:103B0800F324D96E010EF420DA6EDF50CB6FCC6B44
:103B1800C951CB27CA51CC23C751CB5DCC51800AA0
:103B2800CD6FC851800ACD5961E21F0E0101576F50
:103B3800010E596F8390250E00019C6FFA0E9D6F40
:103B480052500C0D000EF324D96E010EF420DA6EDB
:103B5800DECF9EF0DDCF9FF052500C0D080EF324FF
:103B6800D96E010EF420DA6EDECFC7F0DDCFC8F0D3
:103B7800FF0EC725A06FFF0EC821A16F52500C0D74
:103B8800020EF324D96E010EF420DA6EDF50A26F14
:103B9800A36B52500C0D0A0EF324D96E010EF420BB
:103BA800DA6EDF50C96FFF0EC925A46FA56BFF0E33
:103BB800A52352500C0D030EF324D96E010EF420E8
:103BC800DA6EDF50A66FA76B52500C0D0B0EF32464
:103BD800D96E010EF420DA6EDF50CA6FFF0ECA25C7
:103BE800A86FA96BFF0EA92370EC63F052500C0D5F
:103BF800030EF324D96E010EF420DA6EDF50C76F7E
:103C0800C7C0C8F0C96BCA6BCB6BCAC0CBF0C9C000
:103C1800CAF0C8C0C9F0C86B52500C0D0B0EF32483
:103C2800D96E010EF420DA6EDF50CC6FCCC0CDF027
:103C3800CE6BCF6BD06B52500C0D020EF324D96EA5
:103C4800010EF420DA6EDF50D16FD1C0D2F0D36B01
:103C5800D46BD56BD4C0D5F0D3C0D4F0D2C0D3F0D8
:103C6800D26BD251CD03F3CFD6F0F4CFD7F0D86BC7
:103C7800D96BCE03F350D727F450D823000ED9239D
:103C8800D351CD03F350D727F450D823000ED923AE
:103C9800D251CF03F350D827F450D923D351CE03B0
:103CA800F350D827F450D923D451CD03F350D82753
:103CB800F450D923D051D203F350D927D351CF038D
:103CC800F350D927D451CE03F350D927D551CD037A
:103CD800F350D92752500C0D0A0EF324D96E010E59
:103CE800F420DA6EDF50DA6FDAC0DBF0DC6BDD6B04
:103CF800DE6B52500C0D0B0EF324D96E010EF4201E
:103D0800DA6EDF50DF6FDFC0E0F0E16BE26BE36B90
:103D180052500C0D000EF324D96E010EF420DA6E09
:103D2800DECFE4F0DDCFE5F0E4C0E6F0E5C0E7F093
:103D3800000EE7BFFF0EE86FE96FE651E003F3CF2F
:103D4800EAF0F4CFEBF0EC6BED6BE103F350EB270B
:103D5800F450EC23000EED23E751E003F350EB277A
:103D6800F450EC23000EED23E651E203F350EC2768
:103D7800F450ED23E751E103F350EC27F450ED2321
:103D8800E851E003F350EC27F450ED23E351E60348
:103D9800F350ED27E751E203F350ED27E851E10333
:103DA800F350ED27E951E003F350ED27ECC0EDF0B7
:103DB800EBC0ECF0EAC0EBF0EA6BEA51DB03F3CFBF
:103DC800EEF0F4CFEFF0F06BF16BDC03F350EF277C
:103DD800F450F023000EF123EB51DB03F350EF27EF
:103DE800F450F023000EF123EA51DD03F350F027DD
:103DF800F450F123EB51DC03F350F027F450F12396
:103E0800EC51DB03F350F027F450F123DE51EA03C1
:103E1800F350F127EB51DD03F350F127EC51DC03AC
:103E2800F350F127ED51DB03F350F127D651EE257E
:103E3800F26FD751EF21F36FD851F021F46FD951B8
:103E4800F121F56FC851F225F76FC951F321F86FC9
:103E5800CA51F421F96FCB51F521FA6F5250220D56
:103E6800000EF3249E6F030EF4209F6FF7C0A0F09E
:103E7800F8C0A1F0F9C0A2F0FAC0A3F075EC12F0F6
:103E8800F66FF65111E0720E9C6FFB0E9D6FF7C036
:103E98009EF0F8C09FF0F9C0A0F0FAC0A1F0F6C0FB
:103EA800A2F0A36B70EC63F052500C0D040EF324D7
:103EB800D96E010EF420DA6EF7C0DEFFF8C0DEFF1F
:103EC800F9C0DEFFFAC0DEFF0101596B83901200D2
:103ED800020E806F65516411631104E1020E625D88
:103EE80001E211D220EE13F06051D9266151DA2295
:103EF800DE50625DDE506359DE506459DE5065590C
:103F080001E2EED100D262C07EF063C07FF0D890AB
:103F18007F316B6F7E316A6F6A517E276B517F23C9
:103F280060C03AF061C03BF020EE1FF06051D92626
:103F38006151DA22DECF6AF0DECF6BF0DECF6CF0B3
:103F4800DECF6DF07EC06EF07FC06FF0090E706F2F
:103F5800D8906F336E33702FFBD76E516A253C6E45
:103F68006F516B213D6E000E6C213E6E000E6D216F
:103F78003F6ED1EC56F00001806F805101E0C3D153
:103F88006A69010E6B6F7EC06CF07FC06DF06A517C
:103F98006C176B516D1760C06EF061C06FF06C519B
:103FA8006E276D516F232F0E6E257C6F000E6F21CB
:103FB8007D6F7E4B7F2B62B104D066C078F0796B41
:103FC8001AD066516A6F6B6B6A3B6B3BF00E6B17CE
:103FD8006A510F0B6B13F00E6A177CC0D9FF7DC0B6
:103FE800DAFFDF500F0B6C6F6D6B6A516C11786FD5
:103FF8006B516D11796F7CC0D9FF7DC0DAFF78C035
:10400800DFFF20EE03F06051D9266151DA22010E5C
:10401800DF6E60C03AF061C03BF020EE1FF06051E7
:10402800D9266151DA22DECF6AF0DECF6BF0DECF1F
:104038006CF0DECF6DF07EC06EF07FC06FF0090EC1
:10404800706FD8906F336E33702FFBD76E516A251F
:104058003C6E6F516B213D6E000E6C213E6E000E62
:104068006D213F6ED1EC56F00001806F805101E068
:104078004AD16A69010E6B6F7EC06CF07FC06DF02B
:104088006A516C176B516D1760C06EF061C06FF0AC
:104098006C516E276D516F232F0E6E257C6F000EAD
:1040A8006F217D6F62B10CD067C06AF00F0E6A177E
:1040B8007CC0D9FF7DC0DAFFDF50F00B6A1112D047
:1040C80066C06AF067C06BF068C06CF069C06DF0DC
:1040D800050E05D0D8906D336C336B336A33E82EF8
:1040E800F9D76A517A6F7B6B7CC0D9FF7DC0DAFF44
:1040F8007AC0DFFF4FD060C03AF061C03BF020EEDD
:104108001FF06051D9266151DA22DECF6AF0DECF86
:104118006BF0DECF6CF0DECF6DF063516E6F6451E3
:104128006F6F6551706F716B6A516E253C6E6B5184
:104138006F213D6E6C5170213E6E6D5171213F6E45
:10414800D1EC56F00001806F805101E0DCD06A6943
:10415800010E6B6F62C06CF063C06DF0D8906C3765
:104168006D376A516C176B516D1760C06EF061C086
:104178006FF06C516E276D516F232F0E6E250E6EEA
:10418800000E6F210F6E66C010F067C011F0B8EC1A
:1041980062F0A4D020EE03F06051D9266151DA22F2
:1041A800010EDF6EB0D060C03AF061C03BF020EE87
:1041B8001FF06051D9266151DA22DECF6AF0DECFD6
:1041C8006BF0DECF6CF0DECF6DF062C06EF063C0D6
:1041D8006FF064C070F065C071F0080E05D0D8901B
:1041E800713370336F336E33E82EF9D76A516E2509
:1041F8003C6E6B516F213D6E6C5170213E6E6D515E
:1042080071213F6ED1EC56F00001806F80517BE147
:104218006A69010E6B6F62C06CF063C06DF0D89074
:104228006C376D37D8906C376D376A516C176B5196
:104238006D1760C06EF061C06FF06C516E276D51E4
:104248006F232F0E6E250E6E000E6F210F6EDCECA5
:1042580055F00001706B716B726BF00E1114736F77
:104268006651746F6751756F6851766F0F0E6915D7
:10427800776F70517411666F71517511676F725154
:104288007611686F73517711696F6A69010E6B6FE8
:1042980062C06CF063C06DF0D8906C376D37D89001
:1042A8006C376D376A516C176B516D1760C06EF0C3
:1042B80061C06FF06C516E276D516F232F0E6E2504
:1042C8000E6E000E6F210F6E66C010F067C011F001
:1042D80068C012F069C013F0A7EC5CF000015AD76F
:1042E80060C0D9FF61C0DAFFDF506A6F6B6B6B513A
:1042F8000AE16A51010A01E106D6030A01E1FBD687
:10430800010A01E150D7805112002D6E1EC044F001
:104318001FC045F02D5001E0040C010E426E55B04F
:10432800030CE9D142EC63F0000901E1FDD1426AD6
:10433800FBD1176A186A196A1A6A090E0AEC61F041
:10434800000901E0F1D12E0E0E6E0F6A116A100EEF
:10435800106E71EC5DF0000901E1E6D12E44E846EB
:10436800030BE8064DE135C020F03F0E201620C0B3
:1043780021F0226A236A246A22C024F021C023F093
:10438800226A216A3650266E256A3750276E286AB7
:10439800255027262650282227502124296E2850C8
:1043A80022202A6E000E23202B6E000E24202C6E55
:1043B80029283E6E000E2A203F6E000E2B20406EEC
:1043C800000E2C20416E3EC020F03FC021F040C0BE
:1043D80022F041C023F00A0ED8902036213622362A
:1043E8002336E82EF9D71EC0D9FF1FC0DAFF20C038
:1043F800DEFF21C0DEFF22C0DEFF23C0DEFF97D72D
:10440800206A38AE01D0202A010E201633C021F0D0
:104418000F0E21163750030B020DF35021242024D0
:10442800020F436E3450030B206E216A0A0ED89097
:1044380020362136E82EFBD73550226E236AD890D5
:1044480022362336D890223623363644E846030BE4
:10445800246E256A22502426235025222050242603
:1044680021502522242A000E252224C03EF025C0F2
:104478003FF0406A416A43C020F0F70E20263EC054
:1044880021F03FC022F040C023F041C024F0202A90
:1044980005D0D8902136223623362436202EF9D757
:1044A80034D053A43FD0176A186A196A1A6A8D0E55
:1044B8000AEC61F0000901E037D194EC63F02E0EAC
:1044C8000E6E0F6A116A100E106E71EC5DF0000925
:1044D80001E12AD1300E436E03D094EC63F0430619
:1044E8004350FBE138C020F0203A0F0E2016100E82
:1044F800216E226A236A246A202A05D0D8902136A0
:10450800223623362436202EF9D71EC0D9FF1FC0E5
:10451800DAFF21C0DEFF22C0DEFF23C0DEFF24C099
:10452800DEFF05D7176A186A196A1A6A090E0AECB3
:1045380061F0000901E0F8D02E0E0E6E0F6A116AC4
:10454800100E106E71EC5DF0000901E1EDD053A280
:1045580032D03BC020F0060E216ED8902032212E9A
:10456800FCD7FF0E202638503F0B226E236AD890C6
:10457800223623363944010B2226000E2322222A12
:104588002322202A03D0D89022362336202EFBD788
:104598002250246E2350256E266A276A1EC0D9FF32
:1045A8001FC0DAFF24C0DEFF25C0DEFF26C0DEFF05
:1045B80027C0DEFFBCD63950030B206E216AD89085
:1045C80020362136D89020362136D890203621360C
:1045D8003938E842070B2026000E2122202A212202
:1045E8003840E8423F0B1F0B226E236A222A000E36
:1045F800232220502202F3CF24F0F4CF25F0230207
:10460800F350252621502202F35025262450266EE9
:104618002550276E286A296A1EC0D9FF1FC0DAFFF5
:1046280026C0DEFF27C0DEFF28C0DEFF29C0DEFF70
:104638007ED644C0D9FF45C0DAFF53C0DFFF77D626
:10464800176A186A196A1A6A090E0AEC61F00009F1
:104658006BE144C00EF045C00FF0116A100E106EE9
:1046680071EC5DF0000901E062D65ED0176A186A45
:10467800196A1A6A0A0E0AEC61F0000955E144C089
:104688000EF045C00FF0116A100E106E71EC5DF05F
:10469800E9D7176A186A196A1A6A3A0E0AEC61F0B9
:1046A800000942E1040E436E0AD094EC63F044C062
:1046B800D9FF45C0DAFFDF6E444A452A4306435016
:1046C80001E135D6F2D7176A186A196A1A6A8D0E87
:1046D8000AEC61F0000928E194EC63F044C00EF0A4
:1046E80045C00FF0116A400E106E71EC5DF0BAD73C
:1046F800040E426E19D01D50206E216A2150F8E137
:10470800205001E10FD6010A01E113D6020A01E1A6
:10471800C8D6090A8EE0010A93E0070AA7E0010A51
:10472800B8E0030AD0E0E4D7A5EC63F042501200E9
:104738001BC0F6FF1CC0F7FF0800F5CF9BF01B4A13
:104748001C2A00019B5101E11200250E9B1904E06F
:104758009B5165EC63F0ECD7946B956B966B976BFC
:104768001BC0F6FF1CC0F7FF0800F5CF9BF01B4AE3
:104778001C2A300E9B190DE1976B010E966F1BC01A
:10478800F6FF1CC0F7FF0800F5CF9BF01B4A1C2A58
:1047980006D02D0E9B1903E1976B020EEFD72A0E58
:1047A8009B1943E11D50D96EDA6A020EDF26DF5CE1
:1047B800D96EDA6ADECF8CF0DECF8DF08DAF0BD0FC
:1047C8008C5100088C6F8D51D8A0E82A00088D6F95
:1047D800976B020E966F8CC094F08DC095F01BC03D
:1047E800F6FF1CC0F7FF0800F5CF9BF01B4A1C2AF8
:1047F80022D00A0E9403F3CF1EF0F4CF1FF09503D6
:10480800F3501F269B511E26000E1F22D00E1E2479
:10481800946FFF0E1F20956F1BC0F6FF1CC0F7FF9B
:104828000800F5CF9BF01B4A1C2A2F0E9B6503D06E
:10483800390E9B65DED76C0E9B1903E04C0E9B1955
:104848000AE196851BC0F6FF1CC0F7FF0800F5CFEC
:104858009BF01B4A1C2A9B5101E112009BC09AF055
:10486800600E9A6575D0200E9A5F72D01D50D96E71
:10487800DA6A020EDF26DF5CD96EDA6ADECF84F0F0
:10488800DECF85F0926B936B03D00001924B932B94
:10489800925184251E6E935185211F6E1EC0F6FF0E
:1048A8001FC0F7FF000EF86E0E0EF76403D0080065
:1048B800F55005D0F6CFE9FFF7CFEAFFEF50000932
:1048C80004E0E3D7200E65EC63F0000196B30BD04B
:1048D80092511E6E93511F6E924B932B94511E5CF6
:1048E80095511F58EFE384C00FF085C010F0F5EC28
:1048F8005DF003D0200E65EC63F0000192511E6E4E
:1049080093511F6E924B932B94511E5C95511F58D7
:1049180001E30ED7EFD71D50D96EDA6ADF50DF2AD0
:10492800DF2AD96EDA6ADF5065EC63F001D7876B4E
:10493800020E08D0876B080E05D0876B0A0E02D0CE
:10494800876B100E866F1AD09B5165EC63F0F0D61A
:104958009A511E6E1F6A1F50F7E11E50420AE7E087
:10496800010AD9E0070AE9E00B0AE4E01C0A01E1C0
:104978007DD7060AE2E00D0AE3E0E6D796A511D056
:104988001D50D96EDA6A040EDF26DF5CD96EDA6A4A
:10499800DECF8EF0DECF8FF0DECF90F0DECF91F05D
:1049A80027D0440E9A1913E01D50D96EDA6ADF50E9
:1049B800DF2ADF2AD96EDA6ADECF1EF0DDCF1FF0DC
:1049C8001EC08EF01FC08FF0906B916B11D01D50E0
:1049D800D96EDA6ADF50DF2ADF2AD96EDA6ADECFCB
:1049E8008EF0DDCF8FF0000E8FBFFF0E906F916FAE
:1049F800440E9A190CE191AF0AD08E6D8F1FD8B072
:104A08008F2B901FD8B0902B000E91579689986BDA
:104A1800996B8EC088F08FC089F090C08AF091C0E1
:104A28008BF088C00EF089C00FF08AC010F08BC0E0
:104A380011F086C012F087C013F0146A156A10ECE2
:104A48005DF00E5000019A6F88C00EF089C00FF01B
:104A58008AC010F08BC011F086C012F087C013F026
:104A6800146A156AE2EC5AF00EC088F00FC089F09B
:104A780010C08AF011C08BF0090E00019A650BD0A6
:104A8800780E9B1903E0816B070E02D0816B270E0D
:104A9800806F80519A279851600FD96EDA6A9A51BF
:104AA800300FDF6E984B992B885189118A118B1121
:104AB80005E0995103E1200E985DB3E396A908D06B
:104AC8009851600FD96EDA6A2D0EDF6E984B992BCC
:104AD80098C092F099C093F096B103D0836B200EE2
:104AE80002D0836B300E826F82C09AF003D09A5145
:104AF80065EC63F0000196B30BD092511E6E935192
:104B08001F6E924B932B94511E5C95511F58EFE3E7
:104B18009807D8A099079851600FD96EDA6ADF50C4
:104B280065EC63F000019851991104E0F1D7200E6B
:104B380065EC63F0000192511E6E93511F6E924B0B
:104B4800932B94511E5C95511F5801E3F1D5EFD773
:104B580081C0D9FF82C0DAFFDECF98F0DDCF99F0AF
:104B6800835184118511861128E120EE0BF09851AC
:104B7800D9269951DA22DECF90F0DECF91F0DECF40
:104B880092F0DECF93F090519111921193110FE0B2
:104B980020EE13F09851D9269951DA22DE50905D13
:104BA800DE509159DE509259DE50935952E3010E6E
:104BB800906F916B926B936B4CD081C045F082C023
:104BC80046F083C047F084C048F085C049F086C0ED
:104BD8004AF059EC2DF045C09AF046C09BF047C00A
:104BE8009CF048C09DF000019D519C119B1109E16A
:104BF800020E9A5D06E2010E816F826B836B846BF5
:104C0800000C9A290FE19B290DE19C290BE19D29B4
:104C180009E19AC081F09BC082F09CC083F09DC0DE
:104C280084F0120020EE13F09851D9269951DA2217
:104C3800DE509A5DDE509B59DE509C59DE509D59DE
:104C4800E8E383C090F084C091F085C092F086C0FC
:104C580093F020EE0FF09851D9269951DA22DE50C0
:104C6800DE10DE10DE1005E1816B826B836B846BD6
:104C78001200946B956B966B976B8351901909E1B1
:104C88008451911906E1855192197DE18651931954
:104C9800D8A479D09029946F000E9121956F000EB9
:104CA8009221966F000E9321976F20EE13F0985182
:104CB800D9269951DA22DE50945DDE509559DE509E
:104CC8009659DE50975905E3020E946F956B966BD3
:104CD800976B81C045F082C046F094C047F095C0FC
:104CE80048F096C049F097C04AF059EC2DF045C0FD
:104CF8009AF046C09BF047C09CF048C09DF0000168
:104D08009A059B119C119D1184E09A2907E19B2922
:104D180005E19C2903E19D2901E17BD79A519B116B
:104D28009C119D1130E020EE0BF09851D926995135
:104D3800DA22DECF9AF0DECF9BF0DECF9CF0DECF1A
:104D48009DF09D519C119B1103E1020E9A5D17E3A2
:104D580020EE13F09851D9269951DA22DE509A5D47
:104D6800DE509B59DE509C59DE509D5908E29AC08E
:104D780090F09BC091F09CC092F09DC093F0946B12
:104D8800956B966B976B945195119611971162E1FB
:104D980090C094F091C095F092C096F093C097F0AF
:104DA800942B000E95239623972320EE13F0985109
:104DB800D9269951DA22DE50945DDE509559DE509D
:104DC8009659DE5097590DE3020E946F956B966BCA
:104DD800976B93519211911104E1020E905D01E2DB
:104DE80043D781C045F082C046F094C047F095C0D3
:104DF80048F096C049F097C04AF059EC2DF045C0EC
:104E08009AF046C09BF047C09CF048C09DF0000156
:104E18009A519B119C119D111DE09A059B119C11A3
:104E28009D1101E1F6D69A2907E19B2905E19C2904
:104E380003E19D2901E1EDD690519419B1E1915119
:104E48009519AEE192519619ABE19351971901E189
:104E58000BD7A6D798C060F099C061F094C062F0F3
:104E680095C063F096C064F097C065F0666967699D
:104E7800686969696CEC1FF08F6F8F511CE1835171
:104E880084118511861117E098C060F099C061F00F
:104E980083C062F084C063F085C064F086C065F0AA
:104EA80094C066F095C067F096C068F097C069F046
:104EB8006CEC1FF08F6F8F5143E120EE0BF098518F
:104EC800D9269951DA2294C0DEFF95C0DEFF96C03C
:104ED800DEFF97C0DEFF20EE0FF09851D9269951DA
:104EE800DA2210EE13F09851E1269951E222FE0ED3
:104EF800E6248B6FFF0EE6208C6FFF0EE6208D6F89
:104F0800FF0EE6208E6FDE508B5DDE508C59DE5032
:104F18008D59DE508E590BE320EE0FF09851D926AB
:104F28009951DA22DE06000EDE5ADE5ADE5A20EEEB
:104F380004F09851D9269951DA22000EDB800DD061
:104F48008F0507E0010E946F000E956B966B976BBB
:104F580004D0946995699669976994C081F095C061
:104F680082F096C083F097C084F0120052500C0D66
:104F7800030EF324D96E010EF420DA6EDF2A5250A4
:104F88000C0D030EF324D96E010EF420DA6EDF50F7
:104F98000001C76FC86BC969CA6952500C0D0B0E66
:104FA800F324D96E010EF420DA6EDF50CB6FCC6B90
:104FB800C951CB27CA51CC23C751CB5DCC51800AEC
:104FC800CD6FC851800ACD594BE252500C0D030EDB
:104FD800F324D96E010EF420DA6EDF6A52500C0DFC
:104FE800020EF324D96E010EF420DA6EDF2A525035
:104FF8000C0D020EF324D96E010EF420DA6EDF5088
:10500800C76FC86BC969CA6952500C0D0A0EF324E0
:10501800D96E010EF420DA6EDF50CB6FCC6BC9511C
:10502800CB27CA51CC23C751CB5DCC51800ACD6F59
:10503800C851800ACD5914E252500C0D020EF324C7
:10504800D96E010EF420DA6EDF6A52500C0D000E94
:10505800F324D96E010EF420DA6EDE2A000EDD226A
:1050680052500C0D030EF324D96E010EF420DA6EA3
:10507800DF50C76FC7C0C8F0C96BCA6BCB6BCAC05B
:10508800CBF0C9C0CAF0C8C0C9F0C86B52500C0DEB
:105098000B0EF324D96E010EF420DA6EDF50CC6FBC
:1050A800CCC0CDF0CE6BCF6BD06B52500C0D020E36
:1050B800F324D96E010EF420DA6EDF50D16FD1C01F
:1050C800D2F0D36BD46BD56BD4C0D5F0D3C0D4F0A9
:1050D800D2C0D3F0D26BD251CD03F3CFD6F0F4CFF8
:1050E800D7F0D86BD96BCE03F350D727F450D82319
:1050F800000ED923D351CD03F350D727F450D8232A
:10510800000ED923D251CF03F350D827F450D92316
:10511800D351CE03F350D827F450D923D451CD031B
:10512800F350D827F450D923D051D203F350D927BC
:10513800D351CF03F350D927D451CE03F350D927F5
:10514800D551CD03F350D92752500C0D0A0EF32434
:10515800D96E010EF420DA6EDF50DA6FDAC0DBF0B8
:10516800DC6BDD6BDE6B52500C0D0B0EF324D96E2D
:10517800010EF420DA6EDF50DF6FDFC0E0F0E16B84
:10518800E26BE36B52500C0D000EF324D96E010E46
:10519800F420DA6EDECFE4F0DDCFE5F0E4C0E6F02F
:1051A800E5C0E7F0000EE7BFFF0EE86FE96FE651D4
:1051B800E003F3CFEAF0F4CFEBF0EC6BED6BE10337
:1051C800F350EB27F450EC23000EED23E751E003F6
:1051D800F350EB27F450EC23000EED23E651E203E5
:1051E800F350EC27F450ED23E751E103F350EC279B
:1051F800F450ED23E851E003F350EC27F450ED238D
:10520800E351E603F350ED27E751E203F350ED27AE
:10521800E851E103F350ED27E951E003F350ED279E
:10522800ECC0EDF0EBC0ECF0EAC0EBF0EA6BEA5151
:10523800DB03F3CFEEF0F4CFEFF0F06BF16BDC03B0
:10524800F350EF27F450F023000EF123EB51DB036A
:10525800F350EF27F450F023000EF123EA51DD0359
:10526800F350F027F450F123EB51DC03F350F0270F
:10527800F450F123EC51DB03F350F027F450F12301
:10528800DE51EA03F350F127EB51DD03F350F12728
:10529800EC51DC03F350F127ED51DB03F350F12718
:1052A800D651EE25F26FD751EF21F36FD851F02187
:1052B800F46FD951F121F56FC851F225F66FC95134
:1052C800F321F76FCA51F421F86FCB51F521F96F2B
:1052D80052500C0D040EF324D96E010EF420DA6E30
:1052E800F6C0DEFFF7C0DEFFF8C0DEFFF9C0DEFF64
:1052F8005250220D000EF3249E6F030EF4209F6F70
:1053080052500C0D040EF324D96E010EF420DA6EFF
:10531800DECFA0F0DECFA1F0DECFA2F0DECFA3F08B
:1053280075EC12F04B6E4B5019E0720E9C6FFB0E31
:105338009D6F52500C0D040EF324D96E010EF4200B
:10534800DA6EDECF9EF0DECF9FF0DECFA0F0DECFAC
:10535800A1F04BC0A2F0A36B70EC63F00101596B94
:105368001200000E0001746F030E756F350E766F14
:105378000B0E776F020E796F786BF30E7A6F7B6B7B
:10538800A3EC1AF00101646F900E00019C6FFD0EF2
:105398009D6FF3C09EF0F4C09FF070EC63F0F56B66
:1053A800F66BF16BF26BF76BF86BF751D30FD96EA5
:1053B800DA6ADF6AF751E20FD96EDA6A000EDF6E39
:1053C800F74BF82BF8BFF1D7F85103E10F0EF75D53
:1053D800ECE3F96BFA6B30D1350EF925D96E0B0E6B
:1053E800FA21DA6E0D0EDE1801E0EBD09A0E0E6E81
:1053F800FF0E0F6ED30E106E6AEC57F00E500F10A2
:1054080007E1E20E156E89EC4FF015500101F46FBB
:10541800940E0E6EFF0E0F6ED30E106E6AEC57F0E0
:105428000E500F1007E1E20E156E89EC4FF0155083
:105438000101656F790E0E6EFF0E0F6ED30E106EA2
:105448006AEC57F00E500F1007E1E20E156E89EC6A
:105458004FF015500101606FD80E0E6EFF0E0F6EE3
:10546800D30E106E6AEC57F00E500F1007E1E20EE3
:10547800156E89EC4FF0155001015E6FDC0E0E6E53
:10548800FF0E0F6ED30E106E6AEC57F00E500F1011
:1054980007E1E20E156E89EC4FF015500101C86F57
:1054A8000001FB6BFC6BC40E7C6F7D6B800E7E6F06
:1054B800FF0E7F6FFBC080F0FCC081F098EC60F0BD
:1054C800C40E0E6E0F6AD30E106E6AEC57F00E50B3
:1054D8000F1018E10F0E0001FB03F3CFC2F0F4CF59
:1054E800C3F0FC03F350C327350EC2250E6E0D0E14
:1054F800C3210F6EE20E106E116A136A0F0E126E40
:10550800A0EC5DF00001FB4BFC2BFCBFCCD7FC51A1
:1055180003E1100EFB5DC7E3FC6B010EFB6FC40ECD
:105528007C6F7D6B870E7E6FFF0E7F6FFBC080F0F8
:10553800FCC081F098EC60F0C40E0E6E0F6AD30EBA
:10554800106E6AEC57F00E500F1018E10F0E0001A4
:10555800FB03F3CFC2F0F4CFC3F0FC03F350C3272F
:10556800250EC2250E6E0E0EC3210F6EE20E106EB2
:10557800116A136A0F0E126EA0EC5DF00001FB4B6E
:10558800FC2BFCBFCCD7FC5103E1040EFB5DC7E349
:10559800F76BF86BF751D30FD96EDA6ADF6AF751F8
:1055A800E20FD96EDA6A000EDF6EF74BF82BF8BF00
:1055B800F1D7F85103E10F0EF75DECE3F16BF26BF5
:1055C80015D0350EF925D96E0B0EFA21DA6E0A0EB2
:1055D800DE1830E0350EF925D96E0B0EFA21DA6E99
:1055E800200EDE1806E1F26B010EF16FF56BF66B1B
:1055F80021D0F151F21109E0350EF925D96E0B0EC3
:10560800FA21DA6EF551E20F08D0350EF925D96E78
:105618000B0EFA21DA6EF551D30FE16EE26ADFCF95
:10562800E7FFF6BF05D0F65105E10F0EF55D02E282
:10563800F54BF62BF94BFA2BF351F95DF451FA5966
:1056480001E2CAD6800E9C6FFD0E9D6F60C19EF070
:105658009F6B70EC63F0FA0E9C6FFD0E9D6FF4C1AA
:105668009EF09F6B70EC63F0DC0E9C6FFD0E9D6FDF
:1056780065C19EF09F6B70EC63F0EB0E9C6FFD0EA6
:105688009D6FC8C19EF09F6B70EC63F0FB6BFC6B69
:10569800FD0E9C6FFC0E9D6FFBC09EF0FCC09FF042
:1056A8000F0EFB03F3CFC2F0F4CFC3F0FC03F350AB
:1056B800C327350EC225A06F0D0EC321A16F70EC54
:1056C80063F0FB4BFC2BFCBFE3D7FC5103E1100E4E
:1056D800FB5DDEE3FA6B010EF96F0E0E9C6FFD0E9B
:1056E8009D6FF9C09EF0FAC09FF00F0EF903F3CF3B
:1056F800C2F0F4CFC3F0FA03F350C327250EC22536
:10570800A06F0E0EC321A16F70EC63F0F94BFA2B5A
:10571800FABFE3D7FA5103E1040EF95DDEE3FC0EAC
:105728009C6FF90E9D6F70EF63F0838E838066EC3B
:105738003FF0FC6FFC5118E052501C0D1B0EF32477
:10574800D96E020EF420DA6E52501C0D1B0EF32493
:10575800E16E020EF420E26EE7500409DF6E22ECDF
:1057680062F00001FC51120001015E514EE0385117
:1057780039113A113B1149E0525047E152501C0D82
:10578800070EF324D96E020EF420DA6E38C172F1D6
:1057980039C173F13AC174F1716B000E7125756FDF
:1057A800010E7221766F000E7321776F000E74213F
:1057B800786F796B7A6B7B6B7C6BDE50751925E1A2
:1057C800DE50761922E1DE5077191FE1DE50781994
:1057D8001CE1DE50791919E1DE507A1916E1DE5024
:1057E8007B1913E1DE507C1910E1350E2B6E0B0E80
:1057F8002C6E5E5107EC51F00292000E1DEC5BF02E
:105808000292506A83905050120052501C0D170E8D
:10581800F324D96E020EF420DA6EDECF69F1DECF02
:105828006AF1DECF6BF1DECF6CF16AC169F16BC151
:105838006AF16CC16BF16C6B69C1F0F06AC1F1F08F
:105848006BC1F2F06CC1F3F052501C0D170EF3242B
:10585800D96E020EF420DA6EDECF69F1DDCF6AF17F
:1058680069510001F66FF76B0292F86BF96BFA6BEE
:10587800FB6BF46BF56B94D0F4C069F1F5C06AF179
:10588800000E6ABFFF0E6B6F6C6FFF0E0001F025F4
:1058980001016D6FFF0E0001F12101016E6FFF0E16
:1058A8000001F22101016F6FFF0E0001F3210101D8
:1058B800706F69516D1910E16A516E190DE16B51E4
:1058C8006F190AE16C51701907E10001F651F711DF
:1058D80003E102500209026E5250220D000EF32419
:1058E8000001746F030EF420756F350E766F0B0E82
:1058F800776F010E796F786BFD0E7A6F7B6BA3EC77
:105908001AF0FF6FFF5101E017D7FD51FE1101E1B9
:1059180013D7FD511DEC5BF00001FD51F827FE5136
:10592800F923000EFA23FB2352501C0D070EF32413
:10593800D96E020EF420DA6E000EDE240101696FC2
:10594800010EDE206A6F000EDE206B6F000EDE2077
:105958006C6F000EDE206D6F000EDE206E6F000E85
:10596800DE206F6F000EDE20706F52501C0D070E88
:10597800F324D96E020EF420DA6E69C1DEFF6AC123
:10598800DEFF6BC1DEFF6CC1DEFF6DC1DEFF6EC1E5
:10599800DEFF6FC1DEFF70C1DEFF0001F44BF52BA7
:1059A800F4C069F1F5C06AF1000E01016ABFFF0E8B
:1059B8006B6F6C6F0001F0510101695D0001F151DD
:1059C80001016A590001F25101016B590001F351BB
:1059D80001016C5901E250D70001F651F71160E05E
:1059E8005250220D000EF324746F030EF420756FCD
:1059F800350E766F0B0E776FF6C078F0F7C079F03A
:105A0800FD0E7A6F7B6BA3EC1AF0FF6FFF5101E07C
:105A180093D602500209026EF6511DEC5BF00001AC
:105A2800FD51F827FE51F923000EFA23FB235250AB
:105A38001C0D070EF324D96E020EF420DA6E000E48
:105A4800DE240101696F010EDE206A6F000EDE2080
:105A58006B6F000EDE206C6F000EDE206D6F000E87
:105A6800DE206E6F000EDE206F6F000EDE20706F7E
:105A780052501C0D070EF324D96E020EF420DA6E74
:105A880069C1DEFF6AC1DEFF6BC1DEFF6CC1DEFFEC
:105A98006DC1DEFF6EC1DEFF6FC1DEFF70C1DEFFCC
:105AA8000292506A8390839EAED645C0D9FF46C005
:105AB800DAFFDECF72F0DDCF73F04A50491048109C
:105AC80003E1020E475C10E3000120EE13F072516F
:105AD800D9267351DA22DE50475CDE504858DE5032
:105AE8004958DE504A5808E3010E00016C6F000E59
:105AF8006D6B6E6B6F6B8FD16C696D696E696F6959
:105B080076D147C070F048C071F0D8907131616F9C
:105B18007031606F605170276151712372C03AF023
:105B280073C03BF020EE1FF07251D9267351DA2270
:105B3800DECF60F0DECF61F0DECF62F0DECF63F063
:105B480070C064F071C065F0090E666FD890653357
:105B58006433662FFBD7645160253C6E6551612123
:105B68003D6E000E62213E6E000E63213F6ED1EC49
:105B780056F0000901E04FD100016069010E616F24
:105B880070C062F071C063F06051621761516317B1
:105B980072C064F073C065F0625164276351652375
:105BA8002F0E6425D96E000E6521DA6EDF506A6FFC
:105BB8006B6B704B712B72C03AF073C03BF020EEE8
:105BC8001FF07251D9267351DA22DECF60F0DECF92
:105BD80061F0DECF62F0DECF63F070C064F071C0B8
:105BE80065F0090E666FD89065336433662FFBD76E
:105BF800645160253C6E655161213D6E000E622145
:105C08003E6E000E63213F6ED1EC56F0000901E0B4
:105C180002D100016069010E616F70C062F071C04D
:105C280063F0605162176151631772C064F073C00A
:105C380065F062516427635165232F0E6425D96E80
:105C4800000E6521DA6EDF50676F666B66516A1366
:105C580067516B1347B006D06A51686F0F0E6B150A
:105C6800696F0FD06AC060F06BC061F0040E626F9C
:105C7800D89061336033622FFBD760C068F061C091
:105C880069F068C06CF069C06DF04ED072C03AF02F
:105C980073C03BF020EE1FF07251D9267351DA22FF
:105CA800DECF60F0DECF61F0DECF62F0DECF63F0F2
:105CB8004850646F4950656F4A50666F676B605112
:105CC80064253C6E615165213D6E625166213E6ED0
:105CD800635167213F6ED1EC56F0000901E09BD07B
:105CE80000016069010E616F47C062F048C063F04F
:105CF800D89062376337605162176151631772C079
:105D080064F073C065F062516427635165232F0EF8
:105D180064250E6E000E65210F6E91EC61F00EC0C9
:105D28006CF00FC06DF000016E6B6F6B74D072C0B9
:105D38003AF073C03BF020EE1FF07251D926735130
:105D4800DA22DECF60F0DECF61F0DECF62F0DECFA8
:105D580063F047C064F048C065F049C066F04AC0C7
:105D680067F0080E05D0D89067336633653364331F
:105D7800E82EF9D7605164253C6E615165213D6E6E
:105D8800625166213E6E635167213F6ED1EC56F039
:105D9800000941E100016069010E616F47C062F0CE
:105DA80048C063F0D89062376337D890623763375A
:105DB800605162176151631772C064F073C065F077
:105DC80062516427635165232F0E64250E6E000E01
:105DD80065210F6EDCEC55F00E5000016C6F0F5012
:105DE8006D6F10506E6F0F0E11146F6F14D072C05C
:105DF800D9FF73C0DAFFDF50606F616B615101E05A
:105E080073D66051010A01E17CD6030A01E13ED74D
:105E1800010A8DE069D66CC045F06DC046F06EC0D1
:105E280047F06FC048F01200526A4F6A526A030E78
:105E3800526401D090D1525003E1216A226A03D002
:105E4800226A010E216E52501C0D1B0EF324D96ECE
:105E5800020EF420DA6EDF6A52501C0D000EF32495
:105E6800D96E020EF420DA6EDF6A52501C0D070E4E
:105E7800F324D96E020EF420DA6E070EDE6AE80605
:105E8800FDE20D0E2102F3CF69F1F4CF6AF122028F
:105E9800F35001016A279B0E6925D96E020E6A210B
:105EA800DA6EDF506B6F6BC16CF16D6B6E6B6F6B85
:105EB8006EC16FF16DC16EF16CC16DF16C6B6CC12F
:105EC80070F16DC171F16EC172F16FC173F1746BD4
:105ED80073BF746974C175F174C176F174C177F1D7
:105EE8000D0E2102F3CF78F1F4CF79F12202F350AD
:105EF80079279A0E7825D96E020E7921DA6EDF504D
:105F08007A6F7AC17BF17C6B7D6B7E6B7CC17EF195
:105F18007BC17DF17C6B7B6B7BC17FF17CC180F1A8
:105F28007DC181F17EC182F1836B82BF836983C1A8
:105F380084F183C185F183C186F10D0E2102F3CF6F
:105F480087F1F4CF88F12202F3508827990E87252C
:105F5800D96E020E8821DA6EDF50896F89C18AF105
:105F68008B6B8C6B8D6B8AC18DF18C6B8B6B8A6B99
:105F78008AC18EF18BC18FF18CC190F18DC191F1E5
:105F8800926B91BF926992C193F192C194F192C1BF
:105F980095F10D0E2102F3CF96F1F4CF97F122027D
:105FA800F3509727980E9625D96E020E9721DA6E30
:105FB800DF50986F98C199F19A6B9B6B9C6B9D6BA6
:105FC8009E6B9F6BA06B200ED89099379A379B37A2
:105FD8009C379D379E379F37A037E82EF5D78E51CF
:105FE8009925A16F8F519A21A26F90519B21A36F80
:105FF80091519C21A46F92519D21A56F93519E218F
:10600800A66F94519F21A76F9551A021A86F7F512A
:10601800A125A96F8051A221AA6F8151A321AB6F3D
:106028008251A421AC6F8351A521AD6F8451A62163
:10603800AE6F8551A721AF6F8651A821B06F7051FF
:10604800A925B16F7151AA21B26F7251AB21B36FFB
:106058007351AC21B46F7451AD21B56F7551AE2138
:10606800B66F7651AF21B76F7751B021B86F5250E4
:106078001C0D0F0EF324D96E020EF420DA6EB1C196
:10608800DEFFB2C1DEFFB3C1DEFFB4C1DEFFB5C1C2
:10609800DEFFB6C1DEFFB7C1DEFFB8C1DEFFB40E5A
:1060A80000019C6FFA0E9D6F52C09EF09F6B52507C
:1060B8001C0D0F0EF324D96E020EF420DA6EDECF1B
:1060C80069F1DECF6AF1DECF6BF1DECF6CF1DECFA6
:1060D8006DF1DECF6EF1DECF6FF1DECF70F169C109
:1060E800A0F06AC1A1F06BC1A2F06CC1A3F06DC1B0
:1060F800A4F06EC1A5F06FC1A6F070C1A7F0525010
:106108001C0D0F0EF324D96E020EF420DA6EDECFCA
:1061180071F1DECF72F1DECF73F1DECF74F1DECF35
:1061280075F1DECF76F1DECF77F1DECF78F171C190
:10613800A8F072C1A9F073C1AAF074C1ABF075C11F
:10614800ACF076C1ADF077C1AEF078C1AFF070ECCD
:1061580063F0522A6CD601015D6B516A5C6B4A6B25
:106168004B6B020E506E5B6F8390020C9EC0D9FF82
:106178009FC0DAFFDECFB2F0DDCFB3F020EE0EF035
:106188009E51D9269F51DA22DECFA2F0DECFA3F0AE
:10619800DECFA4F0DECFA5F0200EA225AE6F000E54
:1061A800A321AF6F000EA421B06F000EA521B16F1F
:1061B800B15103E1200EB05D0AE320EE16F09E51C6
:1061C800D9269F51DA22DE6ADE6ADE6ADD6A20EEAF
:1061D80016F09E51D9269F51DA22DE50DE10DE10CD
:1061E800DE1001E1040CAE51A26F010EAF15A36FD2
:1061F800A46BA56BA211A411A51101E029D120EE71
:1062080016F09E51D9269F51DA22DE2A000EDE2290
:10621800DE22DE2220EE12F09E51D9269F51DA228C
:10622800DE50DE10DE10DE102CE120EE07F0B25159
:10623800D926B351DA22DECFA2F0DDCFA3F0A251E6
:10624800A46FA351A56FA66BA76BAEC0A8F0AFC093
:10625800A9F0B0C0AAF0B1C0ABF0060E05D0D89036
:10626800AB33AA33A933A833E82EF9D7A451A85DD4
:10627800A551A959A651AA59A751AB5901E2E8D08D
:106288006ED0A269A36920EE09F0B251D926B351A4
:10629800DA22DECFA4F0DDCFA5F0A251A427A351C6
:1062A800A523AEC0A6F0AFC0A7F0B0C0A8F0B1C09B
:1062B800A9F00A0E05D0D890A933A833A733A6337E
:1062C800E82EF9D7A451A615AA6FA551A715AB6F4B
:1062D800AC6BAD6BAA11AC11AD1101E0B9D09EC089
:1062E80045F09FC046F020EE12F09E51D9269F51EE
:1062F800DA22DECF47F0DECF48F0DECF49F0DECF3E
:106308004AF059EC2DF045C0B4F046C0B5F047C08E
:10631800B6F048C0B7F00001B751B611B51104E1A5
:10632800020EB45D01E2020CB42907E1B52905E1CA
:10633800B62903E1B72901E1010C20EE13F0B251AF
:10634800D926B351DA22DE50B45DDE50B559DE509D
:10635800B659DE50B75950E3A051A1110BE120EE18
:1063680016F09E51D9269F51DA22DE6ADE6ADE6A6D
:10637800DD6A040C9EC081F09FC082F020EE12F00E
:106388009E51D9269F51DA22DECF83F0DECF84F0EA
:10639800DECF85F0DECF86F0ACEC25F081C0B4F01E
:1063A80082C0B5F083C0B6F084C0B7F0B451B5115F
:1063B800B611B71101E1070CB405B511B611B71143
:1063C80001E1020CB42907E1B52905E1B62903E189
:1063D800B72901E1010CB2C03AF0B3C03BF0B4C038
:1063E8003CF0B5C03DF0B6C03EF0B7C03FF007EC9A
:1063F8004FF0000901E0010C000120EE12F09E515F
:10640800D9269F51DA22B4C0DEFFB5C0DEFFB6C080
:10641800DEFFB7C0DEFFB2C00EF0B3C00FF0B4C0ED
:1064280010F0B5C011F0B6C012F0B7C013F075EC9B
:106438004DF0000120EE16F09E51D9269F51DA2228
:106448000EC0DEFF0FC0DEFF10C0DEFF11C0DEFF92
:1064580020EE0EF09E51D9269F51DA22AEC0DEFF03
:10646800AFC0DEFFB0C0DEFFB1C0DEFFA269010E23
:10647800A36FAEC0A4F0AFC0A5F0A251A417A3515A
:10648800A517B2C0A6F0B3C0A7F0A451A627A5517E
:10649800A7232F0EA627000EA72320EE1AF09E5141
:1064A800D9269F51DA22A6C0DEFFA7C0DDFF000C67
:1064B80052500C0D030EF324D96E010EF420DA6E3F
:1064C800DF50696F69C16AF16B6B6C6B6D6B6CC186
:1064D8006DF16BC16CF16AC16BF16A6B52500C0DB6
:1064E8000B0EF324D96E010EF420DA6EDF506E6FB6
:1064F8006EC16FF1706B716B726B52500C0D020EA6
:10650800F324D96E010EF420DA6EDF50736F73C175
:1065180074F1756B766B776B76C177F175C176F12F
:1065280074C175F1746B74516F03F3CF78F1F4CFC4
:1065380079F17A6B7B6B7003F3507927F4507A23E7
:10654800000E7B2375516F03F3507927F4507A239B
:10655800000E7B2374517103F3507A27F4507B2388
:1065680075517003F3507A27F4507B2376516F03EB
:10657800F3507A27F4507B2372517403F3507B272E
:1065880075517103F3507B2776517003F3507B27C5
:1065980077516F03F3507B2752500C0D0A0EF324EA
:1065A800D96E010EF420DA6EDF507C6F7CC17DF16C
:1065B8007E6B7F6B806B52500C0D0B0EF324D96EE3
:1065C800010EF420DA6EDF50816F81C182F1836B96
:1065D800846B856B52500C0D000EF324D96E010E9E
:1065E800F420DA6EDECF86F1DDCF87F186C188F13F
:1065F80087C189F1000E89BFFF0E8A6F8B6F8851A2
:106608008203F3CF8CF1F4CF8DF18E6B8F6B830304
:10661800F3508D27F4508E23000E8F238951820367
:10662800F3508D27F4508E23000E8F238851840356
:10663800F3508E27F4508F2389518303F3508E270C
:10664800F4508F238A518203F3508E27F4508F23FE
:1066580085518803F3508F2789518403F3508F277E
:106668008A518303F3508F278B518203F3508F276E
:106678008EC18FF18DC18EF18CC18DF18C6B8C51D7
:106688007D03F3CF90F1F4CF91F1926B936B7E037E
:10669800F3509127F4509223000E93238D517D03DC
:1066A800F3509127F4509223000E93238C517F03CB
:1066B800F3509227F45093238D517E03F350922781
:1066C800F45093238E517D03F3509227F450932373
:1066D80080518C03F35093278D517F03F3509327F8
:1066E8008E517E03F35093278F517D03F3509327E8
:1066F80078519025946F79519121956F7A51922113
:10670800966F7B519321976F6A5194250001DC6F36
:1067180001016B5195210001DD6F01016C5196213A
:106728000001DE6F01016D5197210001DF6F5250AA
:10673800220D000EF3249E6F030EF4209F6FDCC021
:10674800A0F0DDC0A1F0DEC0A2F0DFC0A3F075ECC0
:1067580012F0DB6FDB5111E0720E9C6FFB0E9D6F28
:10676800DCC09EF0DDC09FF0DEC0A0F0DFC0A1F06D
:10677800DBC0A2F0A36B70EC63F0AC0E9C6FFE0E56
:106788009D6F70EC63F0839052500C0D040EF3244F
:10679800D96E010EF420DA6EDCC0DEFFDDC0DEFF4C
:1067A800DEC0DEFFDFC0DEFF0101596B586B91EFE1
:1067B8003CF0000E0001E06F250EDF6F000EDE6F6B
:1067C800050EDD6F0101F45105E1000E0001E06FD7
:1067D800280EDF6F010160510DE1F36B350E0001EA
:1067E8007C6F0D0E7D6F9F0E7E6FFE0E7F6F98EC97
:1067F80060F00DD0D40E00019C6FFA0E9D6F60C141
:106808009EF09F6BF3C1A0F0A16B70EC63F0180EC3
:106818009C6FFE0E9D6F0101F3510F0D350EF32491
:1068280000019E6F0D0EF4209F6F70EC63F0050E53
:106838000001DC6F0F0EDB6FF10EE82EFED7DB2FA9
:10684800FCD7DC2FFAD7E3D0EC0E0F6EFC0E106EDF
:10685800F5EC5DF0030E0101C86105D09650C8192A
:10686800F00BC81905D0C8C193FF9650F00B0A0960
:10687800966E000E0001CE6F030ECF6F920ED06F92
:10688800FE0ED16F010ED26F43EC15F00101646F5B
:10689800645171EC5EF0010164510AE1C7EC36F015
:1068A800000E6D6F030E6E6F7BEC60F00101646F7C
:1068B800645171EC5EF0E06B280EDF6FA4D001012B
:1068C800F3510F0D350EF324D96E0D0EF420DA6E48
:1068D800200EDE1806E1F32B0F0EF36594D0F36B50
:1068E80092D0000E00019C6FFC0E9D6F0101F351C8
:1068F8000F0D350EF32400019E6F0D0EF4209F6FCF
:1069080070EC63F0000ECE6F030ECF6F0101F351F0
:106918000F0D350EF3240001D06F0D0EF420D16F4A
:10692800030ED26F43EC15F00101646F645171ECF2
:106938005EF00101645104E10001E06B3C0EDF6F81
:10694800040E0101641904E10001E06B320EDF6FEF
:10695800050E0001DC6F0F0EDB6FF10EE82EFED77F
:10696800DB2FFCD7DC2FFAD74ED0A70E9C6FFC0E7E
:106978009D6F0101F3510F0D350EF32400019E6F39
:106988000D0EF4209F6F70EC63F0000ECE6F030EB7
:10699800CF6F0101F3510F0D350EF3240001D06FB5
:1069A8000D0EF420D16F070ED26F43EC15F00101E4
:1069B800646F6451CDE10001E06B3C0EC8D7820ED4
:1069C8009C6FFC0E9D6F0101F3510F0D350EF324E2
:1069D80000019E6F0D0EF4209F6F70EC63F013D0D2
:1069E800DFC0DBF0E0C0DCF0DC510DE1DB51250A53
:1069F80001E12AD70D0A01E162D7050A04E01F0A5E
:106A0800B4E00E0ADCE00001DD07D8A0DE070001D3
:106A1800DEBF08D0DE5102E1DD0504E33C0EDF19DC
:106A2800E011DEE1030E010160193BE1839E000ED7
:106A38000E6EC00EC2EC5EF08FEC62F0000E0E6EB1
:106A4800C00EC2EC5EF03C0E0001DF19E01116E149
:106A58000101E9510CE0E90E126E010E136E6AECA9
:106A68005AF0C20E126EFE0E136E6AEC5AF0A00EA9
:106A7800126EFF0E136E6AEC5AF0000C350E7C6F26
:106A88000D0E7D6F410E7E6FFF0E7F6F64C180F02B
:106A9800816B98EC60F0350E126E0D0E136E6AEC79
:106AA8005AF0000C74C0D9FF75C0DAFFDECF8CF045
:106AB800DDCF8DF0795109E1200E785DD8B0020C58
:106AC80076C07AF01F0E7A1701E0020C20EE0EF065
:106AD8007451D9267551DA2276C0DEFF77C0DEFF01
:106AE80078C0DEFF79C0DEFF20EE06F07451D926AB
:106AF8007551DA22DECF88F0DECF89F0DECF8AF05A
:106B0800DECF8BF0885189118A118B1115E18CC069
:106B1800D9FF8DC0DAFF020EDF640ED020EE23F01D
:106B28008C51D9268D51DA22DECF88F0DECF89F05C
:106B3800DECF8AF0DECF8BF0885189118A118B1154
:106B480040E120EE07F08C51D9268D51DA22DECFB4
:106B58007AF0DDCF7BF07A517C6F7B517D6F7E6B55
:106B68007F6B76C080F077C081F078C082F079C002
:106B780083F0060E05D0D890833382338133803377
:106B8800E82EF9D77C51805D7D5181597E5182591B
:106B98007F51835901E3020C20EE23F08C51D92652
:106BA8008D51DA2210EE16F07451E1267551E22269
:106BB800DECFE6FFDECFE6FFDECFE6FFDECFE6FF85
:106BC80087D020EE09F08C51D9268D51DA22DECFFC
:106BD8007AF0DDCF7BF07A517C6F7B517D6F7E6BD5
:106BE8007F6B090ED8907C377D377E377F37E82E4C
:106BF800F9D77CC084F07DC085F07EC086F07FC068
:106C080087F040D074C045F075C046F088C047F0A2
:106C180089C048F08AC049F08BC04AF059EC2DF081
:106C280045C088F046C089F047C08AF048C08BF05C
:106C38000001882907E1892905E18A2903E18B29CF
:106C480001E1010C8B518A11891104E1020E885D62
:106C5800D8A0020C20EE13F08C51D9268D51DA22DF
:106C6800DE50885DDE508959DE508A59DE508B59D6
:106C780001E3020C8451765F8551775B8651785B1E
:106C88008751795B8451765D85517759865178595A
:106C980087517959B7E28CC00EF08DC00FF088C0CB
:106CA80010F089C011F08AC012F08BC013F075EC97
:106CB8004DF0000120EE16F07451D9267551DA22F4
:106CC8000EC0DEFF0FC0DEFF10C0DEFF11C0DEFF0A
:106CD80020EE12F07451D9267551DA2288C0DEFFF1
:106CE80089C0DEFF8AC0DEFF8BC0DEFF20EE16F013
:106CF8007451D9267551DA22DE50DE10DE10DE100E
:106D080001E1020C76C07AF077C07BF078C07CF0A5
:106D180079C07DF00A0E05D0D8907D337C337B3363
:106D28007A33E82EF9D720EE16F07451D92675512A
:106D3800DA227A51DE267B51DE227C51DE227D5119
:106D4800DE227A69010E7B6F76C07CF077C07DF019
:106D58007A517C177B517D178CC07EF08DC07FF0F7
:106D68007C517E277D517F232F0E7E27000E7F23A7
:106D780020EE1AF07451D9267551DA227EC0DEFF52
:106D88007FC0DDFF000C3B0EF66EF90EF76E0900B2
:106D9800F5CFC5F00A00F5CFC6F00001C96BCD6B81
:106DA8000101E96B030EC86105D09650C819F00BB4
:106DB800C81905D0C8C193FF9650F00B0A09966E02
:106DC800CD6ACE6A1FD1CC6B350E176E0B0E186EBE
:106DD800C50E196EB5EC57F017C0CAF018C0CBF045
:106DE800CAC0D9FFCBC0DAFF3B0EDE1801E005D1DF
:106DF80009D1CC5113E1CAC012F0CBC013F0CAECD0
:106E08005BF00001CD6F800ECD6503D0CD51800FB2
:106E1800C96F030EC965E6D0C96BE4D0CC051BE188
:106E28000101F3510001CD1903E07F0ECD1913E1E3
:106E3800CAC012F0CBC013F0CAEC5BF00101636F5B
:106E48005A0E00019C6FFF0E9D6F63C19EF09F6BF1
:106E580070EC63F0C7D0020ECC191BE10101F351AD
:106E68000001CD1903E07F0ECD1913E1CAC012F05D
:106E7800CBC013F0CAEC5BF00101626F620E000137
:106E88009C6FFF0E9D6F62C19EF09F6B70EC63F06C
:106E9800A9D0020ECC652CD0080ECC6129D00101F6
:106EA800F3510001CD190CE07F0ECD1909E0810ED8
:106EB800CD1906E0820ECD1903E0830ECD1918E135
:106EC800C951050DCA0EF324C76F010EF420C86F0F
:106ED800CAC012F0CBC013F0CAEC5BF00001C26F5D
:106EE800CC51C725C36F000EC821C46FFD0E5AD000
:106EF800070ECC652CD01B0ECC6129D00101F351B3
:106F08000001CD190CE07F0ECD1909E0810ECD19D5
:106F180006E0820ECD1903E0830ECD1918E1C951A0
:106F2800130DAA0EF324C76F030EF420C86FCAC04E
:106F380012F0CBC013F0CAEC5BF00001C26FCC5169
:106F4800C725C36F000EC821C46FF80E2BD0280EBA
:106F5800CC6130D00101F3510001CD190CE07F0E56
:106F6800CD1909E0810ECD1906E0820ECD1903E096
:106F7800830ECD191FE1C9510D0D900EF324C76F73
:106F8800020EF420C86FCAC012F0CBC013F0CAECCE
:106F98005BF00001C26FCC51C725C36F000EC8213A
:106FA800C46FE50EC325D96EFF0EC421DA6EC2C0C8
:106FB800DFFF18D0280ECC1915E10101F3510001AB
:106FC800CD1903E07F0ECD190DE1E90E0E6E010E0D
:106FD8000F6ECAC010F0CBC011F0136A080E126E03
:106FE800A0EC5DF0CC2B176A186AC50E196EB5ECCB
:106FF80057F017C0CAF018C0CBF00001CA51CB1126
:1070080001E0F7D6350E00019F6F0B0EA06FA26B43
:10701800910EA16F000EA36F030EA46FFFEC57F043
:107028009F51A01101E0CFD6260E9C6FFB0E9D6FDD
:10703800E90E9E6F010E9F6F70EF63F0350E010130
:10704800756F0B0E766FE9C00EF0EAC00FF09CEC7E
:107058005FF00E500101696FC70E00019E6F9F6BB4
:10706800A06BA16BA26BA36B75EC12F00101726FA0
:1070780072510DE0400E00019C6FFB0E9D6F70EC8D
:1070880063F00001C76BC86BC96BCA6B1200C70EEF
:107098000001746F756B75C176F076C177F0010EDB
:1070A800796F786B700E7A6F010E7B6FA3EC1AF014
:1070B8000101726F725108E0E90E00019C6FFB0E2E
:1070C8009D6F70EC63F0DDD775C1D9FF76C1DAFF2B
:1070D800800EDE1808E0DB0E00019C6FFC0E9D6F31
:1070E80070EC63F0CED720EE0AF07551D9267651B0
:1070F800DA22DF500001EC6FEB6B010120EE0BF0A0
:107108007551D9267651DA22DF500001EB250101AD
:107118006E6F000E0001EC2101016F6FD20E0001AD
:107128009C6FFB0E9D6F6EC19EF06FC19FF070EC5F
:1071380063F0C70E9E6F9F6B01016E510001EC6FEB
:10714800EB6BEBC0A0F0ECC0A1F0A26BA36B75ECED
:1071580012F00101726F725194E1C70E0001746F51
:10716800756B75C176F076C177F0010E796F786B23
:10717800700E7A6F010E7B6FA3EC1AF00101726F2B
:10718800725101E07ED7736B746BE9C00EF0EAC0F0
:107198000FF073C1EBF074C1ECF0050ED89000014C
:1071A800EB37EC37E82EFAD7EB5101017525106E55
:1071B8000001EC5101017621116E69C112F0136AC8
:1071C80091EC58F00E500F105DE173C1EBF074C1F3
:1071D800ECF0050ED8900001EB37EC37E82EFAD723
:1071E80075C1EDF076C1EEF0EB51ED27EC51EE23D1
:1071F8000E0EED25D96E000EEE21DA6EDF50F06F1F
:10720800EF6B73C1F1F074C1F2F0050ED890F1374D
:10721800F237E82EFBD775C1F3F076C1F4F0F151DF
:10722800F327F251F4230F0EF325D96E000EF42143
:10723800DA6EDF50F56FF66BEF51F527F051F62354
:10724800F5C06AF1F6C06BF10101000E6BBFFF0ECD
:107258006C6F6D6FA00E00019C6FFD0E9D6F6AC173
:107268009EF06BC19FF06CC1A0F06DC1A1F070ECF5
:1072780063F06AC1C7F06BC1C8F06CC1C9F06DC1D9
:10728800CAF01200734B742B74BF7FD7745105E199
:107298000F0E735D01E3F5D678D7F3D61850D96E83
:1072A800DA6ADECF22F0DDCF23F01C0E1624266E1C
:1072B800000E1720276E26C00EF027C00FF0116AA7
:1072C800200E106E136A0B0E126EF2EC62F0286A32
:1072D800296A246A256A216A080E206E245022240D
:1072E800196E255023201A6E19C0F6FF1AC0F7FF31
:1072F800000EF86E0E0EF76403D00800F55005D0A6
:10730800F6CFE9FFF7CFEAFFEF502A6E244A252A85
:10731800210E2A6001D0BED02F0E2A1806E05C0E7E
:107328002A1803E036D0244A252A24502224196E2C
:10733800255023201A6E19C0F6FF1AC0F7FF000E59
:10734800F86E0E0EF76403D00800F55005D0F6CF9E
:10735800E9FFF7CFEAFFEF502F0AE5E02450222497
:10736800196E255023201A6E19C0F6FF1AC0F7FFB0
:10737800000EF86E0E0EF76403D00800F55005D025
:10738800F6CFE9FFF7CFEAFFEF505C0A01E082D0C1
:10739800CAD72E0E2A1805E02050285C21502958FB
:1073A8000FE30B0E20182110D8B4060C2E0E2A1845
:1073B80001E0060C296A080E286E216A0B0E8DD78B
:1073C8002A509AEC5EF00E500F1044E0245022240C
:1073D800196E255023201A6E19C0F6FF1AC0F7FF40
:1073E800000EF86E0E0EF76403D00800F55005D0B5
:1073F800F6CFE9FFF7CFEAFFEF501F6E244A252AA0
:107408001F5002EC5CF00E500F10D8B4060C19682F
:107418001A6820C01BF021C01CF019501B261A50F6
:107428001C221B50285C1C50295801E3060C2850CC
:107438002624D96E29502720DA6E2AC0DFFF284A71
:10744800292A28502624D96E29502720DA6E1FC0F1
:10745800DFFF1DD0BE0E0E6EFD0E0F6E2AC010F09F
:10746800116AEEEC60F00E500F1001E0060C600E91
:107478002A6405D07B0E2A6002D0200E2A5E28508E
:107488002624D96E29502720DA6E2AC0DFFF284A21
:10749800292A24D724502224196E255023201A6E15
:1074A8001850D96EDA6A19C0DEFF1AC0DDFF2850FD
:1074B800291001E1060C26C0D9FF27C0DAFFE50E26
:1074C800DE1806E126C0D9FF27C0DAFF050EDF6EF9
:1074D800200E2A6403D01D6A1E6A03D01E6A040E99
:1074E8001D6E20EE0BF02650D9262750DA221DC03B
:1074F800DFFF000C0101676B526B536BFF0E2124F9
:10750800256EFF0E2220266E8986898089828984CD
:1075180089888B68849084928494849883500F011E
:107528001391350EE82EFED700F007D0FC0E0001AF
:107538009C6FFF0E9D6F70EC63F08EA8F7D7E1D0BB
:107548008EA88EAA14D0F45112E1525153110FE0B3
:107558001F0E00019C6FFD0E9D6F52C19EF053C11E
:107568009FF070EC63F0630E0101676FD0D0100ECE
:107578003C6F270E3D6F3E6B3F6BABD08EB28EA437
:1075880010D03C07000E3D5B3E5B3F5B3C2906E1AB
:107598003D2904E13E2902E13F29D8A4B2D0620E78
:1075A80084D0010E82D08EA8ACD0020E7ED0350ECB
:1075B8005225D96E0B0E5321DA6EDF1C866E52519E
:1075C800251805E15351261802E102B2899A524B57
:1075D800532B8B6A030E676F100E3C6F270E3D6F9F
:1075E8003E6B3F6B06D08EA204D08990050E676F64
:1075F8000ED03C07000E3D5B3E5B3F5B3C29F3E150
:107608003D29F1E13E29EFE13F297BE0ECD7100E5F
:107618003C6F270E3D6F3E6B3F6B0DD08EA40BD099
:10762800898A89808B682150525D22505359BDE365
:10763800630E01013AD03C07000E3D5B3E5B3F5BA9
:107648003C29ECE13D29EAE13E29E8E13F2959E0FE
:10765800E5D78EB20DD03C07000E3D5B3E5B3F5B2D
:107668003C294FE13D294DE13E294BE13F2949E1C4
:10767800040E1BD08990050E676F100E3C6F270E05
:107688003D6F3E6B3F6B3DD089848EB40DD03C0777
:10769800000E3D5B3E5B3F5B3C2933E13D2931E118
:1076A8003E292FE13F292DE1060E676F2AD0898AEE
:1076B80089808B682150525D2250535901E271D75D
:1076C800B7D7A60E00019C6FFF0E9D6F70EC63F09C
:1076D800AFD76751236E246A245013E1235001E188
:1076E8004DD7010A01E15FD7030A01E160D7010A1A
:1076F800B0E0070ABFE0010AC7E0030AD8E0640A5D
:10770800E0E0630E0101671902E08EBC19D7898099
:10771800898289848988898A8B680F01138152C17B
:1077280021F053C122F0120002500209026E350EF8
:107738000E6E0B0E0F6E116A106A010E136E126A2E
:10774800A6EC4AF0000EE8CF35FBFF0EE8CF36FB7B
:1077580052501C0D1B0EF324D96E020EF420DA6E63
:107768000201DFA403D0010EE8CF37FB52501C0DF5
:107778001B0EF324D96E020EF420DA6EDFA803D0B4
:10778800020EE8CF37FB52501C0D1B0EF324D96EA6
:10779800020EF420DA6EDFA003D0020EE8CF39FB28
:1077A80052501C0D1B0EF324D96E020EF420DA6E13
:1077B800DFA203D0020EE8CF39FB52501C0D1B0E7E
:1077C800F324D96E020EF420DA6EDFA603D0800E01
:1077D800E8CF38FB8FA403D0080EE8CF3BFB236A21
:1077E800246A300E2324D96E010E2420DA6EDF1CA1
:1077F800226E370E2324D96E0B0E2420DA6E370E34
:107808002324E16E0B0E2420E26EE7502214DF6E73
:10781800234A242A24BEE5D7245003E1070E235C1B
:10782800E0E3506A020E4F6448D052501C0D010E1E
:10783800F324D96E020EF420DA6EDF50216E21C0D7
:1078480040FB52501C0D020EF324D96E020EF42098
:10785800DA6EDF50216E21C041FB52501C0D030E21
:10786800F324D96E020EF420DA6EDF50216E21C0A7
:1078780042FB52501C0D040EF324D96E020EF42064
:10788800DA6EDF50216E21C043FB52501C0D050EED
:10789800F324D96E020EF420DA6EDF50216E21C077
:1078A80044FB52501C0D060EF324D96E020EF42030
:1078B800DA6EDF50216E21C045FB140E1DEC5BF023
:1078C800260E00019C6FFF0E9D6F70EC63F0236A1B
:1078D800246AD70E9C6FFC0E9D6F350E2324D96E3B
:1078E8000B0E2420DA6EDF509E6F9F6B70EC63F0F6
:1078F800234A242A24BEEDD7245003E1130E235C27
:10790800E8E352501C0D1B0EF324D96E020EF4202E
:10791800DA6EDF6A02928390000C0001D16B010ECF
:10792800D06F838E8380D26BD36BD46BD56BE1D051
:107938005250220D000EF324746F030EF420756F5D
:10794800350E766F0B0E776F010E796F786BD80E48
:107958007A6F7B6BA3EC1AF0DA6FDA5118E0180E25
:107968000101576F010E596F0001D96BD86F920E44
:107978009C6FFA0E9D6F52C09EF09F6BDAC0A0F00C
:10798800A16BD8C0A2F0D9C0A3F070EC63F00101DC
:107998005E5135E0385139113A113B1130E05250FF
:1079A8000C0D040EF324D96E010EF420DA6E38C1E2
:1079B800C7F039C1C8F03AC1C9F00001C66B000E62
:1079C800C625CA6F010EC721CB6F000EC821CC6F28
:1079D800000EC921CD6FDE50CA1911E1DE50CB1956
:1079E8000EE1DE50CC190BE1DE50CD1908E1350E61
:1079F8002B6E0B0E2C6E01015E5107EC51F00292BA
:107A08000101575103E002500209026ED8C021F06B
:107A1800D9C022F07EEC3AF021C0D6F022C0D7F0CF
:107A2800FC0E00019C6FFE0E9D6F70EC63F0D6514A
:107A3800D227D751D323000ED423D5238EBC8EA8AA
:107A48005DD0D851D61903E1D951D7190CE05E0E93
:107A58009C6FFE0E9D6FD6C09EF0D7C09FF070EC55
:107A680063F083944BD027EC63F035EC5FF0215042
:107A7800221004E0010E0101596F40D00001CF6BC4
:107A8800050ECE6F1CD0D00E0001C26FC90EE82EB5
:107A9800FED7C22FFCD700D035EC5FF02150221062
:107AA8000EE00001D06BD16B300E9C6FFD0E9D6F08
:107AB800CEC09EF0CFC09FF070EC63F008D00001FC
:107AC800CE07D8A0CF07CE29DEE1CF29DCE18EB8DA
:107AD80008D01D0E9C6FFF0E9D6F70EC63F0D06B8D
:107AE800D16B35EC5FF02150221003E00001D06B20
:107AF800D16B0001D051D11101E01AD70101596BA6
:107B0800839E83901200276E0001C35102E018EC97
:107B18002FF0266A0001C25101E1CED0040E2718C9
:107B280002E1515003E1140E271809E101015C6BD1
:107B38004A6B4B6B0001C36B070EC26F070C3F0EFD
:107B4800271807E1516A01015C6B0001C26BC36B26
:107B580012005F0E271807E101015D6B5C6B0001E5
:107B6800C26BC36B12003F0E276406D05F0E2760FE
:107B780003D0400E2718F0E1400E271809E1010E46
:107B880001015D6F01015C6B0001C26BC36B1200E8
:107B9800200E271803E1010E516EF4D7650E271841
:107BA80009E1515007E001014A6B4B6B010E5C6F14
:107BB8008380EAD76E0E271803E1020E01015C6F7D
:107BC800700E271807E101015D5104E04A6B4B6B09
:107BD800030E5C6F700E271808E1515006E0838091
:107BE80001014A6B4B6B040E0DD0720E271864E12D
:107BF800515062E083804F6A1C0E01014B6F2A0EC0
:107C08004A6F050E5C6FC0D72750CEEC08F0266E81
:107C180065D083802750A7EC59F0266E01015C6B74
:107C28005DD08380350E0E6E0B0E0F6E116A106AD2
:107C3800010E136E126AA6EC4AF002500209026E97
:107C48002BEE35F050C0DFFF010E1DEC5BF0029209
:107C5800080E266E01015C6B506A40D08390266A3C
:107C68003DD0080E271815E18390526A266A506A9B
:107C7800030E4F6409D00F0E4F1806E0010E506E28
:107C880002011B5110091B6F010109D04A6B4B6B94
:107C980025D0090E271805E18390266A506A5C6B87
:107CA800F5D71F0E27641AD0300E276017D027503B
:107CB8000F0B4F6E266AD0D701015C51246E256ADE
:107CC80025500CE124500AE0010A9EE0030AA1E0D5
:107CD800010AA7E0070AC2E0010AC3E026C0C2F011
:107CE8000001C36B1200838E8380506A66EC3FF0FC
:107CF8000101856F855102E085511200686B7D6B2B
:107D08007E6B7F6B806B836B010E826F886BCFD02D
:107D1800866B876B1CD035EC5FF02150221015E084
:107D2800880E0E6E010E0F6E1FEC59F00101816F67
:107D3800000E6825D96EDA6A040EDA2281C1DFFFE7
:107D4800682B864B872B88BB05D08EAC03D00101EE
:107D58008705E1E3010186517D2787517E23000EC7
:107D68007F23802352501C0D170EF324D96E020E68
:107D7800F420DA6EDE507D5DDE507E59DE507F598C
:107D8800DE50805902E3826B836B88AB02D0826B32
:107D9800836B8EBC02D0826B836B870519E2000E61
:107DA80068250E6E0F6A040E0F22FF0E6825D96E25
:107DB800DA6A030EDA22DF50106E116A6851000881
:107DC800126E000ED8A0E82A0108136EA6EC4AF03D
:107DD80001015E5145E0385139113A113B1140E03B
:107DE80052503EE152501C0D070EF324D96E020E7C
:107DF800F420DA6E38C172F139C173F13AC174F105
:107E0800716B000E7125756F010E7221766F000E71
:107E18007321776F000E7421786F796B7A6B7B6BA7
:107E28007C6BDE5075191CE1DE50761919E1DE50C5
:107E3800771916E1DE50781913E1DE50791910E14F
:107E4800DE507A190DE1DE507B190AE1DE507C190B
:107E580007E1000E256E040E266E5E51D8EC58F030
:107E680072EC54F00101846F845121E08A0E000104
:107E78009C6FFB0E9D6F84C19EF09F6B70EC63F04E
:107E8800010E506E52501C0D1B0EF324D96E020EBB
:107E9800F420DA6E52501C0D1B0EF324E16E020E14
:107EA800F420E26EE7500409DF6E50501200825150
:107EB800831101E02DD78FA402D0010E506E83905C
:107EC800839E000C52501C0D070EF324D96E020E2F
:107ED800F420DA6EDECFEBF0DECFECF0DECFEDF0A3
:107EE800DECFEEF052501C0D070EF324D96E020EB1
:107EF800F420DA6E52501C0D0F0EF324E16E020EC0
:107F0800F420E26EDE50E65CDE50E658DE50E658BD
:107F1800DE50E658DE50E658DE50E658DE50E658A9
:107F2800DE50E65815E2010E506E52501C0D1B0E25
:107F3800F324D96E020EF420DA6E52501C0D1B0E7B
:107F4800F324E16E020EF420E26EE7500409DF6EBE
:107F580052501C0D070EF324D96E020EF420DA6E6F
:107F6800DECFC7F0DECFC8F0DECFC9F0DECFCAF073
:107F7800DECFCBF0DECFCCF0DECFCDF0DECFCEF053
:107F880052501C0D170EF324D96E020EF420DA6E2F
:107F9800DECFCFF0DECFD0F0DECFD1F0DECFD2F023
:107FA8000001CF51D36FD051D46FD151D56FD25179
:107FB800D66FD76BD86BD96BDA6BC751D325DB6F0C
:107FC800C851D421DC6FC951D521DD6FCA51D621E2
:107FD800DE6FCB51D721DF6FCC51D821E06FCD5167
:107FE800D921E16FCE51DA21E26F52501C0D0F0EEC
:107FF800F324D96E020EF420DA6EDB51DE5CDC511C
:10800800DE58DD51DE58DE51DE58DF51DE58E051D2
:10801800DE58E151DE58E251DE5815E2010E506E8D
:1080280052501C0D1B0EF324D96E020EF420DA6E8A
:1080380052501C0D1B0EF324E16E020EF420E26E6A
:10804800E7500409DF6E506A5250220D000EF324E7
:108058009E6F030EF4209F6FEBC0A0F0ECC0A1F060
:10806800EDC0A2F0EEC0A3F075EC12F0EF6FEF5187
:1080780015E0010E506E52501C0D1B0EF324D96EE4
:10808800020EF420DA6E52501C0D1B0EF324E16E22
:10809800020EF420E26EE7500409DF6E5050120021
:1080A8008EA604D0C10E216EFE0E03D0BB0E216E2B
:1080B800FF0E226E8EAA04D0C10E236EFE0E03D0D0
:1080C800B60E236EFF0E246E8EA804D0C10E256E48
:1080D800FE0E03D0EE0E256EFE0E266E8EAE04D07A
:1080E800C10E276EFE0E03D0C00E276EFF0E286E3F
:1080F8008EAC04D0C10E296EFE0E03D0B10E296ECF
:10810800FF0E2A6E8EA404D0C10E2B6EFE0E03D075
:10811800CA0E2B6EFF0E2C6E8EA204D0C10E2D6ED1
:10812800FE0E03D0CF0E2D6EFF0E2E6E8EA004D045
:10813800C10E2F6EFE0E03D0C50E2F6EFF0E306ED1
:1081480090AE04D0C10E316EFE0E03D0F90E316E22
:10815800FF0E326E90AC04D0C10E336EFE0E03D00B
:10816800F60E336EFF0E346E90AA04D0C10E356E33
:10817800FE0E03D0F30E356EFF0E366E90A804D0B7
:10818800C10E376EFE0E03D0F00E376EFF0E386E3E
:1081980090A604D0C10E396EFE0E03D0ED0E396ED6
:1081A800FF0E3A6E90A404D0C10E3B6EFE0E03D0B3
:1081B800EA0E3B6EFF0E3C6E90A204D0C10E3D6EDF
:1081C800FE0E03D0E70E3D6EFF0E3E6E90A004D06B
:1081D800C10E3F6EFE0E03D0E40E3F6EFF0E406EE2
:1081E800820E00019C6FF90E9D6F901C9E6F9F6B15
:1081F8008ECFA0F0A16B3FC0A2F040C0A3F03DC05D
:10820800A4F03EC0A5F03BC0A6F03CC0A7F039C022
:10821800A8F03AC0A9F037C0AAF038C0ABF035C012
:10822800ACF036C0ADF033C0AEF034C0AFF031C002
:10823800B0F032C0B1F02FC0B2F030C0B3F02DC0F2
:10824800B4F02EC0B5F02BC0B6F02CC0B7F029C0E2
:10825800B8F02AC0B9F027C0BAF028C0BBF025C0D2
:10826800BCF026C0BDF023C0BEF024C0BFF021C0C2
:10827800C0F022C0C1F070EF63F0070E0E241D6E2F
:10828800000E0F201E6E0EC0D9FF0FC0DAFFDF50A0
:10829800126E12380F0B0A0DF3CF13F0F4CF14F04F
:1082A8000EC0D9FF0FC0DAFFDF500F0B1326000EE8
:1082B800142213281B6E000E14201C6E206A010E57
:1082C8001F6E216A226A236A246AB2D01F502010C6
:1082D80054E021C012F022C013F023C014F024C0CF
:1082E80015F00A0E1202F3CF16F0F4CF17F0186A41
:1082F800196A1302F3501726F4501822000E192297
:108308001202F3501726F4501822000E19220A0EF2
:108318001402F3501826F4501922000E1302F350D9
:108328001826F4501922000E1202F3501826F450A1
:1083380019220A0E1502F3501926000E1402F350E2
:108348001926000E1302F3501926000E1202F350DC
:1083580019261DC0D9FF1EC0DAFFDF501A6E1A3861
:108368000F0B1624216E000E1720226E000E182007
:10837800236E000E1920246E54D021C012F022C0A2
:1083880013F023C014F024C015F00A0E1202F3CF24
:1083980016F0F4CF17F0186A196A1302F35017266B
:1083A800F4501822000E19221202F3501726F45026
:1083B8001822000E19220A0E1402F3501826F4503F
:1083C8001922000E1302F3501826F4501922000E39
:1083D8001202F3501826F45019220A0E1502F3500F
:1083E8001926000E1402F3501926000E1302F3503A
:1083F8001926000E1202F35019261DC0D9FF1EC0FF
:10840800DAFFDF500F0B1624216E000E1720226EA4
:10841800000E1820236E000E1920246E1D06D8A009
:108428001E061F502010010ED8A4000E1F6E206AD1
:108438001B06D8A01C061B2802E11C28D8A446D776
:1084480021C00EF022C00FF023C010F024C011F09C
:10845800120046C027F047C028F03BEC46F0486EB3
:10846800485001E0D4D046C0D9FF47C0DAFF030E18
:10847800DE1801E0BCD020EE04F04650D926475063
:10848800DA22DE0401E0B3D02F0E46240E6E000E71
:1084980047200F6E116A106A020E136E126AF2EC10
:1084A80062F02D0E46240E6E020E47200F6EAA0EA5
:1084B800116E550E106EB8EC62F02F0E46240E6E3B
:1084C800000E47200F6E520E106E116E610E126E66
:1084D800410E136EA7EC5CF0130E46240E6E020ECE
:1084E80047200F6E720E106E116E410E126E610EE5
:1084F800136EA7EC5CF0170E46240E6E020E472092
:108508000F6E20EE0FF04650D9264750DA22DECF04
:1085180010F0DECF11F0DECF12F0DECF13F0A7ECB3
:108528005CF01B0E46240E6E020E47200F6E20EEE6
:108538000BF04650D9264750DA22DECF10F0DECFB6
:1085480011F0DECF12F0DECF13F0A7EC5CF020EED6
:108558001BF04650D9264750DA22DECF60F0DECF36
:1085680061F0DECF62F0DECF63F0010E000160251E
:10857800646F000E6121656F000E6221666F000E48
:108588006321676F20EE2BF04650D9264750DA2238
:1085980064C0DEFF65C0DEFF66C0DEFF67C0DEFFC9
:1085A8002F0E46241D6E000E47201E6E20EE2BF067
:1085B8004650D9264750DA22DECF1FF0DECF20F012
:1085C800DECF21F0DECF22F0246A010E236E20EEEA
:1085D80001F04650D9264750DA22DF5068EC52F0B5
:1085E80020EE04F04650D9264750DA22DF6A1D6A89
:1085F8001E6A1F6A20EE01F04650D9264750DA223B
:10860800DF5089EC21F0000902E0010E486E485065
:1086180012005E51D8B41200500E00019C6FFD0E7E
:108628009D6F70EC63F082EC56F021C079F122C0A6
:108638007AF123C07BF124C07CF1010179517A11D0
:108648007B117C1117E12E0E00019C6FFC0E9D6FB3
:1086580079C19EF07AC19FF07BC1A0F07CC1A1F0E6
:1086680070EC63F00A0E116E000E126A136A146A37
:108678001FEC5EF001017D6B7E6BE00E00019C6FCC
:10868800FF0E9D6F790E01017D25D96E010E7E21A9
:10869800DA6EDF5000019E6F9F6B70EC63F0010192
:1086A8007D4B7E2B7EBFE9D77E5103E1040E7D5DB5
:1086B800E4E3FC0E00019C6FF90E9D6F70EC63F013
:1086C8000C0E9C6FFB0E9D6F70EC63F023EE00F0B8
:1086D80000EEC7F0210EDBCFEBFFE806FCE2D80E78
:1086E800E96FFF0EEA6F22EC38F0C7C038F1C8C056
:1086F80039F1C9C03AF1CAC03BF101013851391109
:108708003A113B11D8B41200F20E00019C6FFA0E18
:108718009D6F38C19EF039C19FF03AC1A0F03BC1AE
:10872800A1F070EC63F0000E9E6F030E9F6F38C1CE
:10873800F8F039C1F9F03AC1FAF0F76B000EF725F5
:10874800A06F010EF821A16F000EF921A26F000E93
:10875800FA21A36F75EC12F00101646F000E00019D
:10876800746F030E756F350E766F0B0E776F796B1E
:10877800080E786F770E7A6F010E7B6FA3EC1AF0F4
:108788000101646F7F6B806BD70E00019C6FFC0E3C
:108798009D6F350E01017F25D96E0B0E8021DA6E93
:1087A800DF5000019E6F9F6B70EC63F001017F4BFF
:1087B800802B80BFE9D7805105E1080E7F5DD8B0D6
:1087C8001200E2D71200C0C0D9FFC1C0DAFFDECF65
:1087D800CAF0DDCFCBF003D00001C24BC32BC2C01F
:1087E800F6FFC3C0F7FF000EF86E0E0EF76403D055
:1087F8000800F55005D0F6CFE9FFF7CFEAFFEF50B4
:108808002F0AEAE0C2C0F6FFC3C0F7FF000EF86EF9
:108818000E0EF76403D00800F55005D0F6CFE9FF37
:10882800F7CFEAFFEF505C0AD7E0000120EE06F030
:10883800C051D926C151DA22DE6ADE6ADE6ADD6AF3
:10884800C2C0F6FFC3C0F7FF000EF86E0E0EF76445
:1088580003D00800F55005D0F6CFE9FFF7CFEAFFBF
:10886800EF500001C46F200EC46114D020EE27F031
:10887800C051D926C151DA22800EDF6EC0C074F013
:10888800C1C075F0000E766F776F786F796F56EC10
:1088980035F023D0C0C016F0C1C017F0C20E186E54
:1088A80052EC39F00001CD6FCD5158E1C0C0B8F09D
:1088B800C1C0B9F03CEC4BF0CD6F20EE27F0C051B1
:1088C800D926C151DA22DF50CC6FCD5108E0040E11
:1088D800CD1944E1CCB542D0050ECD6F3FD0CCB513
:1088E8003DD020EE04F0C051D926C151DA22DFA8CC
:1088F800F3D7CAC015F0CBC016F0C469010EC56F16
:1089080020EE0EF0C051D926C151DA22DECFC6F0D2
:10891800DDCFC7F0C451C617C551C717CAC0C8F0C4
:10892800CBC0C9F0C651C827C751C9232F0EC825C7
:10893800176E000EC921186E57EC5BF0000120EE8F
:1089480006F0C051D926C151DA2215C0DEFF16C083
:10895800DEFF17C0DEFF18C0DEFF9CD7CD51120026
:1089680081C0D9FF82C0DAFFDECF98F0DDCF99F061
:1089780086518511841104E1020E835DD8A0020C92
:1089880020EE13F09851D9269951DA22DE50835DF2
:10899800DE508459DE508559DE50865901E3020CB9
:1089A8008751881189118A1117E098C060F099C021
:1089B80061F087C062F088C063F089C064F08AC043
:1089C80065F066696769686969696CEC1FF0976F9B
:1089D800975102E09751120081C045F082C046F0DD
:1089E80083C047F084C048F085C049F086C04AF08B
:1089F80059EC2DF045C093F046C094F047C095F06F
:108A080048C096F00001935194119511961170E0A9
:108A1800930594119511961101E1020C932907E130
:108A2800942905E1952903E1962901E1010C98C0F3
:108A380060F099C061F083C062F084C063F085C0C3
:108A480064F086C065F0666B676B686B696B6CEC8D
:108A58001FF0976F9751BEE120EE13F09851D92679
:108A68009951DA22FE0EDE248B6FFF0EDE208C6F0A
:108A7800FF0EDE208D6FFF0EDE208E6F20EE0FF0D2
:108A88009851D9269951DA228B51DE5C8C51DE58E7
:108A98008D51DE588E51DE5813E220EE0FF09851BA
:108AA800D9269951DA22DE2A000EDE22DE22DE22C3
:108AB80020EE04F09851D9269951DA22000EDB8075
:108AC80093C083F094C084F095C085F096C086F07A
:108AD80020EE13F09851D9269951DA22DE50835DA1
:108AE800DE508459DE508559DE50865901E274D72C
:108AF800000C1E6E1E5001E0010C55A202D055500C
:108B08001200000EA4EC62F00A0E296E03D094EC59
:108B180063F029062950FBE1266A000E176A186AD5
:108B2800196A1A6A0AEC61F0E80601E097D0AA0E01
:108B3800176E010E186E196A1A6A080E0AEC61F0AF
:108B4800E80651E1296A29501F0FD96EDA6A94ECB8
:108B580063F0DF6E292A030E2964F5D721047EE12C
:108B6800AA0E22187BE1030E286EE80E276E15D098
:108B7800176A186A196A400E1A6EA90E0AEC61F093
:108B880000090EE0150E1D6EC60EE82EFED71D2E2E
:108B9800FCD700D02706D8A0280627502810E8E1DF
:108BA800275028105BE0176A186A196A1A6A3A0E81
:108BB8000AEC61F0000952E1296A29501F0FD96EA9
:108BC800DA6A94EC63F0DF6E292A030E2964F5D77C
:108BD8001FBC03D0246A040E02D0246A0C0E236E34
:108BE80023C026F03BD0176A186A196A1A6AA90EB8
:108BF8000AEC61F01D6E020E1D6003D0266EA90EF0
:108C080002D0010E266E256E030E286EE80E276E22
:108C180014D0176A186A196A1A6A25500AEC61F0A2
:108C280000090EE0150E1D6EC60EE82EFED71D2E8D
:108C3800FCD700D02706D8A0280627502810E9E13D
:108C4800275028100AE0176A020E186E196A1A6A65
:108C5800100E0AEC61F0000901E0266A26C053F004
:108C6800A5EC63F0265001E14AD7559048D7396AF8
:108C780020EE03F02750D9262850DA22DF5001E1F0
:108C8800A7D02F0E27241D6E000E28201E6E20EE62
:108C98002BF02750D9262850DA22DECF1FF0DECF5E
:108CA80020F0DECF21F0DECF22F0246A010E236E01
:108CB80020EE01F02750D9262850DA22DF5068EC40
:108CC80052F0000901E082D020EE03F02750D926A7
:108CD8002850DA22DF6A20EE17F02750D9262850CC
:108CE800DA2210EE1FF02750E1262850E222E6CFC4
:108CF8002DF0E6CF2EF0E6CF2FF0E6CF30F010EED5
:108D08002BF02750E1262850E222E6CF31F0E6CFBB
:108D180032F0E6CF33F0E6CF34F02D50315C356ECB
:108D28002E503258366E2F503358376E30503458D4
:108D3800386EDE50355CDE503658DE503758DE501F
:108D4800385846E220EE02F02750D9262850DA2279
:108D5800020EDE183DE12F0E27241D6E000E28207E
:108D68001E6E20EE17F02750D9262850DA22DECFC3
:108D780029F0DECF2AF0DECF2BF0DECF2CF020EE6C
:108D88002BF02750D9262850DA22DECF2DF0DECF5F
:108D98002EF0DECF2FF0DECF30F029502D241F6EBD
:108DA8002A502E20206E2B502F20216E2C50302040
:108DB800226E246A010E236E20EE01F02750D92678
:108DC8002850DA22DF5068EC52F002D0010E396EDA
:108DD8003950120049C00FF04AC010F0690E116EE8
:108DE80086EC55F00001686F685101E099D020EEDB
:108DF8000EF04950D9264A50DA22DFAC91D069C02A
:108E08003AF06AC03BF020EE1CF04950D9264A508F
:108E1800DA22DECF3CF0DECF3DF0DECF3EF0DECF13
:108E28003FF0D1EC56F00001686F685179E120EE0F
:108E380020F04950D9264A50DA22DECF6BF0DDCF38
:108E48006CF020EE0BF06B51D9266C51DA22000E33
:108E5800DB8A49C0D9FF4AC0DAFFDECF12F0DDCF86
:108E680013F06BC014F06CC015F020EE06F04950FA
:108E7800D9264A50DA22DECF16F0DECF17F0DECF41
:108E880018F0DECF19F01EEC60F01C0E00016B2507
:108E98000E6E000E6C210F6E20EE0AF04950D92696
:108EA8004A50DA22DECF10F0DECF11F0DECF12F01A
:108EB800DECF13F0A7EC5CF0160E00016B250E6EEA
:108EC800000E6C210F6E106A116A210E126E500E80
:108ED800136EA7EC5CF0120E00016B250E6E000EEF
:108EE8006C210F6E000E116A106AB8EC62F0000176
:108EF80020EE03F06951D9266A51DA22010EDF6E9D
:108F080069C046F06AC047F02DEC42F00001686F76
:108F180020EE0EF04950D9264A50DA22BF0EDF164D
:108F28006851120089688B68F29E8E280BE1590EF1
:108F380000019C6FFB0E9D6F8ECF9EF09F6B70ECB7
:108F480063F00AD04A0E00019C6FFA0E9D6F8ECF17
:108F58009EF09F6B70EC63F090280AE1170E9C6FEF
:108F6800FC0E9D6F8ECF9EF09F6B70EC63F009D066
:108F78006F0E9C6FFA0E9D6F8ECF9EF09F6B70ECFC
:108F880063F0290E426E960E416E7F0EE82EFED7D4
:108F9800412EFCD7422EFAD700F0780E00019C6FC4
:108FA800FE0E9D6F70EC63F089988498090E426EEE
:108FB8001E0E416EE40EE82EFED7412EFCD7422E3F
:108FC800FAD700D06B0E00019C6FFE0E9D6F70ECFF
:108FD80063F0899A849A090E426E1E0E416EE40E61
:108FE800E82EFED7412EFCD7422EFAD700D0DC0E51
:108FF80000019C6FFE0E9D6F70EC63F088908D9061
:1090080090280AE0170E9C6FFC0E9D6F90CF9EF083
:109018009F6B70EC63F009D0FF0E9C6FF90E9D6F8B
:1090280090CF9EF09F6B70EC63F08D80A30E426E24
:10903800570E416E020EE82EFED7412EFCD7422E67
:10904800FAD700D089688B688A6883928382290E50
:10905800426E960E416E7F0EE82EFED7412EFCD74B
:10906800422EFAD700F054EC40F0EFD71F6A1DAE3D
:1090780012D01D1E1C1E1B1E1A1E191E181E171E7E
:10908800166C000E1722182219221A221B221C22E3
:109098001D22010E1F6E15AE12D0151E141E131EB2
:1090A800121E111E101E0F1E0E6C000E0F22102213
:1090B80011221222132214221522010E1F1A206ACD
:1090C800216A226A236A246A256A266A276A165050
:1090D8001710181019101A101B101C101D1045E03D
:1090E800010E1E6E0AD0D890163617361836193665
:1090F8001A361B361C361D361E2A1DAEF4D7D890DC
:10910800203621362236233624362536263627368B
:1091180016500E5C17500F58185010581950115807
:109128001A5012581B5013581C5014581D501558DB
:1091380011E316500E5E17500F5A1850105A195056
:10914800115A1A50125A1B50135A1C50145A1D50B7
:10915800155A2080D8901D321C321B321A3219320F
:109168001832173216321E2ECAD71F5010E0271E8B
:10917800261E251E241E231E221E211E206C000EC4
:10918800212222222322242225222622272220C00D
:109198000EF021C00FF022C010F023C011F024C03F
:1091A80012F025C013F026C014F027C015F01200E5
:1091B800176818680E50D96EDA6ADECF19F0DDCF5D
:1091C8001AF019C014F01AC015F019501A1003E15A
:1091D8000E680F68120014C0F6FF15C0F7FF000EE6
:1091E800F86E0E0EF76403D00800F55005D0F6CFE0
:1091F800E9FFF7CFEAFFEF50166E144A152A200E42
:10920800166403D03A0E1618E6E13A0E161868E10D
:10921800000E136E010E126E19C0F6FF1AC0F7FF8A
:10922800000EF86E0E0EF76403D00800F55005D056
:10923800F6CFE9FFF7CFEAFFEF50106E2F0E10645C
:1092480039D019C0F6FF1AC0F7FF000EF86E0E0EDF
:10925800F76403D00800F55005D0F6CFE9FFF7CF43
:10926800EAFFEF50106E3A0E106024D0020E192457
:10927800106E000E1A20116E145010181BE11550B4
:10928800111818E119C0F6FF1AC0F7FF000EF86EA2
:109298000E0EF76403D00800F55005D0F6CFE9FFAD
:1092A800F7CFEAFFEF50106ED00E1024126E136A3B
:1092B800FF0E132213BE04D013500DE112040BE26B
:1092C80012C017F013C018F00E50D96EDA6A14C025
:1092D800DEFF15C0DDFF17C00EF018C00FF012003A
:1092E8000E6A0F6A120060C045F061C046F0476A16
:1092F800486A496A4A6A8AEC50F045C078F046C024
:1093080079F0020E0001781979110DE0795106E122
:10931800030E785D03E26251631105E178C060F0E5
:1093280079C061F012007A6B7B6B7AC064F07BC005
:1093380065F0643B653BF00E651764510F0B6513D0
:10934800F00E641760C066F061C067F0645166276C
:1093580065516723F50E66250E6E010E67210F6EA7
:10936800DCEC55F000017A51040DF350680FD96E0A
:10937800DA6A0EC0DEFF0FC0DEFF10C0DEFF11C0CC
:10938800DEFF7A4B7B2B7B5103E1040E7A5DCDE344
:109398006251631103E17A6B7B6B06D0FF0E622585
:1093A8007A6FFF0E63217B6F7A51040DF350680FBB
:1093B800D96EDA6ADE50DE10DE10DE1004E1796B59
:1093C800030E786F18D060C045F061C046F07A513E
:1093D800040DF350680FD96EDA6ADECF47F0DECF9E
:1093E80048F0DECF49F0DECF4AF08AEC50F045C0B5
:1093F80078F046C079F00001625163118FE179512C
:1094080003E1020E785D8AE37A4B7B2B7B5186E180
:10941800040E7A5D83E2C8D72F6C69666461746153
:10942800302E62696E20002F6C6966646174613148
:109438002E62696E20002F6C696664617461322E39
:1094480062696E20002F6C696664617461332E62F4
:10945800696E20002F6C696664617461342E6269DC
:109468006E20002F6C696664617461352E62696EC6
:1094780020002F6C696664617461362E62696E2003
:10948800002F6C696664617461372E62696E200012
:109498002F6C696664617461382E62696E20002FD2
:1094A8006C696664617461392E62696E20002F6C84
:1094B800696664617461612E62696E20002F6C694F
:1094C8006664617461622E62696E20002F6C696641
:1094D80064617461632E62696E20002F6C69666432
:1094E800617461642E62696E20002F6C6966646124
:1094F8007461652E62696E20002F6C696664617400
:1095080061662E62696E2000000000000000000005
:109518000000000000000000000000000000000043
:109528000000000000000000000000000000000033
:109538000000000000000000000000000000000023
:10954800000000000EC018F00FC019F012501310E0
:1095580001E1120018C0D9FF19C0DAFF10C0DFFFFF
:1095680012501824146E13501920156EFF0E14246F
:10957800D96EFF0E1520DA6E10C0DFFF135004E11C
:10958800030E125C01E2120020EE01F01850D926F9
:109598001950DA2210C0DFFF20EE02F01850D92649
:1095A8001950DA2210C0DFFF12501824146E13501D
:1095B8001920156EFE0E1424D96EFF0E1520DA6ED2
:1095C80010C0DFFF12501824146E13501920156EA6
:1095D800FD0E1424D96EFF0E1520DA6E10C0DFFFC1
:1095E800135004E1070E125C01E2120020EE03F0B2
:1095F8001850D9261950DA2210C0DFFF125018244B
:10960800146E13501920156EFC0E1424D96EFF0E1B
:109618001520DA6E10C0DFFF135004E1090E125C4A
:1096280001E2120018C014F019C015F0141E151E1E
:10963800144A152A030E1414166E176A16501826A3
:10964800175019221650125E1750135AFC0E121694
:109658000BD018C0D9FF19C0DAFF10C0DFFF1206FF
:10966800D8A01306184A192A12501310F2E1120052
:10967800B8C0D9FFB9C0DAFFDECFBCF0DDCFBDF08E
:10968800B8C074F0B9C075F0000E766F776F786F58
:10969800796F56EC35F0BF6FBF5103E00001BF5141
:1096A8001200BCC03AF0BDC03BF020EE16F0B85135
:1096B800D926B951DA22DECF3CF0DECF3DF0DECF3D
:1096C8003EF0DECF3FF0D1EC56F00001BF6FBF5146
:1096D800E5E120EE1AF0B851D926B951DA22DECFE9
:1096E800BAF0DDCFBBF0BAC0D9FFBBC0DAFFDF509C
:1096F800BE6FBE5103E1040EBF6FD0D720EE04F059
:10970800B851D926B951DA2210EE1AF0B851E1262B
:10971800B951E22200EE0BF0E650E926E550EA22C4
:10972800EF503F0BDF6E20EE1AF0B851D926B95131
:10973800DA2210EE0BF0DE50E126DD50E222E7B629
:1097480018D020EE1AF0B851D926B951DA22DECF56
:109758000EF0DDCF0FF01C0EB825106E000EB921EB
:10976800116E136A0B0E126E71EC5CF00E500F1036
:1097780095E0B8C09EF0B9C09FF00001A16BA06B46
:10978800BAEC30F00001BF6FBF5188E18AD71BC027
:109798000EF01CC00FF0116A106A136A080E126EE0
:1097A800A6EC4AF0266A020E256E25501B24D96EB7
:1097B80026501C20DA6E25501B24216E26501C20B2
:1097C800226E2128E16E000E2220E26EE750236E01
:1097D800233AF00E2316231625501B24E16E26503B
:1097E8001C20E26EE750246E24380F0B2310DF6E26
:1097F800254A262A26BED9D7265003E1070E255C1E
:10980800D4E325501B24D96E26501C20DA6E1DC0C7
:109818000EF01EC00FF01FC010F020C011F00A0E8D
:10982800126E136A146A156A10EC5DF00E3AF00EA7
:109838000E1625501B24E16E26501C20E26EE750C0
:10984800216E21380F0B0E10DF6E1BC0D9FF1CC014
:10985800DAFFDF2A1DC00EF01EC00FF01FC010F087
:1098680020C011F00A0E126E136A146A156AE2EC2F
:109878005AF00EC01DF00FC01EF010C01FF011C02E
:1098880020F01D501E101F1020108CE11BC0D9FFA6
:109898001CC0DAFFDF06090EDF64090C1BC0D9FF04
:1098A8001CC0DAFF100EDF6E100C000E0101AB6F4A
:1098B8000A0EAA6F000EA96F050EA86F7DD00101D0
:1098C800AB6B140EAA6F70D06E0E0F6EFC0E106E7E
:1098D800F5EC5DF08FB204D00101AB6B1E0EAA6FE0
:1098E800090E0001FE6F1E0EFD6FE40EE82EFED776
:1098F800FD2FFCD7FE2FFAD700F056D0C40E0F6EFE
:10990800FE0E106EF5EC5DF0060E0001B16F090E4B
:10991800B26FFE0EB36FF90EB46FB56B49EC58F029
:109928000101646F645171EC5EF001016451D8E18A
:10993800AB6B230ED4D7090E0F6EFE0E106EF5EC2E
:109948005DF0000E0001CE6F030ECF6FDE0ED06FFC
:10995800010ED16F010ED26F43EC15F00101646F57
:10996800645171EC5EF0010164510AE1B5EC29F033
:10997800000E6D6F030E6E6F7BEC60F00101646F7B
:10998800645171EC5EF0010CAAC1FDF0ABC1FEF0B0
:109998000001FE5109E1FD510A0A91E01E0A94E016
:1099A8000A0AACE03D0AC7E0140E0101AA19AB117E
:1099B80003E0A807D8A0A907A9BF000CA951E4E1B2
:1099C800A805E2E2000C1F6A15AE12D0151E141E7F
:1099D800131E121E111E101E0F1E0E6C000E0F22DB
:1099E800102211221222132214221522010E1F6E98
:1099F8001DAE10D01D1E1C1E1B1E1A1E191E181E61
:109A0800171E166C000E1722182219221A221B2262
:109A18001C221D2216501710181019101A101B108E
:109A28001C101D103BE0010E1E6E0AD0D890163691
:109A38001736183619361A361B361C361D361E2AA6
:109A48001DAEF4D716500E5C17500F58185010580A
:109A5800195011581A5012581B5013581C501458AA
:109A68001D50155810E316500E5E17500F5A185017
:109A7800105A1950115A1A50125A1B50135A1C5086
:109A8800145A1D50155AD8901D321C321B321A32E6
:109A980019321832173216321E2ED4D71F5010E042
:109AA800151E141E131E121E111E101E0F1E0E6CE4
:109AB800000E0F2210221122122213221422152224
:109AC8000EC00EF00FC00FF010C010F011C011F052
:109AD80012C012F013C013F014C014F015C015F022
:109AE8001200020E105E000E115A125A135A20EE7E
:109AF80013F00E50D9260F50DA22FE0EDE24146E13
:109B0800FF0EDE20156EFF0EDE20166EFF0EDE2025
:109B1800176E1450105C15501158165012581750E3
:109B2800135805E30E6A0F6A106A116A120020EED4
:109B380027F00E50D9260F50DA22DECF14F0DECFF0
:109B480015F0DECF16F0DECF17F020EE09F00E503C
:109B5800D9260F50DA22DECF18F0DDCF19F01850D1
:109B68001A6E19501B6E1C6A1D6A1A501002F3CF28
:109B78001EF0F4CF1FF0206A216A1102F3501F264D
:109B8800F4502022000E21221B501002F3501F26F1
:109B9800F4502022000E21221A501202F3502026DF
:109BA800F45021221B501102F3502026F450212298
:109BB8001C501002F3502026F450212213501A0290
:109BC800F35021261B501202F35021261C5011027B
:109BD800F35021261D501002F350212614501E2444
:109BE8000E6E15501F200F6E16502020106E175045
:109BF8002120116E1200838E83800001FB6BFC6BA9
:109C08002DEC5AF025C0FDF026C0FEF0040E000130
:109C1800FE5D07E3000EFD25FB6FFC0EFE21FC6FC9
:109C280004D0FDC0FBF0FEC0FCF001015E5133E042
:109C3800385139113A113B112EE052500C0D040ED7
:109C4800F324D96E010EF420DA6E38C16EF139C1F1
:109C58006FF13AC170F16D6B000E6D25716F010ED9
:109C68006E21726F000E6F21736F000E7021746F7A
:109C7800DE50711910E1DE5072190DE1DE507319D2
:109C88000AE1DE50741907E1000E256E040E266EF7
:109C98005E51D8EC58F08FB415D05250220D000EFA
:109CA800F32400019E6F030EF4209F6F000EA06F37
:109CB800040EA16F010EA36FA26BFB0EA46F1AEC2A
:109CC8000CF0FA6F0001FA5109E0400E9C6FFD0E8E
:109CD8009D6FFAC09EF09F6B70EC63F0BAEC27F0B2
:109CE800596B8390839EB90E00019C6FFC0E9D6F8B
:109CF800CECF9EF09F6BCDCFA0F0A16B70EF63F03D
:109D0800F3C123F071D005EC63F0236EF31979E009
:109D1800290E226E960E216E7F0EE82EFED7212E7A
:109D2800FCD7222EFAD700F06CD010EC5FF0246E2E
:109D3800245067E024B0542A24B254060F0E541657
:109D4800000E0E6EC00EC2EC5EF08FEC62F0000EDC
:109D58000E6EC00EC2EC5EF054500F0D350EF3249B
:109D6800126E0D0EF420136E6AEC5AF0110E226E6C
:109D78003C0E216ECB0EE82EFED7212EFCD7222ECC
:109D8800FAD700F024A43DD00F6A0E6A54C010F030
:109D9800B5EC60F05A0E00019C6FFC0E9D6F54C02C
:109DA8009EF09F6B70EC63F054C023F0000E0E6EB3
:109DB800800EC2EC5EF08FEC62F0000E0E6E800E2C
:109DC800C2EC5EF054500F0D350EF324126E0D0EDA
:109DD800F420136E6AEC5AF0000E0E6EC00EC2EC40
:109DE8005EF08FEC62F00DD001016051216E226AA5
:109DF800225007E12150010A86E0030A84E0010AA3
:109E080094E0235012003AC027F03BC028F03BEC06
:109E180046F0000901E0010C3AC00EF03BC00FF01B
:109E28003CC010F03DC011F03EC012F03FC013F02E
:109E380075EC4DF00EC044F00FC045F010C046F070
:109E480011C047F020EE2BF03A50D9263B50DA22C9
:109E580044C0DEFF45C0DEFF46C0DEFF47C0DEFF70
:109E68002F0E3A240E6E000E3B200F6E116A106AF8
:109E7800020E136E126AF2EC62F02F0E3A24426E52
:109E8800000E3B20436E496A010E486E4A6A4B6ACF
:109E980004D048504A2649504B2220EE09F03A5047
:109EA800D9263B50DA22DE504A5CDE504B581FE27E
:109EB80042C01DF043C01EF04A5044241F6E4B5050
:109EC8004520206E000E4620216E000E4720226E8F
:109ED80048C023F049C024F020EE01F03A50D926BA
:109EE8003B50DA22DF5068EC52F00009D2E020EE55
:109EF80009F03A50D9263B50DA224A50DE1803E1DD
:109F08004B50DE18D8A4010C000C226A236A1B6A85
:109F18001C6A01D0152A010E216E1550D96EDA6A15
:109F2800200EDE1813E0F70E176E18681550D96E5C
:109F3800DA6ADF50196E1A6A1750192618501A2251
:109F48001A5003E1050E195C01E3216A21C01DF0D6
:109F58001E6A1D501E1006E0DDD71C6A010E1B6E1E
:109F6800152A25D01550D96EDA6ADF50176E186A8F
:109F780018501DE117502B0AF3E0060AEEE017D03F
:109F88000A0E2202F3CF17F0F4CF18F02302F35091
:109F980018261550D96EDA6ADF50175E000E185A67
:109FA800300E1724226E000E1820236ED9D7D00E3B
:109FB800176E18681550D96EDA6ADF50196E1A6A6A
:109FC8001750192618501A221A5005E10A0E195C62
:109FD80002E2010E01D0000E1F6E206A1F502010F1
:109FE800CFE11B501C100DE122C017F023C018F060
:109FF800171E181E174A182A17C015F018C016F091
:10A00800120022C015F023C016F01200818E819C28
:10A01800200EF66E940EF76E000EF86E0DEE35F00B
:10A0280011EE2CF00900F5CFEEFFE550E150FAE112
:10A03800E250F8E1D40EF66EBD0EF76E000EF86E23
:10A0480003EEAAF010EE4CF00900F5CFEEFFE55054
:10A05800E150FAE1EE0EF66EC20EF76E000EF86EE3
:10A0680002EE90F010EE34F00900F5CFEEFFE55067
:10A07800E150FAE1160EF66EC40EF76E000EF86E99
:10A0880001EEC6F010EE2DF00900F5CFEEFFE55019
:10A09800E150FAE16E0EF66EC70EF76E000EF86E1E
:10A0A8000900F5CF55F005EE00F018EE35F0EE6A30
:10A0B800E550E150FCE1E250FAE104EE00F011EE67
:10A0C80000F0EE6AE550E150FCE1E250FAE103EEFF
:10A0D80000F0AA0EEE6AE806FDE102EE00F0900E2E
:10A0E800EE6AE806FDE101EE00F0690EEE6AE806A8
:10A0F800FDE100EE4CF0090EEE6AE806FDE156902F
:10A108005692000EF86E000159EF0FF020EE03F0A2
:10A118004550D9264650DA22DF6A20EE2BF045500A
:10A12800D9264650DA22DE68DE68DE68DD6845C07A
:10A138003AF046C03BF047C03CF048C03DF049C04B
:10A148003EF04AC03FF0D1EC56F0000904E0466A00
:10A15800040E456E040C2D0E45240E6E020E46208C
:10A168000F6E91EC61F0550E0E1803E1AA0E0F1850
:10A1780004E0466A030E456E030C20EE2FF04550AE
:10A18800D9264650DA22E90EDE1812E020EE2FF02A
:10A198004550D9264650DA22EB0EDE1809E020EEAB
:10A1A8002FF04550D9264650DA22E80EDE1827E16E
:10A1B800650E45240E6E000E46200F6ED40E106EEE
:10A1C800FF0E116E136A030E126E71EC5CF00E50E6
:10A1D8000F1003E1456A466A1200810E45240E6E8F
:10A1E800000E46200F6E8E0E106EFF0E116E136A53
:10A1F800050E126E71EC5CF00E500F10EBE0466A23
:10A20800020E456E020C2F6E950E00019C6FFC0E1F
:10A218009D6F2FC09EF09F6B2BC0A0F02CC0A1F0AB
:10A2280070EC63F05DD082EC56F021C030F022C0B3
:10A2380031F023C032F024C033F02BC0D9FF2CC03A
:10A24800DAFFDF6A20EE01F02B50D9262C50DA22F3
:10A2580033C0DFFF20EE02F02B50D9262C50DA2233
:10A26800DF6A20EE03F02B50D9262C50DA2232C0B8
:10A27800DFFF20EE04F02B50D9262C50DA22DF6ABB
:10A2880020EE05F02B50D9262C50DA2231C0DFFF02
:10A2980020EE06F02B50D9262C50DA22DF6A20EE69
:10A2A80007F02B50D9262C50DA2230C0DFFF1200DD
:10A2B80082EC56F021C030F022C031F023C032F0D9
:10A2C80024C033F02BC01BF02CC01CF030C01DF094
:10A2D80031C01EF032C01FF033C020F0CBEF4BF07E
:10A2E8002F502D6E2E6A2E50D8A412002D50010A20
:10A2F8009AE0030ADDE012000001FC6B8380838E84
:10A308006AD02DEC5AF025C0FAF026C0FBF0040EF6
:10A318000001FB5D03E3010EFC6F03D0FFC0FDF0FD
:10A32800FE6B8FB414D05250220D000EF3249E6F92
:10A33800030EF4209F6F000EA06F040EA16F010E94
:10A34800A36FA26BFD0EA46F1AEC0CF0FF6FFF5108
:10A3580009E0400E9C6FFD0E9D6FFFC09EF09F6B45
:10A3680070EC63F001015E5133E0385139113A1154
:10A378003B112EE052500C0D040EF324D96E010E41
:10A38800F420DA6E38C16EF139C16FF13AC170F15B
:10A398006D6B000E6D25716F010E6E21726F000ED0
:10A3A8006F21736F000E7021746FDE50711910E108
:10A3B800DE5072190DE1DE5073190AE1DE5074198E
:10A3C80007E1000E256E040E266E5E51D8EC58F09B
:10A3D800BAEC27F0596B0001FC5193E0839E8390FF
:10A3E80012000F015969116B196B216B8C948C92B7
:10A3F8008C90889A110E136E3C0E126ECB0EE82EBE
:10A40800FED7122EFCD7132EFAD700F0110E136EBA
:10A418003C0E126ECB0EE82EFED7122EFCD7132E52
:10A42800FAD700F0020E136EA00E126E920EE82EEE
:10A43800FED7122EFCD7132EFAD700D0000E0E6EC0
:10A44800300EC2EC5EF02A0E126E8E0EE82EFED78B
:10A45800122EFCD7000E0E6E300EC2EC5EF0000E0F
:10A468000E6E300EC2EC5EF0000E0E6E390EC2ECAF
:10A478005EF0000E0E6E140EC2EC5EF0000E0E6E54
:10A48800560EC2EC5EF0000E0E6E6D0EC2EC5EF063
:10A49800000E0E6E700EC2EC5EF0000E0E6E0C0E0C
:10A4A800C2EC5EF0000E0E6E060EC2EC5EF0000E00
:10A4B8000E6E010EC2EC5EF0D00E126ECA0EE82EC1
:10A4C800FED7122EFCD71200266E2650D8A4040CF4
:10A4D8002350241001E1040C55B0030C55B4020CB0
:10A4E80053B608D0090ED8901F36203621362236AA
:10A4F800E82EF9D7230424101AE11FC017F020C052
:10A5080018F021C019F022C01AF0180E0AEC61F0F8
:10A51800000945E11DC010F01EC011F0FE0E126EBC
:10A52800CBEC5DF000093BE0236A246A38D053C0C5
:10A5380025F0060E251609E023C017F024C018F0F0
:10A54800196A1A6A970E0AEC61F01FC017F020C04A
:10A5580018F021C019F022C01AF0190E0AEC61F0A7
:10A5680000091DE11DC010F01EC011F0FC0E126E96
:10A57800CBEC5DF0000908E0020E1E262306D8A0E9
:10A58800240623502410EEE1106A116AFD0E126EA3
:10A59800CBEC5DF0000903E1246A010E236EA5EC03
:10A5A80063F023502410D8A4010C000CB8C0D9FFC4
:10A5B800B9C0DAFFDECFBFF0DDCFC0F0B8C074F0AD
:10A5C800B9C075F0000E766F776F786F796F56ECBB
:10A5D80035F0C36FC35153E1C16BC26BBFC03AF0D2
:10A5E800C0C03BF020EE16F0B851D926B951DA2296
:10A5F800DECF3CF0DECF3DF0DECF3EF0DECF3FF0E9
:10A60800D1EC56F00001C36FC35139E120EE1AF0C6
:10A61800B851D926B951DA22DECFBCF0DDCFBDF072
:10A62800BCC0D9FFBDC0DAFFE50EDE1810E020EE91
:10A638001AF0B851D926B951DA22DECFBCF0DDCFF5
:10A64800BDF0BCC0D9FFBDC0DAFFDF5009E1C14B86
:10A65800C22BBA51C11906E1BB51C21910E002D090
:10A66800C16BC26BB8C09EF0B9C09FF0A16B010E60
:10A67800A06FBAEC30F00001C36FC351AFE0040E15
:10A68800C31902E1070EC36FC3511200838E838082
:10A698000001D16BD26BD36BD46B5250220D000EDC
:10A6A800F324746F030EF420756F350E766F0B0E5E
:10A6B800776F010E796F786BD50E7A6F7B6BA3EC91
:10A6C8001AF0D06F01015E5135E0385139113A1155
:10A6D8003B1130E052500C0D040EF324D96E010EDC
:10A6E800F420DA6E38C1C7F039C1C8F03AC1C9F0F0
:10A6F8000001C66B000EC625CA6F010EC721CB6FBD
:10A70800000EC821CC6F000EC921CD6FDE50CA19CA
:10A7180011E1DE50CB190EE1DE50CC190BE1DE5011
:10A72800CD1908E1350E2B6E0B0E2C6E01015E5112
:10A7380007EC51F002920001D5511DEC5BF00001CD
:10A74800CE6FCF6BCE51D127CF51D223000ED3235A
:10A75800D4230101596B839E8390120052501C0D23
:10A76800070EF324D96E020EF420DA6E000EDE24F2
:10A77800C76F010EDE20C86F000EDE20C96F000E05
:10A78800DE20CA6F000EDE20CB6F000EDE20CC6FFD
:10A79800000EDE20CD6F000EDE20CE6F52501C0D55
:10A7A800070EF324D96E020EF420DA6EC7C0DEFF5E
:10A7B800C8C0DEFFC9C0DEFFCAC0DEFFCBC0DEFFF7
:10A7C800CCC0DEFFCDC0DEFFCEC0DEFF52501C0D78
:10A7D800070EF324D96E020EF420DA6EDECFCFF026
:10A7E800DECFD0F0DECFD1F0DECFD2F05250220D46
:10A7F800000EF3249E6F030EF4209F6FCFC0A0F0CD
:10A80800D0C0A1F0D1C0A2F0D2C0A3F075EC12F074
:10A81800D36FD35103E0010E506E010C506A120041
:10A82800C4C0D9FFC5C0DAFFDECFC6F0DDCFC7F0A0
:10A83800C4C0B8F0C5C0B9F0000EBB6F010EBA6F46
:10A84800DAEC52F0C86FC85147E1C6C03AF0C7C049
:10A858003BF020EE16F0C451D926C551DA22DECFDE
:10A868003CF0DECF3DF0DECF3EF0DECF3FF0D1EC66
:10A8780056F00001C86FC8512FE120EE1AF0C451FC
:10A88800D926C551DA22DECF0EF0DDCF0FF0116ADE
:10A89800106A136A200E126EF2EC62F0000120EECC
:10A8A8001AF0C451D926C551DA22DECF0EF0DDCF19
:10A8B8000FF01C0EC425106E000EC521116E136A10
:10A8C8000B0E126EBDEC5FF020EE03F0C651D926D8
:10A8D800C751DA22010EDF6EC851120052501C0D0A
:10A8E800070EF324D96E020EF420DA6EDECFF0F0F4
:10A8F800DECFF1F0DECFF2F0DECFF3F0DECFF4F012
:10A90800DECFF5F0DECFF6F0DECFF7F0F1C0F0F0F5
:10A91800F2C0F1F0F3C0F2F0F4C0F3F0F5C0F4F0D7
:10A92800F6C0F5F0F7C0F6F00001F76BF0C0F8F0EC
:10A93800F1C0F9F0F2C0FAF0F3C0FBF066EC3FF0BA
:10A94800FE6FFE5102E0FE5112008FB414D0525037
:10A95800220D000EF3249E6F030EF4209F6F000E4D
:10A96800A06F040EA16F010EA36FA26BFC0EA46F63
:10A978001AEC0CF0FF6FFF510BE0400E9C6FFD0EC0
:10A988009D6FFFC09EF09F6B70EC63F0FF5112004B
:10A99800B2EC53F0000C01015A6B4E6A486B496BDC
:10A9A800020E596F8390586B576B526A030E5264AC
:10A9B80001D049D052500C0D030EF324D96E010E6C
:10A9C800F420DA6EDF6A52500C0D020EF324D96EB1
:10A9D800010EF420DA6EDF6A52500C0D000EF324DB
:10A9E800D96E010EF420DA6EDE6ADD6A52500C0D63
:10A9F800040EF324D96E010EF420DA6EDE6ADE6AE4
:10AA0800DE6ADD6A52500C0D0B0EF324D96E010E6E
:10AA1800F420DA6E100EDF6E52500C0D0A0EF3247D
:10AA2800D96E010EF420DA6E020EDF6E52500C0D54
:10AA3800080EF324D96E010EF420DA6E240EDE6EB1
:10AA4800DD6A522AB3D7526A0101566B120083801D
:10AA5800838E000E0E6E040E0F6E116A1068010EC2
:10AA6800136E126AA6EC4AF0270E00019C6FFE0EC8
:10AA78009D6F70EC63F0CB6BCC6BCBC04BF0010ED1
:10AA88004B164B324B3283504B187F0B4B18836E4F
:10AA98002E0E65EC63F08FB415D05250220D000EC7
:10AAA800F32400019E6F030EF4209F6F000EA06F29
:10AAB800040EA16F010EA36FA26BC80EA46F1AEC4F
:10AAC8000CF0CA6F0001CA5109E0720E9C6FFF0EAC
:10AAD8009D6FCAC09EF09F6B70EF63F0CB4BCC2B81
:10AAE800CCBFCBD7CC5103E10A0ECB5DC6E3130E26
:10AAF8009C6FFF0E9D6F70EC63F0839E8390839034
:10AB0800506A1200090E186E0F5010103BE00FC06B
:10AB1800D9FF10C0DAFFDE50DE1034E00FC0D9FFD5
:10AB280010C0DAFFDECF12F0DDCF13F012C0D9FF6C
:10AB380013C0DAFFDF5026E00FC0D9FF10C0DAFFDC
:10AB480010EE05F0DE50E126DD50E22220EE02F0A4
:10AB58000F50D9261050DA22E650DE1813E1E650DD
:10AB6800DE1810E10FC0D9FF10C0DAFF10EE01F0B7
:10AB7800DE50E126DD50E222E7509BEC63F0126ED6
:10AB880012A0186A185003E0166A176A08D00FC096
:10AB9800D9FF10C0DAFFDECF16F0DDCF17F0115065
:10ABA800D96EDA6A16C0DEFF17C0DDFF1850120032
:10ABB80020EE03F00E50D9260F50DA22DF50166E21
:10ABC800176A186A196A20EE02F00E50D9260F503B
:10ABD800DA22DF5016C013F017C014F018C015F0B1
:10ABE800126A1210166E1350176E1450186E155004
:10ABF800196E20EE01F00E50D9260F50DA22DF50E0
:10AC080016C013F017C014F018C015F0126A12100D
:10AC1800166E1350176E1450186E1550196E0EC01C
:10AC2800D9FF0FC0DAFFDF5016C013F017C014F0B9
:10AC380018C015F0126A1210166E1350176E1450C1
:10AC4800186E1550196E16C00EF017C00FF018C008
:10AC580010F019C011F01200256E2550D8A4040C6C
:10AC68002350241001E1040C55B0030C53B608D04E
:10AC7800090ED8901F36203621362236E82EF9D70D
:10AC8800245006E1020E235C03E2276A110E02D06B
:10AC9800276A120E266E26C028F01FC017F020C0A3
:10ACA80018F021C019F022C01AF028500AEC61F0FF
:10ACB80000091DE11DC00EF01EC00FF0020E116E3E
:10ACC800106A71EC5DF0000908E0020E1E262306EA
:10ACD800D8A0240623502410EDE1120E281807E10D
:10ACE800176A186A196A1A6A0C0E0AEC61F0A5EC60
:10ACF80063F023502410D8A4010C000C26EC61F05A
:10AD0800CC0E35EC63F0660E35EC63F018EC63F0AE
:10AD1800276E275005E1216A226A236A246A1200F5
:10AD2800256A266A2550270FD96EDA6A18EC63F06F
:10AD3800DF6E254A262A26BEF5D7265003E1040EE3
:10AD4800255CF0E3450E00019C6FFC0E9D6F27C04B
:10AD58009EF09F6B28C0A0F0A16B29C0A2F0A36B46
:10AD68002AC0A4F0A56B27C0A6F028C0A7F029C068
:10AD7800A8F02AC0A9F070EC63F02A502910281016
:10AD880003E1060E275CC7E327C021F028C022F0A4
:10AD980029C023F02AC024F01200446A20EE2BF0C8
:10ADA8003A50D9263B50DA223C50DE1809E13D5092
:10ADB800DE1806E13E50DE1803E13F50DE1839E0A8
:10ADC8003AC027F03BC028F03BEC46F0446E4450B4
:10ADD80030E12F0E3A241D6E000E3B201E6E3CC043
:10ADE8001FF03DC020F03EC021F03FC022F0246A91
:10ADF800010E236E20EE01F03A50D9263B50DA229C
:10AE0800DF5030EC56F0000906E03C683D683E68CB
:10AE18003F68010E446E20EE2BF03A50D9263B5085
:10AE2800DA223CC0DEFF3DC0DEFF3EC0DEFF3FC091
:10AE3800DEFF4450120002500209026E040E5260F6
:10AE480033D0350E0E6E0B0E0F6E5250050DCA0E16
:10AE5800F324106E010EF420116E136A050E126EA3
:10AE68007BEC5FF03A0E0E6E0B0E0F6E5250130D08
:10AE7800AA0EF324106E030EF420116E136A130E3B
:10AE8800126E7BEC5FF04D0E0E6E0B0E0F6E525075
:10AE98000D0D900EF324106E020EF420116E136A3D
:10AEA8000D0E126E7BEC5FF0030E526409D0010E9A
:10AEB800506E02011B5110091B6F000EE8CF36FBC4
:10AEC800250E1DEC5BF002928390120003D00E4A0F
:10AED8000F2A102A1050D96EDA6ADF50116E0EC090
:10AEE800F6FF0FC0F7FF000EF86E0E0EF76403D0E2
:10AEF8000800F55005D0F6CFE9FFF7CFEAFFEF508D
:10AF0800111813E10EC0F6FF0FC0F7FF000EF86E20
:10AF18000E0EF76403D00800F55005D0F6CFE9FF10
:10AF2800F7CFEAFFEF500009D2E10EC0F6FF0FC0DD
:10AF3800F7FF000EF86E0E0EF76403D00800F55008
:10AF480005D0F6CFE9FFF7CFEAFFEF50116E1050AA
:10AF5800D96EDA6ADF50115C0E6E0F6AD8A00F0640
:10AF68001200175018100AE140C117F041C118F03B
:10AF78001750181003E1176A186A120017C012F068
:10AF880018C013F019C014F0DEEC5FF01250172649
:10AF98001350182217C0D9FF18C0DAFFDF5006E196
:10AFA8000101406B416B176A186A120017C012F052
:10AFB80018C013F019C014F0FEEC5FF012501724FB
:10AFC8000101406F13501820416F40C1D9FF41C1A2
:10AFD800DAFFDF5009E040C1D9FF41C1DAFF000EB6
:10AFE800DF6A404B412B02D0406B416B17C017F012
:10AFF80018C018F01200A96BAA6B9FC0ABF0A0C0D4
:10B00800ACF0A107D8A0A20727D0A3C074F0A4C0B1
:10B0180075F0A50E766F776B796B010E786FB10EB0
:10B028007A6F7B6BA3EC1AF0B105B2111EE1A55142
:10B03800AD6FAE6BAF6BB06BABC0D9FFACC0DAFF16
:10B04800ADC0DFFFAB4BAC2BA94BAA2B0A0EAD1939
:10B05800AE11AF11B01109E0A151A95DAA51800A42
:10B068004B6EA251800A4B58D0E3ABC0D9FFACC09D
:10B07800DAFFDF6AA951AA1103E19F6BA06B1200E6
:10B088009FC09FF0A0C0A0F01200B3C0B7F0B4C03A
:10B09800B8F0B70E0E6EDCEC48F00EC0BBF00FC077
:10B0A800BCF00001BCBF0B0CD890BB35D96EBC35C9
:10B0B800DA6E4E0ED926010EDA22DECFB9F0DDCFD8
:10B0C800BAF0B951BA1105E0B9C0D9FFBAC0DAFF70
:10B0D800DF6AB151B21105E0B1C0D9FFB2C0DAFFE1
:10B0E800DF6AD890BB35D96EBC35DA6E4E0ED926DC
:10B0F800010EDA22B1C0DEFFB2C0DDFFB55101E1B9
:10B10800000CB30E7C6FB10E7D6F7E6B7F6BAFEC66
:10B1180000F00001B66FB65112000EC015F00FC056
:10B1280016F010C017F011C018F01206D8A01306B8
:10B1380012280CE113280AE10E6A0F6A1200154A58
:10B14800162A174A182A1206D8A0130615C0F6FFA1
:10B1580016C0F7FF0800F55015E017C0D9FF18C052
:10B16800DAFFDF500FE0125013100CE017C0D9FFC0
:10B1780018C0DAFF15C0F6FF16C0F7FFDE50090049
:10B18800F518DDE015C0F6FF16C0F7FF0800F5CF8B
:10B1980014F017C0D9FF18C0DAFFDF50145C0E6E28
:10B1A8000F6AD8A00F061200296E39D020EE01F0E0
:10B1B8002550D9262650DA22DF502D6E20EE03F0D6
:10B1C8002550D9262650DA22DF502C6E20EE05F0C5
:10B1D8002550D9262650DA22DF502B6E20EE07F0B4
:10B1E8002550D9262650DA22DF502A6E2AC011F0BF
:10B1F8002BC012F02CC013F02DC014F01FEF5EF01E
:10B2080025C00EF026C00FF041EC41F00EC02AF028
:10B218000FC02BF010C02CF011C02DF0E7D729502B
:10B22800276E286A2850D8A412002750010ABEE0C9
:10B23800030AE6E0120025EE04F0DE50DE10FBE023
:10B2480000C516F001C517F0060E1624D96E050EB6
:10B258001720DA6EDF50146E060E1624D96E070E0C
:10B268001720DA6EDF50156E164A172A1068010E7D
:10B27800116E16C012F017C013F0105012161150AC
:10B28800131612C000F513C001F5F29E25EE04F066
:10B29800DE06000EDD5AF28E0EC0D9FF0FC0DAFFAF
:10B2A80015C0DFFF25EE04F0010EDBBE05D0000E51
:10B2B800DE5C010EDE5801E2898214501200115042
:10B2C80002E0115003E10F505AEF63F01150D96EAC
:10B2D800DA6A040ED926DE50DE1014E01150D96E59
:10B2E800DA6A040ED9261150E16EE26A020EE126EE
:10B2F800DE50E65CE650800A166EDE50800A16586C
:10B30800D8B012001150D96EDA6A020ED926DECFF3
:10B3180012F0DDCF13F01150D96EDA6ADECF14F0D7
:10B32800DDCF15F012501424D96E13501520DA6EA3
:10B338000FC0DFFF1150D96EDA6A020ED926DE2A55
:10B34800000EDD22000CAF0E00019C6FFD0E9D6FFC
:10B358004AC19EF04BC19FF070EC63F011D0030E10
:10B368000BD0050E236E01014A6B4B6B2DD00A0ED4
:10B3780003D0010E01D0020E236E26D0236A24D0FA
:10B388004AC121F04BC122F0225009E0020A0DE027
:10B398000E0A0FE0010A11E02A0A13E0EFD7215044
:10B3A8000A0ADDE01E0ADDE0E9D72150BC0AE3E025
:10B3B800E5D721501C0ADBE0E1D72150AC0AD9E0DF
:10B3C800DDD721500F0ADAE1235012000E50120285
:10B3D800F3CF16F0F4CF17F0186A196A0E5013025B
:10B3E800F3501726F4501822000E19220F5012029B
:10B3F800F3501726F4501822000E19220E5014028A
:10B40800F3501826F45019220F501302F35018263F
:10B41800F450192210501202F3501826F450192231
:10B4280015500E02F35019260F501402F350192626
:10B4380010501302F350192611501202F350192616
:10B4480016C00EF017C00FF018C010F019C011F098
:10B458001200286A296A0101686B2A6A30D035EC23
:10B468005FF02150221020E02A0E0E6E0F6A1FECAA
:10B4780059F0276E2AA80CD0E80E00019C6FFE0E2A
:10B488009D6F27C09EF09F6B70EC63F083900CD08B
:10B49800000E01016825D96EDA6A040EDA2227C087
:10B4A800DFFF682B284A292A2AAA07D0000E282459
:10B4B800256E040E2920266E12008EAC02D02904B7
:10B4C800CEE328C025F029C026F01200150E146E10
:10B4D800C60EE82EFED7142EFCD700D020D0150EAD
:10B4E800146EC60EE82EFED7142EFCD700D0010E1F
:10B4F8000E6E12C0F6FF13C0F7FF000EF86E0E0EA8
:10B50800F76403D00800F55005D0F6CFE9FFF7CF70
:10B51800EAFFEF50C2EC5EF0124A132AD7D712C0E6
:10B52800F6FF13C0F7FF000EF86E0E0EF76403D097
:10B538000800F55005D0F6CFE9FFF7CFEAFFEF5046
:10B548000009CDE11200838002500209026E5605FF
:10B558000DE1000EE8CF35FB500EE8CF36FB000EAC
:10B56800E8CF37FBE8CF38FB566B1DD02BEE35F014
:10B5780057C1DFFF000EE8CF36FB0D0EE8CF37FBD3
:10B58800000EE8CF38FB8FA403D0600EE8CF38FB5D
:10B598008FA406D037CB0FF0200E0F120FC037FB49
:10B5A800010EE8CF39FB030E8CEC63F0050E1DECA1
:10B5B8005BF002920101576B83901200166A176ABA
:10B5C800186A196A125013101410151029E0010E88
:10B5D8001A6E06D0D89012361336143615361A2A33
:10B5E80015AEF8D7D89016361736183619361250C1
:10B5F8000E5C13500F58145010581550115809E389
:10B6080012500E5E13500F5A1450105A1550115AFA
:10B618001680D89015321432133212321A2EE2D70D
:10B6280016C00EF017C00FF018C010F019C011F0B6
:10B638001200016E00000BEE35F08490849A13908E
:10B64800F29E83A4FED789688EA8FED78EA815D04F
:10B6580001041CE0EE50866E861E8B6A8EA2FED711
:10B6680089908EB2FED78EA4FED78980898A8EB43F
:10B67800FED78EA802D0012EE9D78B68F90E896E05
:10B68800129012981380F28E015012008EA2FED7EB
:10B6980002B2899AEE50866E861E8B6AE1D7000048
:10B6A800032EFDD7000C1A0E17240E6E000E18205C
:10B6B8000F6E91EC61F00EC01DF00FC01EF01F6AF6
:10B6C800206A15C0D9FF16C0DAFF030EDE181CE188
:10B6D800140E17240E6E000E18200F6E91EC61F0F8
:10B6E8000E50196E0F501A6E1B6A1C6A1AC01CF095
:10B6F80019C01BF01A6A196A19501D121A501E1225
:10B708001B501F121C5020121DC015F01EC016F031
:10B718001FC017F020C018F01200166E0C0E161875
:10B7280007E0A5EC63F042EC63F0000901E1FF0CCF
:10B738001650400983EC63F0135083EC63F0125009
:10B7480083EC63F0115083EC63F0105083EC63F0EA
:10B75800010E156E165002E1950E156E080E16189C
:10B7680002E1870E156E155083EC63F00C0E161867
:10B7780002E194EC63F00A0E156E94EC63F0146E1B
:10B7880014AE02D0152EF9D714501200125013100F
:10B79800D8B4000C12C0D9FF13C0DAFFDF5001E1A2
:10B7A800000C12C00EF013C00FF09CEC5FF00EC03E
:10B7B80014F00FC015F0020E1418151001E0000C5B
:10B7C800160E0E6E12C0D9FF13C0DAFFDF5048EC18
:10B7D8005EF00009D8B4000C170E0E6E20EE01F0D2
:10B7E8001250D9261350DA22DF5048EC5EF00009D7
:10B7F80001E1000C1638F00B17101200106E350E10
:10B80800F66EF90EF76E0900F550105C2CE3360E53
:10B81800F66EF90EF76E10500900F55C04E30F6A36
:10B82800010E0E6E010C370EF66EF90EF76E09005A
:10B83800F550105C08E3380EF66EF90EF76E1050EE
:10B848000900F55CECE2390EF66EF90EF76E0900A8
:10B85800F550105C08E33A0EF66EF90EF76E1050CC
:10B868000900F55CDCE20E6A0F6A1200866A846AD7
:10B878008B6889680101686B83928394546B556B5C
:10B8880009D0000E5425D96E040E5521DA6EDF6AF0
:10B89800544B552B55BFF5D75505F3E3546B556BF2
:10B8A80009D0350E5425D96E0B0E5521DA6EDF6A94
:10B8B800544B552B55BFF5D75505F3E30F011769C1
:10B8C800D6501F0B4009D66ED6980F0ED612D588C3
:10B8D800D5120E01C29BD58E0F0C0EC015F00FC0ED
:10B8E80016F010C017F011C018F015C0D9FF16C017
:10B8F800DAFFDF50146E17C0F6FF18C0F7FF000E0E
:10B90800F86E0E0EF76403D00800F55005D0F6CF98
:10B91800E9FFF7CFEAFFEF50145C196E1A6AD8A056
:10B928001A06174A182A154A162A1206D8A0130604
:10B938001250131003E019501A10D7E019C00EF076
:10B948001AC00FF012000EC0D9FF0FC0DAFF10C0E6
:10B95800DFFF0E4A0F2A1150106E1250116E13504D
:10B96800126E136A0EC0D9FF0FC0DAFF10C0DFFFD6
:10B978000E4A0F2A1150106E1250116E1350126E8B
:10B98800136A0EC0D9FF0FC0DAFF10C0DFFF0E4ADE
:10B998000F2A1150106E1250116E1350126E136A46
:10B9A8000EC0D9FF0FC0DAFF10C0DFFF0E4A0F2A02
:10B9B8001200526A030E526401D02AD052500C0D64
:10B9C800030EF324D96E010EF420DA6EDF6A5250AA
:10B9D8000C0D020EF324D96E010EF420DA6EDF6A24
:10B9E80052500C0D000EF324D96E010EF420DA6EBD
:10B9F800DE6ADD6A52500C0D040EF324D96E010E76
:10BA0800F420DA6EDE6ADE6ADE6ADD6A522AD2D78E
:10BA1800526A8390596B12001250131014101510AB
:10BA280023E0010E166E06D0D8901236133614365F
:10BA38001536162A15AEF8D712500E5C13500F584B
:10BA4800145010581550115808E312500E5E135038
:10BA58000F5A1450105A1550115AD89015321432E2
:10BA680013321232162EE8D70EC00EF00FC00FF0A8
:10BA780010C010F011C011F01200526A0E6A0F6A5D
:10BA880052501C0D070EF324D96E020EF420DA6E04
:10BA9800070EDE6AE806FDE252501C0D1B0EF32469
:10BAA800D96E020EF420DA6EDF6A52501C0D170EA2
:10BAB800F324D96E020EF420DA6EDE6ADE6ADE6ADC
:10BAC800DD6A0E4A0F2A0FBEDBD70F5003E1040EC2
:10BAD8000E5CD6E38390506A1200070E136ED00EE8
:10BAE800126E0FD094EC63F0146E14280DE1E40E7E
:10BAF80000D000D0E82EFCD700D000D01206D8A085
:10BB0800130612501310EEE1FE0E141801E0000C9B
:10BB180094EC63F00EC0D9FF0FC0DAFFDF6E0E4A57
:10BB28000F2A1006D8A0110610501110F1E194EC5C
:10BB380063F094EC63F0010C0EC014F00FC015F024
:10BB480013D01206D8A0130610C0D9FF11C0DAFF0F
:10BB5800104A112A14C0E1FF15C0E2FF144A152A41
:10BB6800DFCFE7FFE7500BE01250131008E0E9D7EA
:10BB780014C0D9FF15C0DAFFDF6A144A152A120665
:10BB8800D8A013061228F4E11328F2E1120041ECC0
:10BB980061F0000901E1000C125083EC63F0FD0E26
:10BBA80012181EE0020E146E136A10C0D9FF11C0DD
:10BBB800DAFFDF5083EC63F0104A112A1306D8A08D
:10BBC800140613501410F1E194EC63F094EC63F054
:10BBD80094EC63F0156E15501F0B050A01E0000C7C
:10BBE800010C15D00FC0F6FF10C0F7FF000EF86E5D
:10BBF8000E0EF76403D00800F55005D0F6CFE9FF24
:10BC0800F7CFEAFFEF5065EC63F00F4A102A0FC038
:10BC1800F6FF10C0F7FF000EF86E0E0EF76403D0A3
:10BC28000800F55005D0F6CFE9FFF7CFEAFFEF504F
:10BC38000009D8E1120011C015F012C016F013C0A7
:10BC480017F014C018F026EC61F0CC0E35EC63F058
:10BC5800990E35EC63F00C0E35EC63F0196A1A6A2C
:10BC68001950150FD96EDA6ADF5035EC63F0194AAE
:10BC78001A2A1ABEF5D71A5002E026EF61F0040E10
:10BC8800195CEEE326EF61F00F6E0E5001E1000C37
:10BC98002F0E0F6409D03A0E0F6006D00E50D96EE1
:10BCA800DA6A0F50D00F17D0400E0F6409D0470E34
:10BCB8000F6006D00E50D96EDA6A0F50C90F0BD03C
:10BCC800600E0F64000C670E0F60000C0E50D96EEA
:10BCD800DA6A0F50A90FDF6E010C226E3D0E236E3B
:10BCE800F90E246E216A0AD023C0F6FF24C0F7FF9C
:10BCF800234A242A0800F550F7E1212A2250211866
:10BD080007E023C0F6FF24C0F7FF0800F550ECE178
:10BD1800350E00019C6FFE0E9D6F22C09EF09F6B3A
:10BD280023C0A0F024C0A1F070EF63F0106E310EB4
:10BD3800F66EF90EF76E0900F550105C1CE3320E32
:10BD4800F66EF90EF76E10500900F55C04E30F6A01
:10BD5800010E0E6E010C330EF66EF90EF76E090029
:10BD6800F550105C08E3340EF66EF90EF76E1050BD
:10BD78000900F55CECE20E6A0F6A12000F6E8792FA
:10BD88000A0EE82EFED700D00EB002D0879401D05C
:10BD98008784000E116E010E106E0FAE02D0838ADA
:10BDA80001D0839AD8900F36879000F000F08780F2
:10BDB80000F000F08790104A112A11BEEED71150FA
:10BDC80003E1090E105CE9E38782120001091220E1
:10BDD800010001001700002D119420D00F0001016F
:10BDE800091220010001001700002D119420D00F26
:10BDF800000101091220010001001700002D119413
:10BE080020D00F00010109122001000100170000D5
:10BE18002D119420D00F0001010E0E6E0F6A888636
:10BE28008782878400F000F0879400F000F0106AA1
:10BE3800116A8DA602D00E500F12D8900E36879038
:10BE480000F000F0878000F000F08790104A112A77
:10BE580011BEEFD7115003E1030E105CEAE30F5057
:10BE6800120025EE04F0010EDBBE05D0000EDE5CEC
:10BE7800010EDE5801E2898225EE04F0010EDBBED8
:10BE88000FD0DE28010EDE580BE3D70E00019C6FA1
:10BE9800FC0E9D6F04C59EF005C59FF070EC63F025
:10BEA80004C521F005C522F012009F0E166E176812
:10BEB80014C018F015C019F016501826175019227A
:10BEC800195005E11A0E185C02E2010E01D0000EAD
:10BED8001A6E1B6A1A501B1005E05F0E1414146EBC
:10BEE800156A120014C014F015C015F0120010C025
:10BEF80016F011C017F00EC014F00FC015F010D0D6
:10BF080016C0D9FF17C0DAFFDF50186E164A172A75
:10BF180014C0D9FF15C0DAFF18C0DFFF144A152A6C
:10BF28001206D8A013061228EBE11328E9E1120043
:10BF38000EC010F00FC011F002D00E4A0F2A0EC02A
:10BF4800F6FF0FC0F7FF000EF86E0E0EF76403D071
:10BF58000800F55005D0F6CFE9FFF7CFEAFFEF501C
:10BF68000009EBE110500E5C0E6E11500F580F6E69
:10BF780012000EC014F00FC015F010C016F011C05A
:10BF880017F012501310D8B4120016C0D9FF17C0FA
:10BF9800DAFF14C0E1FF15C0E2FFDFCFE7FF164A62
:10BFA800172A144A152A1206D8A01306125013107D
:10BFB800ECE11200156A166A04D0124A132A154ACF
:10BFC800162A12C0D9FF13C0DAFFDF500EE014C0E2
:10BFD8000EF012C0D9FF13C0DAFFDF500F6E106ADF
:10BFE800DFEC62F00E500F10E8E115C012F016C039
:10BFF80013F01200156A166A04D0124A132A154A59
:10C00800162A12C0D9FF13C0DAFFDF500EE014C0A1
:10C018000EF012C0D9FF13C0DAFFDF500F6E106A9E
:10C02800DFEC62F00E500F10E8E015C012F016C0F9
:10C0380013F012001A0E14240E6E000E15200F6E47
:10C0480016C010F017C011F0B8EC62F012C0D9FF9A
:10C0580013C0DAFF030EDE18D8A41200140E14243D
:10C068000E6E000E15200F6E18C010F019C011F0DA
:10C07800B8EF62F0596B8380838E000E0E6E040E4B
:10C088000F6E116AF60E106E010E136E126AA6EC90
:10C098004AF0270E00019C6FFE0E9D6F70EC63F056
:10C0A800130E9C6FFF0E9D6F70EC63F0839E839060
:10C0B80012000E6E0E500EE0ACEC63F0200EE82E6F
:10C0C800FED7AFEC63F0CC0E00D0E82EFDD700D041
:10C0D80000D01200ACEC63F0C00E00D0E82EFDD703
:10C0E800AFEC63F0350EE82EFED700F012006DC0FD
:10C0F80049F06EC04AF0EEEC46F0716F715112E1F2
:10C108006DC00FF06EC010F06F0E116E86EC55F01A
:10C118000001716F715106E16DC0D9FF6EC0DAFF81
:10C12800DE6ADD6A71511200800E826F7CC083F076
:10C138007DC084F0856B866B876B886B830E766F0A
:10C148007EC077F07FC078F0820E796F23EC05F01F
:10C15800000185517C25D96E86517D21DA6EDF6A12
:10C16800000C000EF2BE010E116E0F50030B7F6E15
:10C178000EC07EFF10C080FF3F0E81168184F29EA4
:10C18800550E826EAA0E826E818281B2FED781948C
:10C1980011B002D0F29E01D0F28E1200350E0E6E52
:10C1A8000B0E0F6E116A106A010E136E126AA6EC5E
:10C1B8004AF002500209026E2BEE35F059C1DFFF3A
:10C1C800226A010E216E7EEC3AF002928380010110
:10C1D800596B120002D00E4A0F2A0EC0F6FF0FC08C
:10C1E800F7FF0800F55009E00EC0F6FF0FC0F7FF93
:10C1F8000800F55010181110EEE10EC0F6FF0FC040
:10C20800F7FF0800F5500E6E0F6A12001B6E1BAE8A
:10C218000ED01B9E106A116A126A136A370E91ECCF
:10C228005BF01C6E010E1C6402D01C50120017C07B
:10C2380010F018C011F019C012F01AC013F01B50FA
:10C2480091EF5BF0ACEC63F00A0E0F6EF80EE82E7F
:10C25800FED70F2EFCD700D0AFEC63F0E00E00D075
:10C26800E82EFDD77AEC63F0090E0F6E840EE82EE7
:10C27800FED70F2EFCD7AFEF63F0130E0F6E880EAC
:10C288000E6E0ED094EC63F0FF0A0DE0E40E00D0C1
:10C2980000D0E82EFCD700D000D00E06D8A00F069C
:10C2A8000E500F10EFE10E500F10D8A4010C000C27
:10C2B800010E146E200E0E180F1011E0F70E106EFE
:10C2C80011680EC012F00FC013F010501226115052
:10C2D8001322135003E1050E125C01E3146A14C023
:10C2E8000EF00F6A120000004F01000F000000005E
:10C2F80009FF0000004F01000F0000000009FF00C7
:10C3080000004F01000F0000000009FF0000004F6F
:10C3180001000F0000000009FF0020EE01F00E50A0
:10C32800D9260F50DA22DF50136E146A0EC0D9FFD7
:10C338000FC0DAFFDF50106E1350116E1050136EDD
:10C3480011C014F013C00EF014C00FF0120060906A
:10C358000F0E0F01596F070E396F356F4F0E936E21
:10C368008A6A8A888A828A82010E8F6E130E0E016B
:10C37800B76F0F0EFA6F100EFC6F140EB86F140C17
:10C388009F0E106E1168200E0E10126E000E0F1008
:10C39800136E1050122611501322135005E11A0E75
:10C3A800125C02E2010E01D0000E0E6E0F6A12003E
:10C3B80021BE04D021500FE120040DE220C022F05C
:10C3C80021C023F0221E231E224A232A22C020F045
:10C3D80023C021F0120020C020F021C021F012005B
:10C3E8001B6A1C6A09D01AC00FF0106A19C011F034
:10C3F80063EC59F01B4A1C2A1B501724D96E1C5099
:10C408001820DA6EDF501A6E1A50EDE11200350B63
:10C418001FE7800102E805800102E805800102E8C3
:10C4280005800102E80568706469736B2E636667AE
:0BC43800004850393132314400000050
:10C44400350E0E6E0B0E0F6E116A106A010E136E0E
:10C45400126AA6EC4AF0010EE8CF35FB025002093D
:10C46400026E010E1DEC5BF0029212009F0E106E24
:10C4740011680EC012F00FC013F0105012261150A4
:10C484001322135005E11A0E125C02E2010E01D0D0
:10C49400000E0E6E0F6A1200BF0E106E11680EC0F1
:10C4A40012F00FC013F01050122611501322135023
:10C4B40005E11A0E125C02E2010E01D0000E0E6EAE
:10C4C4000F6A1200D00E106E11680EC012F00FC069
:10C4D40013F01050122611501322135005E10A0EC6
:10C4E400125C02E2010E01D0000E0E6E0F6A120001
:10C4F4009F869E84090E0E01FD6F9F98890E9B6E88
:10C504009C6A9E989D8E9D889D9AC599F28AF28E0A
:10C514009E909D9C9E9A9E8A1200136A110E126E22
:10C5240009D00A0EE82EFED700D0010E0E6E200EA2
:10C53400C2EC5EF01206D8A013061228F2E113280A
:10C54400F0E112000E6E0E5009E0966A4F0E936EE3
:10C55400220E966E400E956E968A400C966A100EC8
:10C56400966E2A0E966E900E936EF4D70EC0D9FF77
:10C574000FC0DAFF10C0DFFF0E4A0F2A11C010F0FF
:10C58400116A0EC0D9FF0FC0DAFF10C0DFFF0E4AD8
:10C594000F2A1200ACEC63F0200EE82EFED7AFECAD
:10C5A40063F0300EE82EFED77AEC63F00F6EB00E17
:10C5B40000D0E82EFDD70F5012000E50D96EDA6A63
:10C5C4000F50DE1804E10EC00EF00F6A12000E2A9E
:10C5D4000E04D96EDA6ADF50F0E10E6A0F6A1200B7
:10C5E4000EC014F00FC015F014C0D9FF15C0DAFF47
:10C5F40010C0DFFF144A152A1206D8A013061250E1
:10C604001310F2E11200070E8C6E9150070B0E6EA0
:10C61400888A8DAA02D0080E0E26020E0101601926
:10C6240003E10E1C0F0B0E6E0E501200106A116AFD
:10C63400D8901032CCEC62F0000901E0108E112A7F
:10C64400070E1164F5D710501200000EE8CF00F564
:10C65400E8CF01F5E8CF02F5E8CF03F5E8CF04F51C
:10C66400E8CF05F5000C0F6E106A0F50010B5DEC5E
:10C6740060F0D8900F32102A070E1064F6D7070C1A
:10C68400B4EC63F094EC63F041EC61F0000901E078
:10C69400010CA5EC63F0000C0F50030B7F6E0EC071
:10C6A4007EFF3F0E8116818000F000F08050120062
:10C6B4000E6E03D0B6EC63F004000E01CDA9FAD7D8
:10C6C4000EC09AFF12000E6E03D0B6EC63F00400A5
:10C6D4000E01CDA9FAD70EC09AFF12009E0E206E4D
:10C6E4009CC01BF09DC01CF0200E1D6E9CEF23F01F
:10C6F40088888DA803D0010E0E6E01D00E6A0E50EC
:10C7040012000E6E0EC092FF0E01CDA1FDD7CD9189
:10C71400925012000E6E02D0838C839C0E060E285B
:10C72400FBE1120092680E01CDA1FDD7CD9192508C
:10C7340012000E6E0E5001E0010C55501200838061
:10C74400506A83901200B2EC63F094EF63F083902C
:10C75400596B120083988898120083988888120075
:0BC76400858012008590120012000179
:10F9300000819FE0FC407E80FC000020004F4B00D7
:10F940004449534B5F455252004E4F545F5245411C
:10F950004459004E4F5F46494C45004E4F545F4F4F
:10F9600050454E4544004E4F545F454E41424C4534
:10F9700044004E4F5F46494C455F53595354454DE3
:10F9800000000D0A202532582025325820253273D8
:10F9900020253273202532732025327320253273BF
:10F9A00020253273202532732025327320253473AD
:10F9B0002025347320253473202534732025347397
:10F9C00020253473202534732025347320000D0A3C
:10F9D00048504469736B204D6B20494920283138C9
:10F9E0004634364B34302920257320257320257367
:10F9F000205374617274696E672E2E2E0D0A000DED
:10FA00000A4461746120706F7274206973202558F4
:10FA1000202D2053686F756C64206265203C3E2069
:10FA200030784646000D0A5365656B20657272207A
:10FA30002564203E2025642C202564203E2025645A
:10FA40002C202564203E202564000D0A5374617427
:10FA5000757320706F7274206973202558202D20D3
:10FA600053686F756C642062652030784646000DDF
:10FA70000A4461746120706F727420697320255884
:10FA8000202D2053686F756C6420626520307846A5
:10FA900046000D0A526420752025642072746E2081
:10FAA00025642C2025642062797465732072656159
:10FAB000640D0A000D0A4D617820566563746F72FB
:10FAC000206469736B20256420256C642028256CD4
:10FAD000582920000D0A44736B73656C20697320EC
:10FAE00025642C206E756D62657220697320256413
:10FAF0002000466F756E6420616E2052544320666C
:10FB0000696C652061742025580D0A004C6F6F6B7D
:10FB1000696E6720666F7220616E205254432066C2
:10FB2000696C650D0A000D0A5573696E672064697A
:10FB3000736B2067656F6D65747279202573200083
:10FB400046696E6446696C65206661696C6564200F
:10FB50007365617263680D0A000D0A5374617475F0
:10FB60007320706F7274206973202558202D204FE8
:10FB70004B000D0A5365656B20746F20256C642063
:10FB80006661696C6564202564000D0A57726974AA
:10FB9000655F736563746F7273206661696C20259D
:10FBA00064000D0A454550524F4D206469736B2027
:10FBB0006E756D626572202564000D0A4469736B71
:10FBC0002073656C656374206E756D6265722025A7
:10FBD00064005365656B696E6720746F207365639D
:10FBE000746F722025580D0A0046696E6446696C70
:10FBF00065206661696C656420726561640D0A0048
:10FC00000D0A4F70656E696E672065786973746957
:10FC10006E6720257320000D0A4461746120706FA7
:10FC20007274206973202558202D204F4B000D0A37
:10FC3000476F7420256C7520202D207265736574C4
:10FC400074696E67002025582025582025582025E6
:10FC50005820256C752020200A000D0A57726F74F9
:10FC600065206469736B6E6F3A20256420000D0A6D
:10FC700057616974696E6720666F72206361726490
:10FC800020000D0A46696C65202573206973206F7A
:10FC900070656E20000D0A7274635F72656164287E
:10FCA00025642C255829000D0A4F70656E696E6712
:10FCB000206E657720257320000D0A2530325825E7
:10FCC0003032582045786974200020436F6C6420DE
:10FCD00025582C2025582C202558004E6F74206163
:10FCE000204C4946206469736B0D0A000D0A526569
:10FCF000616420646573637269626520000D0A4661
:10FD0000696C6520255820697320257320000D0A31
:10FD10004469736B202558206973202573200020C7
:10FD200041544E20617373657274656420256400CC
:10FD30000D0A48737420627974657332202564005B
:10FD40000D0A5772697465206661696C202564002C
:10FD50000D0A52656164696E67205254430D0A00B2
:10FD60000D0A416D69676F2039313231440D0A0047
:10FD70000D0A53532F38302039313232440D0A00E6
:10FD80000D0A44736B73656C206973202564200031
:10FD90000D0A5265616420256420627974657300E0
:10FDA000566563746F722069732025580D0A000D23
:10FDB0000A53533830657865632025642000222A71
:10FDC0002B2C3A3B3C3D3E3F5B5D7C7F000D0A4F58
:10FDD00070656E696E672025732020000D0A4465EA
:10FDE00062756720697320256420000D0A436C6FDB
:10FDF000636B20697320256420000D0A50726F74B4
:10FE00006F20697320256420000D0A52656164200B
:10FE1000636F6E66696720000D0A46696C656E61E6
:10FE20006D6520257320000D0A466F726D61747434
:10FE3000696E67200072633D25752046525F257309
:10FE40000D0A002A2A204E4F204449534B202A2ACB
:10FE5000002A2A20566572696679202A2A000D0A2E
:10FE600073627974657331202564000D0A417373E0
:10FE700065727420454F49000D0A417373657274B1
:10FE80002041544E000D0A4E6F206361726420259C
:10FE9000640064657363726962652E636667002F30
:10FEA0006C6966646174612E62696E000D0A456E4C
:10FEB00061626C6520505000EB7690455846415485
:10FEC000202020000D0A4D6F756E74696E6720004A
:10FED0004465632020352032303231000D0A4173F1
:10FEE00073657274205050002025582077204154AB
:10FEF0004E20004C6F6164696E672E2E2E002049E3
:10FF00004420255825303258002A2A2052514120B9
:10FF10002A2A00466D742065786974200020476F96
:10FF2000742041544E000D0A53746174757300318E
:10FF3000323A30383A3435005B2532582025645D3A
:10FF4000004572726F722025640048504469736BDB
:10FF500020003C6964656E743E00204944312025D0
:10FF6000580020494432202558004E6F20636172AA
:10FF7000640072633D2564200044534B53454C009C
:10FF80004E414D452558004449534B2558004641A4
:10FF90005433320044454255470050524F544F00AD
:10FFA0005265616479007B4552527D00302E3232B9
:10FFB000004946432000454F49200052454E20004D
:10FFC000535251200044415620004E444143004EBC
:10FFD000524644004641540052544300434C4B00A7
:10FFE000253258004430004431004432004433008C
:0FFFF0004434004435004436004437002B0000F1
:020000040020DA
:10000000FF0FFF0FFF0FFF0FFF0FFF0FFF0FFF0F80
:020000040030CA
:0C0000008CFFFFFC8EFFFFFFFFFFFFFFE7
:00000001FF
